:100000000C94A9060C94DA060C94DA060C94DA0621
:100010000C94DA060C94DA060C94DA060C94DA06E0
:100020000C94DA060C94DA060C94DA060C94DA06D0
:100030000C94DA060C94A2870C94DA060C94DA0677
:100040000C94DA060C94E6850C94DA060C94DA0625
:100050000C94DA060C94DA060C94DA060C941285E9
:100060000C94DA060C94637D0C94397D0C94DA06BA
:100070000C94DA060C94DA060C94DA060C94DA0680
:100080000C94B8850C94DA060C94DA060C94DA0613
:100090000C94DA060C94DA060C94DA060C944A8A6C
:1000A0000C94DA060C94DA060C948A850C94DA0621
:1000B0000C94DA060C94DA060C94DA060C945C853F
:1000C0000C94DA060C94DA060C94DA060C94DA0630
:1000D0000C94DA060C94DA060C94037D0C94D97C0B
:1000E0000C94DA060C9451070C94A6910C94B80861
:1000F0000C9406180C94C0070C9495730C944873D8
:100100000C94A8720C94AA170C9441740C94AE0829
:100110000C9420180C9425740C9482180C94DC0810
:100120000C94131A0C94F8720C9480170C94AA1D5A
:100130000C94BB740C94D5720C9415740C94FE152D
:100140000C94561B0C9431100C9429740C942D743F
:100150000C94DF1B0C94FE190C94F10F0C94A20765
:100160000C94C4070C94541D0C9400740C94E47209
:100170000C9461170C940B7C0C9412740C940A74FC
:100180000C943B740C949E150C94C5960C94D80753
:100190000C94C36A0C94741B0C9445200C94DF07D8
:1001A0000C9451160C94BC710C940E740C94241D78
:1001B0000C94C2740C9441180C941B740C94670733
:1001C0000C947F1D0C94B5070C9445740C94A319E2
:1001D0000C9437740C9442160C94EF740C94337492
:1001E0000C9489160C9411280C944C190C94B80793
:1001F0000C941F740C94276E0C94B3070C94A47287
:100200000C94A7720C947A080C94AE1B0C94991859
:100210000C94A6720C9419160C94A5070C94E10684
:100220000C9481070C94C5190C94A8740C949974BF
:100230000C94FB890C9406740C946B070C9440741A
:100240000C9408280C948C070C94C8070C943597D0
:100250000C94A9070C944E080C9401070C94067397
:100260000C94A5724E414E494E495459494E46CDC3
:10027000CCCC3D0AD7233C17B7D13877CC2B32955D
:1002800095E6241FB14F0A000020410000C842003B
:10029000401C4620BCBE4CCA1B0E5AAEC59D740005
:1002A000407A10F35A00A0724E18090010A5D4E845
:1002B0000000E87648170000E40B54020000CA9AD8
:1002C0003B000000E1F5050000809698000000402A
:1002D000420F000000A0860100000010270000006F
:1002E00000E803000000006400000000000A0000B5
:1002F0000000000100000000002C76D888DC674F69
:100300000823DFC1DFAE59E1B1B796E5E3E453C698
:100310003AE651997696E8E6C28426EB898C9B6290
:10032000ED407C6FFCEFBC9C9F40F2BAA56FA5F43A
:1003300090055A2AF75C936B6CF9676DC11BFCE062
:10034000E40D47FEF520E6B500D0ED902E030094B5
:100350003577050080841E080000204E0A0000004A
:10036000C80C333333330F986E12831141EF8D2154
:1003700014893BE65516CFFEE6DB18D1844B381BBB
:10038000F77C1D901DA4BBE424203284725E228180
:1003900000C9F124ECA1E53D27485454502F312EDB
:1003A00030203430302042616420526571756573AD
:1003B000740D0A5365727665723A205765626475EA
:1003C000696E6F2F312E370D0A436F6E74656E7430
:1003D0002D547970653A20746578742F68746D6C4B
:1003E0000D0A0D0A3C68313E4550494320464149BB
:1003F0004C3C2F68313E00485454502F312E302051
:10040000323030204F4B0D0A5365727665723A20B8
:100410005765626475696E6F2F312E370D0A41631F
:10042000636573732D436F6E74726F6C2D416C6CCA
:100430006F772D4F726967696E3A202A0D0A436FF4
:100440006E74656E742D547970653A2000436F6E3A
:100450006E656374696F6E3A20636C6F73650D0A25
:10046000436F6E74656E742D547970653A206170B7
:10047000706C69636174696F6E2F782D7777772D53
:10048000666F726D2D75726C656E636F6465640066
:10049000506F7374206661696C65640055706C6F91
:1004A0006164204661696C65643A2000234E6F20C8
:1004B00073656E736F7220666F722074656D702045
:1004C000262068756D696469747921004E6F205328
:1004D000656E736F72210020666F722074656D7097
:1004E00020262068756D696469747921002353653D
:1004F0006E736F72204572726F72200053656E7357
:100500006F72204572726F7221002357726F6E678F
:100510002073656E736F7220666F722074656D70E4
:1005200020262068756D6964697479210057726F9F
:100530006E672053656E736F7221004320483D0043
:10054000543D00202020202020202020202020207A
:1005500020202000202020202020202020202020BB
:1005600020202000202020202020202020202020AB
:1005700020202000495020616464726573733A2022
:1005800000496E76616C696420534D207374657008
:10059000732070657220616E676C653D00534D205D
:1005A00073746570732070657220616E676C653D51
:1005B000003C68343E436F70797269676874284301
:1005C000293230323020456455484B204861732031
:1005D00043656E7472652E3C2F68343E3C2F626F0B
:1005E00064793E3C2F68746D6C3E003C703E4C61FB
:1005F0006D7020616E64204F746865722053746161
:10060000747573EFBC9A3C2F703E003C68313E43DA
:10061000616E6E6F74206765742073656E736F72A0
:100620002072656164696E6773213C2F68313E00FA
:100630003C21646F63747970652068746D6C3E3C16
:1006400068746D6C3E3C686561643E3C6D657461C8
:1006500020636861727365743D227574662D38225B
:100660003E3C7469746C653E4F6E6C696E652065C6
:1006700078706572696D656E74206F6E20706F6C36
:100680006172697A6174696F6E206F66206C696748
:1006900068743C2F7469746C653E3C2F68656164B6
:1006A0003E3C626F64793E3C68313E4F6E6C696ED1
:1006B00065206578706572696D656E74206F6E2057
:1006C000706F6C6172697A6174696F6E206F6620F9
:1006D0006C696768743C2F68313E00506172616DCF
:1006E000657465727320726573657420646F6E65DE
:1006F0002100736573757365722F736D6C6967681C
:1007000074706F2F73312F00616E676C65206469A0
:1007100072656374696F6E3A200043757272656E1C
:100720007420534D206973202300534D3A54616265
:100730006C652073746570732070657220616E67DC
:100740006C653D00534D3A506F6C61726F69642067
:1007500073746570732070657220616E676C653D9F
:1007600000234448543D00236E65743D424C4500CF
:10077000236E65743D5769466900236E65743D427A
:1007800054002366747020757365726E616D653AEE
:10079000003A0023486F7374207365727665722087
:1007A000495020616E6420506F72743A0023526584
:1007B0006C617920646576696365733A00235265DC
:1007C0006C617920737461747573206C6162656CFF
:1007D000733A20002352656C6179207374617465EB
:1007E000733A002352656C61792070696E733A0028
:1007F000234E6F2E206F662072656C6179733D0009
:1008000046696E64696E67205769466920495000E1
:100810004E45543D426C7565746F6F7468204C454D
:10082000004E45543D426C7565746F6F7468004EA0
:1008300045543D57694669005344206F70656E20EA
:100840006661696C004E6577206461746120636F36
:100850006C6C656374696F6E207374617274656427
:100860000043757272656E742073657474696E6787
:10087000733A0053797374656D20726573657420E3
:10088000617420002073746570732070657220613C
:100890006E676C653D0020737465707320706572BF
:1008A00020616E676C653D005461626C6520536524
:1008B00074203000235475726E7461626C6520532D
:1008C0006574203000506F6C6172697A65722053D4
:1008D000657420300023506F6C6172697A657220F4
:1008E000536574203000576946692049503A004CDE
:1008F0006F67676572204E616D653A2000526562D0
:100900006F6F74696E672E2E2E0053657276657256
:1009100020506F7274207570646174656400535068
:100920004F52543D004950207570646174656400F5
:100930005349503D0074696D6520696E7465727627
:10094000616C3D0023776562736572766572206223
:100950006567696E73005461626C6520536574202D
:100960003000235475726E7461626C652053657437
:10097000203000506F6C6172697A65722053657423
:1009800020300023506F6C6172697A657220536564
:100990007420300053797374656D207265737461CF
:1009A0007274656421002053797374656D207265DB
:1009B00073746172746564210023436F6D6D616EA1
:1009C00064400054657374204C616D70732F4661F0
:1009D0006E7300444843502053756363657373001E
:1009E00044484350204641494C4544007765627372
:1009F0006572766572202E2E2E006572726F7220DF
:100A00006F70656E696E672066696C653A20004C90
:100A1000616D70204F74686572002354696D6520A4
:100A20002020202020446174652020202020536550
:100A3000636F6E647320506F6C61726F69642054D1
:100A400061626C652054286F43292048282529209D
:100A50002000646F6E652100696E69742E20646FDA
:100A60006E652E00534420696E69742E206661699C
:100A70006C65642100696E69742E206661696C651D
:100A800064210057656C636F6D6520746F20456449
:100A900055484B00496E697469616C697A696E6783
:100AA00020534420636172642E2E2E0075706C6F8B
:100AB000616420627920465450206661696C6564E7
:100AC000210075706C6F616420627920465450205B
:100AD0004F4B21007C3C3E5E2B3D3F2F5B5D3B2C12
:100AE0002A225C00000020002300260029002C00A0
:100AF0002F0032000001000003010601090100007F
:100B00000A0B02090C0D0E08070304010000000087
:100B100000000000000000000000000000000000D5
:100B20000000000000000000000012111000000092
:100B300000000000000000000000000000000000B5
:100B40000000000000000100010010100200010080
:100B50000100B00000001600000028000000100096
:100B60000000200000000100010000000000000063
:100B70000000000000000000000000000000000075
:100B8000000000000000FF000000FFFF0000FFFF6A
:100B90000000FFFF0000CFBF0000C7BF0000C3BFC1
:100BA0000000C1BF0000C0BF000000000000C0BFC7
:100BB0000000C1BF0000C3BF0000C7BF0000CFBF1F
:100BC0000000FFFF0000FFFF000000000000000029
:100BD0000000000000000000000000000000000015
:100BE0000000000000000000000000000000000005
:100BF00000000000000000000000000000000000F5
:100C000000000000000000000000557365722D61B7
:100C100067656E743A202A0D0A446973616C6C6FC3
:100C2000773A202F0D0A004E6574776F726B206D36
:100C300061696E7461696E656420617420000000F2
:100C40002200250028002B002E0031003400020174
:100C50000000050108010B0100002100240027000D
:100C60002A002D00300033000101000004010701BB
:100C70000A010102102020080810204010204080A6
:100C80000201020108040201010204081020408050
:100C900080402010080402018004020180402010DE
:100CA0000804020108040201010204081020408027
:100CB0000102040810204080050505050705080805
:100CC0000808020202020A0A0808040404040101D6
:100CD00001010101010103030303030303030407EB
:100CE00007070C0C0C0C0C0C0C0C02020202060682
:100CF0000606060606060B0B0B0B0B0B0B0B4170C7
:100D000070656E64206D6561732E200053696E6797
:100D10006C65206D6561732E200053617665206DD2
:100D200065617375726520746F3A00202020202061
:100D300020202020202020202020200020202020D3
:100D40002020202020202020202020200000359757
:100D5000C59611241FBECFEFD1E2DEBFCDBF00E0AC
:100D60000CBF1AE0A0E0B2E0EEE2F2E601E00BBF59
:100D700002C007900D92A832B107D9F727E1A8E287
:100D8000BAE001C01D92A631B207E1F716E0C8EA49
:100D9000D6E000E006C021970109802FFE010E94E5
:100DA00078ABC73AD10780E00807A9F70E94EE9A0E
:100DB0000C9405B10C9400008EBD0DB407FEFDCF60
:100DC0000895DC015996ED91FC913097B9F0838933
:100DD0009489A589B6894285538564857585841B68
:100DE000950BA60BB70B811520E89207A105B1055D
:100DF00038F08FEF9FE7A0E0B0E0089590E080E04A
:100E00000895CF93DF931F92CDB7DEB76983DC01DE
:100E1000ED91FC910280F381E02D41E050E0BE01B4
:100E20006F5F7F4F19950F90DF91CF910895FC016F
:100E300020812EBD9B012150310941F051810DB41B
:100E400007FEFDCF4EB55EBD4193F5CF61507109F0
:100E5000860F971F0DB407FEFDCF2EB5FC01208332
:100E60000895E091A40CF091A50C90818091A30CC1
:100E700080958923808308958EBD00000DB407FE00
:100E8000FDCF8EB5089590E02091A60C233339F460
:100E90000C96982F990F990F990F80E00895489616
:100EA000F8CFCF93DF931F92CDB7DEB76983DC0114
:100EB000ED91FC910280F381E02D41E050E0BE0114
:100EC0006F5F7F4F19950F90DF91CF910895FC01CF
:100ED000818D928D0895CF93DF931F92CDB7DEB7AA
:100EE0006983DC01ED91FC910280F381E02D41E00A
:100EF00050E0BE016F5F7F4F19950F90DF91CF914A
:100F00000895FC019485FB018485981303C081E05A
:100F1000983008F080E00895CF93DF931F92CDB70B
:100F2000DEB76983DC01ED91FC910280F381E02D55
:100F300041E050E0BE016F5F7F4F19950F90DF9148
:100F4000CF9108950A960C948C07FC0176876587EB
:100F50000895DC01ED91FC91068CF78DE02D19953B
:100F600091E089270895862F089581E086270895C6
:100F700021E0FC018485883008F020E0822F08956C
:100F8000FC01848595850895FC01848995890895DF
:100F90002CEF33E0FC0131832083FB014089518930
:100FA00062897389FC014283538364837583089546
:100FB000DC01ED91FC91048CF58DE02D199490E00D
:100FC00080E00895CF92DF92EF92FF921F93CF932C
:100FD000DF93EC0180E2689FF0011124E155F34FAB
:100FE0009385917161F0842F827449F080E0DF91E4
:100FF000CF911F91FF90EF90DF90CF900895142F25
:101000006A8B80919E0290919F02A091A002B09164
:10101000A1028E879F87A88BB98BC488D588F12CB5
:10102000E12C7601DD24CC24CF8AD88EE98EFA8E8D
:10103000828D938DB0E0A0E0AC01BD014C295D290B
:101040006E297F294F8B588F698F7A8F838588719E
:10105000B1F4848D958DA68DB78D8B8B9C8BAD8BCC
:10106000BE8B81E08D831F701C831E821F821886B9
:1010700019861A861B861C861D8681E0B8CF8031B2
:1010800009F0B4CF9E012D5E3F4F8B8D9C8D0E9449
:10109000578E882309F4AACF84E0E4CFFC01818D28
:1010A000928D009711F00C94C28E089561E0FC01BE
:1010B00084810C94997DCF93DF93EC018FEF8EBDEB
:1010C0002FEF8F819885AC014F5F5F4F58874F831B
:1010D0008130924028F40DB407FEFDCF2EBDF1CF34
:1010E0000DB407FEFDCFCE010E9456081E82DF918F
:1010F000CF910895CF93DF93EC01E98DFA8D30976E
:1011000049F481E090E09B838A8390E080E0DF9166
:10111000CF91089513821282898D9A8D0E94179023
:10112000E98DFA8D22813381232B59F7F0CFCF93AC
:10113000DF931F92CDB7DEB741E050E0BE016F5F95
:101140007F4F0E94B791019731F4898190E00F9011
:10115000DF91CF9108958FEF9FEFF9CFFC01818D43
:10116000928D009711F00C9497088FEF9FEF0895E0
:101170000F931F93CF93DF93EC01898D9A8D10E02D
:1011800000E0009799F00E9497088C010F3F10072C
:1011900069F0898D9A8DFC0142855385648575853A
:1011A00041505109610971090E94F18EC801DF9116
:1011B000CF911F910F910895CF92DF92EF92FF92FE
:1011C0000F931F93CF93DF93CDB7DEB7AF970FB6D3
:1011D000F894DEBF0FBECDBF7C016A010CEF13E0B7
:1011E0001A8309831C861B8688EE93E0A0E0B0E09A
:1011F0008D879E87AF87B88B86E893E09A8789872B
:10120000188F0F8B198E1A8E1B8E1C8E88E089A367
:101210001BA70AA71CA61DA61EA61FA680917510B7
:1012200090917610A0917710B09178108EA39FA323
:10123000A8A7B9A78B839C83AD83BE8318861F8222
:10124000AE01465D5F4FCE0101960E94B2828130B1
:101250009105B1F4D701ED91FC910488F589E02D59
:101260001DA30CA38CA59DA5AEA5BFA58EA39FA372
:10127000A8A7B9A7A601BE016C5D7F4FC70119954C
:10128000AF960FB6F894DEBF0FBECDBFDF91CF9102
:101290001F910F91FF90EF90DF90CF9008959F9254
:1012A000AF92BF92CF92DF92EF92FF920F931F9374
:1012B000CF93DF935C017B018B01D0E0C0E0F801AC
:1012C00091908F016501CC0EDD1EC6010E94B0A970
:1012D000981621F0692DC6010E94B8A92196CA323C
:1012E000F1E0DF0761F7C701DF91CF911F910F9107
:1012F000FF90EF90DF90CF90BF90AF909F900895B8
:10130000DF92EF92FF920F931F93CF93DF93D82E2C
:101310000CEE1BE0E801EE24E394F12C2296809180
:10132000A8029091A9028E159F059CF061E088812A
:101330000E94B67E6091E70B88810E94997D64EFE0
:1013400071E080E090E00E940C7F8FEFE81AF80ACD
:10135000E5CFDD2009F45EC0CCEEDBE0EE24E394C3
:10136000F12C22968091A8029091A902E816F90624
:101370002CF56091E90B88810E94997D68EE73E0FD
:1013800080E090E00E940C7FAFEFEA1AFA0A6091C9
:10139000E90B8A810E94997D68EE73E080E090E01D
:1013A0000E940C7F6091E70B88810E94997D68EE16
:1013B00073E080E090E00E940C7FD3CF68EE73E092
:1013C00080E090E00E940C7F93E4E92E92E0F92EF9
:1013D000C1E0D0E0B2E0EB0EF11C0E5F1F4F809138
:1013E000A8029091A9028C179D07A4F0D701ED9156
:1013F000FC91EE0FFF1FE951F44F6081F8018081ED
:101400000E94997D68EC70E080E090E00E940C7F83
:101410002196E0CFDF91CF911F910F91FF90EF9038
:10142000DF90089581E08093DD028091DE028823C1
:1014300041F088E080938E1460E083E894E10C949E
:101440005F890895CF93DF93EC01FB0124813581FF
:101450000E94537BCE01DF91CF9108958091DE02EF
:101460008823F9F08091DD028823D9F081E00E9481
:101470008C898BE39FE10197F1F760E080E00E94A7
:101480009D8964E675E083E894E10E94A97C61E0AF
:1014900080E00E949D8964E575E083E894E10C9406
:1014A000A97C08958F929F92AF92BF92CF92DF92C4
:1014B000EF92FF920F931F93CF93DF938C01862FB0
:1014C0000B30110509F09FC090910C14992309F07D
:1014D000F89462E10E943F7FEC0180910C14882314
:1014E00009F07894209701F180E090ECA9E7B4EC42
:1014F0008093FF1390930014A0930114B0930214EF
:101500008093031490930414A0930514B0930614CD
:10151000CE3F8FEFD80709F4A9C0CF3FDC0709F40D
:1015200062C0CCEFDFEF30C1C0910714E090081427
:101530006E2D70E090E080E00E9493A82DEC3CECD2
:101540004CEC5DE30E94F2A84B015C016C2F70E053
:1015500090E080E00E9493A89B01AC01C501B4011A
:101560000E943AAA6093FF137093001480930114B1
:1015700090930214D0910914F0900A146D2F6F7794
:1015800070E090E080E00E9493A84B015C016F2D19
:1015900070E090E080E00E9493A82DEC3CEC4CECD5
:1015A0005DE30E94F2A89B01AC01C501B4010E9459
:1015B0003AAAD7FD26C06093031470930414809355
:1015C000051490930614CE0DCD0FCF0D81E090E061
:1015D00020910B14C21302C090E080E0892B09F423
:1015E00093C0CFEFDFEFCE01DF91CF911F910F912D
:1015F000FF90EF90DF90CF90BF90AF909F908F9033
:1016000008959058D8CFCFEFDFEF0631110509F0DC
:10161000BBC090910C14992309F0F89461E00E94EA
:101620003F7FEC0180910C14882309F07894209777
:1016300001F180E090ECA9E7B4EC8093FF13909364
:101640000014A0930114B093021480930314909398
:101650000414A0930514B0930614CF3FDC0719F2CD
:10166000209709F451C0229609F05BCFCEEFDFEF4F
:101670008BC0C0910814D091071460910714709129
:10168000081476276727762790E080E00E9491A8CB
:101690002DEC3CEC4CEC5DE30E94F2A86093FF1350
:1016A000709300148093011490930214E0900A1434
:1016B000F09009146F2D6F77762F6E2D90E080E0FB
:1016C0000E9491A82DEC3CEC4CEC5DE30E94F2A84A
:1016D000F7FC18C0609303147093041480930514EE
:1016E000909306148C2F8D0F8E0D8F0DC1E0D0E0DE
:1016F00090910B14891302C0D0E0C0E0D195C19540
:10170000D109ABCF9058E6CFC090FF13D090001412
:10171000E0900114F090021420E030E048EC52E434
:10172000C701B6010E944EABD0E0C0E0181614F419
:10173000CBEFDFEF20E030E0A901C701B6010E9446
:101740008CA887FF02C0CAEFDFEFC0900314D090CF
:101750000414E0900514F090061420E030E048EC0A
:1017600052ECC701B6010E948CA887FF02C0C9EFE6
:10177000DFEF20E030E040EF52E4C701B6010E9405
:101780004EAB18160CF483C00C30110509F02BCFAA
:1017900081E08093DF0E8CE58093E10E1092E00EE5
:1017A0001092E20E60E08EE190E10E94EF7481E021
:1017B0000E946F880E94E77E6B017C018091D90EA8
:1017C000811168C081E08093D90E8093D80E9FEF7D
:1017D0009093D70E1092D60E94E09093D50E8093EE
:1017E000B40E8091B40E886B8093B40E8091B30ECA
:1017F000813009F028C11092B30E0E94E77E6B0180
:101800007C018091B40E8093BB008091DB0E90919F
:10181000DC0EA091DD0EB091DE0E892B8A2B8B2B76
:10182000A1F00E94E77E0091DB0E1091DC0E20916A
:10183000DD0E3091DE0E6C197D098E099F090617A9
:1018400017072807390708F446C08091BC0083FDBC
:10185000D8CF85EC8093BC000E94E77E6B017C01B1
:101860008091D90E813009F4F0C08091D60E853078
:1018700008F00DC18091D60EA5EBBEE0E1E1FCE0E1
:1018800090E0981769F12D9121939F5FFACFC8EFEF
:10189000DFEF7ACF8091DB0E9091DC0EA091DD0E10
:1018A000B091DE0E892B8A2B8B2B09F487CF0E94F7
:1018B000E77E0091DB0E1091DC0E2091DD0E309161
:1018C000DE0E6C197D098E099F0906171707280778
:1018D000390708F073CF8091DA0E0E944E8880E0BD
:1018E0001092A20C8093A10C082F10E0CEEFDFEF36
:1018F000882309F478CECDEFDFEF053011050CF425
:1019000072CEC8EEDAE08EE190E10E94A87488877A
:101910002196CE01885E9A4080179107A4F3C0916A
:10192000F00A0091F10A602F70E090E080E00E94E0
:1019300093A82DEC3CEC4CEC5DE30E94F2A86B010B
:101940007C016C2F70E090E080E00E9493A89B01E6
:10195000AC01C701B6010E943AAA6B017C01C0929A
:10196000E80AD092E90AE092EA0AF092EB0AD091F2
:10197000F20A1091F30A6D2F6F7770E090E080E02B
:101980000E9493A84B015C01612F70E090E080E021
:101990000E9493A82DEC3CEC4CEC5DE30E94F2A875
:1019A0009B01AC01C501B4010E943AAAD7FD71C0E8
:1019B0006093EC0A7093ED0A8093EE0A9093EF0A1D
:1019C000C00FCD0FC10F8091F40AC8130ACE20E0DA
:1019D00030E048EC52E4C701B6010E944EABD0E0C3
:1019E000C0E0181614F4CBEFDFEF20E030E040EA5F
:1019F00050E4C701B6010E948CA887FF02C0CAEF5D
:101A0000DFEFC090EC0AD090ED0AE090EE0AF09083
:101A1000EF0A20E030E040EF51ECC701B6010E9430
:101A20008CA887FF02C0C9EFDFEF20E030E040EF75
:101A300052E4C701B6010E944EAB18160CF0D3CD8C
:101A4000C8EFDFEFD0CD85EE05CF8091DB0E909112
:101A5000DC0EA091DD0EB091DE0E892B8A2B8B2B34
:101A600009F4FECE0E94E77E0091DB0E1091DC0EA1
:101A70002091DD0E3091DE0E6C197D098E099F09D3
:101A8000061717072807390708F0EACE24CF85E0A4
:101A9000F3CE90588DCFCF93DF93EC010E94C28E8E
:101AA000882311F01D8281E0DF91CF9108953F924C
:101AB0004F925F926F927F928F929F92AF92BF925E
:101AC000CF92DF92EF92FF920F931F93CF93DF930A
:101AD000CDB7DEB72C970FB6F894DEBF0FBECDBFE3
:101AE0005C01DC015B968D909C905C9716964D9006
:101AF0005D906D907C9019974114510461047104BC
:101B000009F468C0BFEF4B1A5B0A6B0A7B0A312CE1
:101B1000F40181859285A385B4859C01AD012F5F79
:101B20003F4F4F4F5F4F29873A874B875C87730141
:101B300062011D821E821F821886F40181859285B2
:101B4000A385B4852D813E814F815885281739079B
:101B50004A075B0708F056C089859A85AB85BC8526
:101B60008C159D05AE05BF0550F482E0C82ED12C22
:101B7000E12CF12C92E0492E512C612C712C9E010C
:101B80002F5F3F4FB701A601C4010E94D68D882365
:101B9000C9F189819A81AB81BC81892B8A2B8B2BDE
:101BA00009F1260137019FEF491A590A690A790A92
:101BB0002D813E814F8158852F5F3F4F4F4F5F4FA3
:101BC0002D833E834F8358873FEFC31AD30AE30A1E
:101BD000F30AB3CFF40140805180628073803324D4
:101BE000339496CFC414D504E604F70409F70FEF35
:101BF0001FEF2FEF3FE0B701A601C4010E94348D13
:101C0000811119C080E02C960FB6F894DEBF0FBE8C
:101C1000CDBFDF91CF911F910F91FF90EF90DF909B
:101C2000CF90BF90AF909F908F907F906F905F907C
:101C30004F903F900895F5014681578160857185E9
:101C4000411551056105710539F097018601C401FF
:101C50000E94348D8823B1F2D5011696CD92DD9283
:101C6000ED92FC921997332051F0D701C6010196ED
:101C7000A11DB11DF40180839183A283B383F5017B
:101C80008789908DA18DB28D892B8A2B8B2B39F46E
:101C9000C78AD08EE18EF28E84818068848381E051
:101CA000B2CF3F924F925F926F927F928F929F92AC
:101CB000AF92BF92CF92DF92EF92FF920F931F935A
:101CC000CF93DF9300D000D000D01F921F92CDB7EA
:101CD000DEB77C01DC0115968C91811115C0FE01E7
:101CE0003196CE010C966F0130E23193E817F90777
:101CF000E1F7DA0130E087E09D91B92E992329F1CF
:101D00009E3239F48A3011F480E0D9C038E08AE09C
:101D1000F3CFE4EDFAE04491442321F0319694139B
:101D2000FACFF2CF831780F34FED490F4E3560F7AE
:101D30004FE9490F4A3118F440EEB42EB90EF601BE
:101D4000E30FF11DB0823F5FD7CF89818032E1F28E
:101D5000322E8B01FB01838D948DD7015C969C9371
:101D60008E935B97168217821086118612861386D1
:101D700014861586F80182859385A485B5854389E7
:101D800054896589768984179507A607B70708F0EF
:101D90004DC025E0B695A795979587952A95D1F7DB
:101DA000F82FFF70AF2ED80115968C91823008F471
:101DB000ABCFC8010E94970897FDA6CFF801828596
:101DC0009385A485B5854F96A11DB11D8287938704
:101DD000A487B587F0E2AF9EB00111246155734F1F
:101DE0006115710509F490CFDB018C91882341F0D6
:101DF000853E09F057C0BB2029F0BB24B394BACF6D
:101E0000B1100EC0F701A28A80919E0290919F02AC
:101E1000A091A002B091A10286879787A08BB18B79
:101E2000DB018C918111E9CFBB24B394832D8271A6
:101E3000823109F069CFBB2009F459C0C7010E9463
:101E4000F28B009709F460CF20E2FC0111922A95F1
:101E5000E9F72BE0F601DC0101900D922A95E1F7FC
:101E600021E238E2DC0151963C932E93509740E0FA
:101E700058E01F965C934E931E9753963C932E9377
:101E8000529759963C932E93589757965C934E933E
:101E900056970E946E8B882309F436CF432DF701A5
:101EA00062890AC04BE050E0C6010E94AEAD892BAA
:101EB00009F060CF432D6A2DC7010E94E2072B96DF
:101EC0000FB6F894DEBF0FBECDBFDF91CF911F914B
:101ED0000F91FF90EF90DF90CF90BF90AF909F90C9
:101EE0008F907F906F905F904F903F900895F80192
:101EF0008581823009F408CFC8010E94570D8823DC
:101F000009F402CFD8015B96ED91FC915C9716968F
:101F10008D909D90AD90BC901997B2E08B1A91086E
:101F2000A108B108858504C0880C991CAA1CBB1C9B
:101F30008A95D2F786859785A089B189880E991EE2
:101F4000AA1EBB1E848124013501480E511C611C50
:101F5000711C84149504A604B70401F1E1E04E1A43
:101F60005108610871080E946E8B882309F4CCCE59
:101F7000EFEAFCE011928FEA9EE08E179F07D1F7FF
:101F800040929E0250929F026092A0027092A10223
:101F90008091100C81608093100CDBCFD8015B9690
:101FA000ED91FC91258580E092E0A0E0B0E004C0D6
:101FB000880F991FAA1FBB1F2A95D2F7F8014389E2
:101FC000548965897689840F951FA61FB71F838B57
:101FD000948BA58BB68BD70152961C928FEA9CE00E
:101FE00033CFCF93DF93CDB7DEB76D970FB6F894AD
:101FF000DEBF0FBECDBF442391F1AB01BC011C82FB
:102000001B828CE593E09A8389831E8222E0CE01B5
:1020100001960E94510E81110EC090E081E0911155
:1020200001C080E06D960FB6F894DEBF0FBECDBF45
:10203000DF91CF910895CE0101960E94858F88236C
:1020400061F3CE0101960E94F28B009731F325EEE9
:10205000FC0120831E820E946E8B982FDFCF81E0CF
:10206000E1CF1F93CF93DF93CDB7DEB76D970FB658
:10207000F894DEBF0FBECDBFAB011C821B822CE5E6
:1020800033E03A8329831E8221E0BC01CE01019610
:102090000E94510E11E081110CC010E0812F6D964D
:1020A0000FB6F894DEBF0FBECDBFDF91CF911F9169
:1020B0000895CE0101960E944B0DF0CF8FEF0E9444
:1020C000DC068EB508958F929F92AF92BF92FF92D9
:1020D0000F931F93CF93DF93EC01F62E49015A0122
:1020E0008E81882319F0CE010E945B0860E08C810C
:1020F0000E94997D8CE291E00E9497828F2D8064EE
:102100000E94DC0608E110E0D501C401002E04C0E5
:10211000B695A795979587950A94D2F70E94DC0605
:1021200008501109083F8FEF180771F785E9FF2064
:1021300021F088E0F8120DC087E80E94DC0610E06C
:102140000E945E108A8787FF06C01F3F21F01F5F35
:10215000F7CF8FEFF2CFDF91CF911F910F91FF90CB
:10216000BF90AF909F908F900895AF92BF92CF9203
:10217000DF92EF92FF920F931F93CF93DF93EC01C7
:102180006901C801820F931F8130924050F58E8102
:10219000882379F088819981AA81BB81841795076A
:1021A000A607B70731F48F819885C816D90608F0BD
:1021B00042C0488359836A837B838B85833039F09F
:1021C00089E0440F551F661F771F8A95D1F79A0142
:1021D000AB0161E1CE010E946310882389F083E0A6
:1021E0008D83CE010E94560880E0DF91CF911F9130
:1021F0000F91FF90EF90DF90CF90BF90AF90089538
:102200000E94DB815B010E945E108A878F3F69F428
:102210000E94DB816A197B096D327140A0F38FE067
:102220008D83CE010E945608DCCF8E3FB1F4188614
:102230001F8281E08E838FEF8EBD2FEF8F81988577
:102240008C159D0560F40DB407FEFDCF2EBD8F816A
:102250009885019698878F83F1CF8DE0E1CFC801F3
:102260000197F7012FEFAF014E195F094817590782
:1022700038F40DB407FEFDCF3EB531932EBDF3CF3C
:102280000DB407FEFDCF2EB5E80EF91EF701208331
:102290008F819885080F191F18870F8389858823D8
:1022A00019F00115124030F08E81882319F0CE010B
:1022B0000E945B0881E099CF0F931F93CF93DF9328
:1022C000EC01890182E1411551056105710599F023
:1022D0008B85833039F089E0440F551F661F771FC7
:1022E0008A95D1F79A01AB0168E1CE010E94631093
:1022F000882319F084E08D8338C08EEF8EBDF801FD
:10230000C8019E5F0DB407FEFDCF20812EBD0DB428
:1023100007FEFDCF21812EBD3296E817F90791F710
:102320000DB407FEFDCF8FEF0E94DC068FEF0E94F9
:10233000DC060E945E108A878F71853089F488E5FB
:1023400092E00E9497828823A9F020E030E0A90162
:102350006DE0CE010E946310882371F084E1CBCF41
:1023600081E18D83CE010E945608CE010E9456085D
:1023700080E00AC085E1BFCF0E945E108111EECFE0
:10238000CE010E94560881E0DF91CF911F910F91FD
:102390000895FC01DB0112968D919C911397938314
:1023A00082838CE593E09183808314968C911497BB
:1023B000848315968C911597858316964D915D9122
:1023C0006D917C91199746835783608771871A9620
:1023D0004D915D916D917C911D97428753876487E4
:1023E00075871E964D915D916D917C9151974687B1
:1023F0005787608B718B52968C915297828B539634
:102400004D915D916D917C915697438B548B658B6B
:10241000768B57964D915D916D917C915A97478B34
:10242000508F618F728F5B968D919C91948F838F6B
:102430000895DC015996ED91FC91309721F081E0EF
:102440009581911101C080E00895CF93DF93EC0155
:10245000898D9A8D009741F00E944B0D898D9A8D40
:102460000E9437AC1A8E198EDF91CF910895EF92AA
:10247000FF920F931F93CF93DF93EC017B018A01AF
:102480001B821A8288EE93E0A0E0B0E08C839D83EB
:10249000AE83BF838EED93E0998388838DE190E0D6
:1024A0000E949BAB9A8F898F009779F02DE1F701FD
:1024B000DC0101900D922A95E1F74CE050E0B80163
:1024C000CE010C960E9406AE188EDF91CF911F911F
:1024D0000F91FF90EF900895E091A40CF091A50C5E
:1024E00080819091A30C892B80830895AF92BF9235
:1024F000CF92DF92EF92FF920F931F93CF93DF93D0
:1025000000D01F92CDB7DEB78C016B017A018091AC
:10251000A60C8333E9F45B016801C40ED51EC01616
:10252000D106A9F10E9431078FE00E943C07812F5C
:102530000E943C07802F0E943C070F5F1F4F80E0E6
:102540000E943C07F50181935F010E946C12E7CF66
:10255000843369F50E94310719830A838F2D8F77A1
:102560008B83EC8264E070E0CE0101960E94170735
:10257000A70170E060E0C6010E94D6ADE114F1044D
:1025800021F0B701C6010E9417070E946C12C70113
:102590000F900F900F900F90DF91CF911F910F919F
:1025A000FF90EF90DF90CF90BF90AF9008950E9482
:1025B00031070F3F110509F030F419820A831B829D
:1025C00063E070E0D1CF17FD0BC019820A8333E0BE
:1025D000169507953A95E1F7007E08600B83F0CFDA
:1025E000C80126E0969587952A95E1F7807E1983A4
:1025F0000A830115104C18F480618B83E1CF886148
:10260000FCCFCF93DF931F92CDB7DEB72091A70CFD
:1026100030E0322F2227260F371F90E0982F88278F
:1026200041E050E0BE016F5F7F4F820F931F0E9419
:10263000761289810F90DF91CF910895AF92BF926A
:10264000CF92DF92EF92FF920F931F93CF93DF937E
:1026500000D000D01F921F92CDB7DEB78C017B0156
:102660006A018091A60C8333E1F45801A40EB51ED3
:10267000A016B10609F46FC00E94310780EF0E94D6
:102680003C07812F0E943C07802F0E943C070F5F70
:102690001F4FF70181917F010E943C070E946C123D
:1026A000E7CF5B01A40EB51E8433C1F40E9431074D
:1026B00019830A838D2D80688B83CC8264E070E05F
:1026C000CE0101960E941707AE14BF0409F441C061
:1026D000F70181917F010E943C07F6CF0E943107EC
:1026E0000F3F110509F028F419820A8384E08B83D7
:1026F0000CC017FD17C019820A8333E016950795A1
:102700003A95E1F7007E0C600B8386E0C816D10491
:10271000A0F5F701DE011496EA15FB0599F0819109
:102720008D93FACFC80126E0969587952A95E1F713
:10273000807E19830A830115104C10F48461D7CF71
:102740008C61D5CFB6016D5F7F4FCE0101960E949F
:1027500017070E946C12C60128960FB6F894DEBFC8
:102760000FBECDBFDF91CF911F910F91FF90EF90E2
:10277000DF90CF90BF90AF90089563E070E0CE01FE
:1027800001960E941707F70181917F010E943C0783
:10279000AE14BF04C1F7DDCFCF93DF931F92CDB747
:1027A000DEB741E050E0BE016F5F7F4F90E080E018
:1027B0000E94761289810F90DF91CF910895CF9377
:1027C000DF93C4E1D0E00E94CC13882361F061E084
:1027D00070E080E090E00E940C7F2197A1F780E0FC
:1027E000DF91CF91089581E0FBCFCF93DF931F92CC
:1027F000CDB7DEB7898341E050E0BE016F5F7F4F08
:1028000090E080E00E941E130F90DF91CF91089519
:1028100063E070E00C940113DA01E091A70CF0E0A2
:10282000FE2FEE27E60FF71F90E0982F8827A901CB
:10283000BD018E0F9F1F0C941E13CF93DF931F9229
:102840001F92CDB7DEB779836A8322E030E0AE0114
:102850004F5F5F4F60E170E00E940C140F900F908B
:10286000DF91CF910895CF93DF931F921F92CDB741
:10287000DEB779836A8322E030E0AE014F5F5F4FBD
:1028800064E070E00E940C140F900F90DF91CF91E4
:102890000895CF93DF931F92CDB7DEB72091A70C99
:1028A00030E0322F2227260F371F90E0982F8827FD
:1028B000498341E050E0BE016F5F7F4F820F931F5D
:1028C0000E941E130F90DF91CF910895CF93C82FD0
:1028D000462F61E070E00E94491461E070E08C2FA7
:1028E0000E9401138111F9CFCF910895DA01E0918F
:1028F000A70CF0E0FE2FEE27E60FF71F90E0982FD1
:102900008827A901BD018E0F9F1F0C9476126F922C
:102910007F929F92AF92BF92CF92DF92EF92FF92FF
:102920000F931F93CF93DF931F921F92CDB7DEB704
:10293000982E8B013A01690122E030E0AE014F5F31
:102940005F4F64E270E00E947614E980FA80FE2412
:10295000EF24FE24E00EF11E970137704091A60C83
:10296000092D10E0C801433309F04CC00896982F98
:102970008827990F990F990F820F931F473309F4F6
:1029800046C0A9014C0D5D1D4130584008F43FC0C0
:1029900060E078E05B01A21AB30AA501B3010E94CE
:1029A0001E13A6014A195B09B3016A0D7B1D8091B4
:1029B000A60C833349F5085F1F4F000F000F000F6F
:1029C00080E0902F0E941E13EC0CFD1CF982EA821D
:1029D00022E030E0AE014F5F5F4F64E270E0892D8E
:1029E0000E940C140F900F90DF91CF911F910F91C7
:1029F000FF90EF90DF90CF90BF90AF909F907F902F
:102A00006F9008954096B3CF005F1F4FD6CFA601B9
:102A1000B301D8CFEF92FF921F93CF93DF931F9212
:102A20001F92CDB7DEB7182F22E030E0AE014F5F26
:102A30005F4F60E270E00E947614E980FA80FE2425
:102A4000EF24FE2422E030E0AE014F5F5F4F60E2F2
:102A500070E0812F0E94761489819A8198278927B6
:102A60009827E816F90689F487E0189FF0011124E9
:102A7000E75AF34FF582E482C7010F900F90DF9180
:102A8000CF911F91FF90EF9008957C01DBCFFF92D3
:102A90000F931F93CF93DF931F921F92CDB7DEB793
:102AA000F82E22E030E0AE014F5F5F4F66E270E04B
:102AB0000E94761409811A8110270127102722E02D
:102AC00030E0AE014F5F5F4F66E270E08F2D0E94F5
:102AD000761489819A8198278927982708171907DA
:102AE00049F4C8010F900F90DF91CF911F910F9182
:102AF000FF9008958C01E3CF44E050E0BC018FE0EB
:102B000090E00C941E1308951F93CF93DF93182F1A
:102B100080E591E00E94A775812F0E940A15EC01C3
:102B2000812F0E940814873121F08C3111F0D0E000
:102B3000C0E0CE01DF91CF911F910895FC01848503
:102B4000883010F40C94841590E080E00895CF92C2
:102B5000DF92EF92FF921F93CF93DF93182F7B01A9
:102B6000EA014130584010F0C0E0D8E080E591E043
:102B70000E94A775812F0E940A156C01812F0E9467
:102B80000814873111F08C3121F5CC16DD0670F375
:102B900080E591E00E94A7759E01A70170E060E0CA
:102BA000812F0E94871460E270E0812F0E946614DA
:102BB00062E070E0812F0E94011384FD0DC0812F1F
:102BC0000E9408148823B9F080E591E00E94A7755F
:102BD000EFCFD0E0C0E0DCCF40E162E070E0812FD9
:102BE0000E944914CE01DF91CF911F91FF90EF9089
:102BF000DF90CF900895D0E0C0E0F4CF0F931F9303
:102C0000CF93DF938C01EA01FC018485883048F47E
:102C10000E94A715892B39F481E090E0F801938395
:102C20008283D0E0C0E0CE01DF91CF911F910F9160
:102C300008950A960C94FE151F93CF93DF931F926D
:102C4000CDB7DEB7182F80E591E00E94A775812FE0
:102C50000E94430727E0129FF0011124E75AF34F27
:102C600022813381377041E050E0BE016F5F7F4FBA
:102C7000820F931F0E94761289810F90DF91CF916E
:102C80001F910895FC01808D883040F4218D328D94
:102C9000232B21F00E941C1690E008958FEF9FEFE8
:102CA0000895CF93DF93FC012485283028F08FEF1F
:102CB0009FEFDF91CF910895EC010190F081E02D1D
:102CC0000084F185E02D1995892B89F38C850E946C
:102CD0001C1690E0EECF1F93CF93DF93182F87E061
:102CE000189FE0011124C75AD34F8881998100971A
:102CF00061F480E591E00E94A775812F0E9447153D
:102D00002E81821B910999838883DF91CF911F9136
:102D10000895FC018485883010F40C946B1690E0C3
:102D200080E008954F925F927F928F929F92AF9230
:102D3000BF92CF92DF92EF92FF920F931F93CF93A8
:102D4000DF931F921F92CDB7DEB7782E6B014A0139
:102D5000A82EB12C27E0829FC0011124FC01E75A64
:102D6000F34F7F010081118180E591E00E94A775FA
:102D70000815190554F4872D0E944715F70126817F
:102D80008C01021B1109118300830115110519F52E
:102D9000872D0E940814843159F0882349F001E0FE
:102DA00010E08C3111F410E000E01195019511094B
:102DB000C8010F900F90DF91CF911F910F91FF905D
:102DC000EF90DF90CF90BF90AF909F908F907F90CB
:102DD0005F904F900895801691060CF4840187E06F
:102DE0008A9DF0018B9DF00D1124E75AF34FE2808C
:102DF000F380C114D10451F12701F7E05F22872D40
:102E00000E944307840D951D2091A60C273309F4D9
:102E100053C09801240D351D2130384008F44CC0B2
:102E200020E038E0490184189508A401B6010E9409
:102E300076122601480C591C6801C818D908872D3C
:102E40000E944307A601B2010E947612E00EF11E15
:102E500087E08A9DF0018B9DF00D1124E75AF34F16
:102E6000F382E28220813181201B310B3183208368
:102E70008681800F912F911D8A3F910510F4232B9D
:102E8000F1F487E08A9DF0018B9DF00D1124E75A43
:102E9000F34F1682F982EA8222E030E0AE014F5F02
:102EA0005F4F68E270E0872D0E940C1460E470E0D0
:102EB000872D0E9466147CCFA801B601C5CF8683FA
:102EC00077CFCF93DF93FC01218D328D2115310512
:102ED00029F48FEF9FEFDF91CF910895EC01808D62
:102EE0004217530708F0A9010E94921618161906F6
:102EF00084F7298D3A8D281B390B3A8F298FEBCF18
:102F00000F931F93CF93DF931F92CDB7DEB7FC01D2
:102F1000218D328D232B41F48FEF9FEF0F90DF91A6
:102F2000CF911F910F9108958C0141E050E0BE01B7
:102F30006F5F7F4FFC01808D0E9492161816190654
:102F40005CF7F801818D928D0197928F818F898135
:102F500090E0E4CF0F931F93CF93DF9300D000D086
:102F60001F921F92CDB7DEB78C01D80159964D91B3
:102F70005C915A974115510551F0ED91FC91048CEB
:102F8000F58DE02D70E060E0C8011995EECFF801F5
:102F9000808D0E946B16892BB1F148E050E0BE0194
:102FA0006F5F7F4FD80158968C910E949216181629
:102FB0001906F4F4D801509684E0FE013196019090
:102FC0000D928A95E1F78D8190E0982F88272E81C8
:102FD000820F911DF801958B848B8F81282F30E013
:102FE000322F22278885820F932F911D928F818FF8
:102FF00028960FB6F894DEBF0FBECDBFDF91CF91FC
:103000001F910F91089590E080E0F2CFCF93DF936E
:103010001F92CDB7DEB741E050E0BE016F5F7F4F3A
:10302000FC0184850E9492161816190634F48981D1
:1030300090E00F90DF91CF9108958FEF9FEFF9CF40
:10304000FC018485883010F40C94921690E080E0A6
:103050000895CF93C82F80E591E00E94A77568E09E
:1030600070E08C2FCF910C946614CF93C82F80E51D
:1030700091E00E94A77560E170E08C2FCF910C94D5
:103080006614CF92DF92EF92FF920F931F93CF932C
:10309000DF9300D000D0CDB7DEB78C016B017A0191
:1030A000FC01808D883010F40E9435188CEF93E07D
:1030B0009A838983F60182819381A481B5818B8370
:1030C0009C83AD83BE83B701CE0101960E949377A6
:1030D000F801808F8830A0F4F586E486128E118E78
:1030E00081E026960FB6F894DEBF0FBECDBFDF910C
:1030F000CF911F910F91FF90EF90DF90CF900895A7
:1031000080E0EFCFCF93DF93EC01888D883020F4FF
:103110000E94351888E0888FDF91CF910895CF9372
:10312000C82F80E591E00E94A7758C2FCF910C9459
:103130000814EF92FF920F931F93CF93DF937C01BC
:103140008091A60CD4E0833309F0D8E001E91CE0BB
:10315000C0E0F801219131918F01F70184819581BF
:103160002817390729F0CF5FDC13F3CF80E006C0C2
:103170008C2F0E948F188431B1F781E0DF91CF91BD
:103180001F910F91FF90EF9008959F92AF92BF9281
:10319000CF92DF92EF92FF920F931F93CF93DF9323
:1031A000EC017B018091A60C811121C01B821A8247
:1031B00088EE93E0A0E0B0E08C839D83AE83BF8374
:1031C00080EB93E09983888388E08C8788EE93E096
:1031D0009E878D87CE01DF91CF911F910F91FF9038
:1031E000EF90DF90CF90BF90AF909F90089534E024
:1031F000932E833311F028E0922E81E9C82E8CE0C3
:10320000D82E10E098E0B92EA12CD6012D913D9139
:103210006D01F701848195812817390791F4812F79
:103220000E948F18082F873111F08C3139F5812FCA
:103230000E946B16892B59F50C3119F4812F0E94CD
:1032400029181F5F9112E1CFA11008C0D701ED919D
:10325000FC910084F185E02DC70119951B821A822B
:1032600088EE93E0A0E0B0E08C839D83AE83BF83C3
:1032700080EB93E099838883BC86A8CF843149F0A2
:103280008111DFCFF601329711821082DACFB12E91
:10329000D8CFAA24A394D5CF8F929F92AF92BF92FA
:1032A000CF92DF92EF92FF920F931F93CF93DF9312
:1032B000CDB7DEB72F970FB6F894DEBF0FBECDBFE8
:1032C0005C014B017A018091A60C8823C9F104E0CE
:1032D000833309F008E0B501CE0101960E94C518BC
:1032E00081E9C82E8CE0D82E10E0F60121913191B1
:1032F0006F01F501848195812817390751F4812FD9
:103300000E948F18873129F4A701B401812F0E94F0
:10331000A7151F5F0113E9CFC7012F960FB6F894C9
:10332000DEBF0FBECDBFDF91CF911F910F91FF90F8
:10333000EF90DF90CF90BF90AF909F908F900895C7
:10334000F12CE12CE9CFCF93DF93EC018C85883011
:10335000D0F40E948F18843189F0882379F0883165
:1033600069F021E08C3159F4E881F9810084F1851C
:10337000E02DCE01199521E0892B09F420E0822F60
:10338000DF91CF91089580E0FBCFCF92DF92EF9253
:10339000FF92CF93DF93EC018C85883068F40E9414
:1033A00029180E94DB816B017C018C850E948F189B
:1033B000811109C088E08C87DF91CF91FF90EF9059
:1033C000DF90CF90089561E070E080E090E00E948F
:1033D0000C7F0E94DB81AB01BC014C195D096E09B9
:1033E0007F098D859E85B0E0A0E0481759076A07E0
:1033F0007B07D8F28C850E943518DCCFCF93DF9302
:10340000EC018C85883060F40E948F18873111F0B0
:103410008C3131F48C850E9484158115984088F395
:10342000DF91CF910895CF92DF92EF92FF920F93A9
:103430001F93CF93DF93CDB7DEB7AF970FB6F89456
:10344000DEBF0FBECDBF8C016B017A018CEF93E024
:103450009A8389831B821C821D821E821C861B8686
:1034600048EE53E060E070E04D875E876F87788BB1
:1034700026E833E03A872987988F8F8B198E1A8E2A
:103480001B8E1C8E28E029A39BA78AA71CA61DA61D
:103490001EA61FA6D8011C968C91883060F40E944D
:1034A0008F18882321F0F80184850E94291888E06C
:1034B000D8011C968C938091751090917610A091F4
:1034C0007710B09178108EA39FA3A8A7B9A78B837C
:1034D0009C83AD83BE8318861F82AE01465D5F4F1D
:1034E000B601CE0101960E94B2820097C1F0D801C8
:1034F000ED91FC910684F785E02D8CEF93E09DA380
:103500008CA38CA59DA5AEA5BFA58EA39FA3A8A7A0
:10351000B9A7A701BE016C5D7F4FC8011995AF9691
:103520000FB6F894DEBF0FBECDBFDF91CF911F91D4
:103530000F91FF90EF90DF90CF9008958F929F9220
:10354000AF92BF92CF92DF92EF92FF920F931F93B1
:10355000CF93DF9300D000D000D01F92CDB7DEB75D
:103560009091A60C911115C018E0812F2A960FB6E4
:10357000F894DEBF0FBECDBFDF91CF911F910F91A9
:10358000FF90EF90DF90CF90BF90AF909F908F9083
:10359000089528E0F22E933311F494E0F92E6B0194
:1035A000082F80E591E00E94A7759E012F5F3F4F95
:1035B0005901490110E0812F0E940814F401819300
:1035C0004F018823C1F01F5FF112F5CFF12CF501F7
:1035D00091915F019D3149F0983139F09A519230C3
:1035E00020F0F3941F11F3CFBFCF60E170E08F2D77
:1035F0000E9466141F2DE12EF12CF701EE0FFF1F24
:10360000EF56F34F1182108283EE93E00197F1F7AA
:10361000402F70E060E0812F0E9449144FEF62E07C
:1036200070E0812F0E944914B601CD2889F4809161
:10363000AE029091AF0201968115F0EC9F0798F1D0
:103640009093AF028093AE026091AE027091AF0290
:10365000812F0E94331461E070E0812F0E94661474
:1036600027E02E9DC0012F9D900D11249C01275A0B
:10367000334F7901F9011182108222E030E0AE016E
:10368000475F5F4F68E270E0812F0E947614898562
:103690009A85982789279827F70193838283168232
:1036A0001582148262CF80E090ECCACF0F931F93F3
:1036B000CF93DF93EC018B01888D883010F40E944A
:1036C0003518B80182E00E949E1A888F883050F425
:1036D0001D870C871A8E198E81E0DF91CF911F9183
:1036E0000F91089580E0F9CF9F92AF92BF92CF9251
:1036F000DF92EF92FF920F931F93CF93DF938C0192
:103700005B01942EE52EFC01C688D788F08C80E5FD
:1037100091E00E94A7758F2D0E940A15C92DDE2DFC
:103720008C179D0708F4EC019E01A501B6018F2DB1
:103730000E948714F801868997898C0F9D1F978BAB
:10374000868BCE01DF91CF911F910F91FF90EF906B
:10375000DF90CF90BF90AF909F900895CF93FC01E2
:10376000C08D80E591E00E94A77560E270E08C2F2B
:103770000E94661462E070E08C2F0E94011384FDA9
:1037800016C062E070E08C2F0E94011383FF0AC014
:1037900048E162E070E08C2F0E94491480E090E0E4
:1037A000CF91089580E591E00E94A775E3CF40E1B5
:1037B00062E070E08C2F0E94491481E0F0CFFF920C
:1037C0000F931F93CF93DF93EB01FC01178A168AA7
:1037D0002A81211109C02B81211106C02C812111C0
:1037E00003C02D81222301F141155105E9F08A0121
:1037F000FC01F08C80E591E00E94A775AE014E5F60
:103800005F4F24E030E06CE070E08F2D0E940C14DC
:10381000B8018F2D0E941D1481E090E0DF91CF91BF
:103820001F910F91FF90089580E0F7CF7F928F92C4
:103830009F92AF92BF92CF92DF92EF92FF920F933F
:103840001F93CF93DF93CDB7DEB7A6970FB6F8944B
:10385000DEBF0FBECDBF8C01762E942E852E20E2CA
:10386000A22ECE0101967C01DC01EA2D1D92EA9583
:10387000E9F76801F3E4CF0ED11C8CEF93E09AA333
:1038800089A38FEF8BA38CA38DA38EA343E450E079
:10389000BE016F5D7F4FC6010E94DF1B019609F4D8
:1038A000BFC081E089838A8386E0B82EBB821C82F8
:1038B000D80114966D917D918D919C9117970E94DE
:1038C00080AB6D837E838F83988789869A8680E814
:1038D00090E09C878B874CE150E0B701C6010E94C5
:1038E000741BFE0137968AE1DF011D928A95E9F784
:1038F0004801B8E08B0E911CF401D70101900D92A4
:10390000BA94E1F740E150E0B701C6010E94741B90
:10391000F7011192AA94E9F796E0A92EB12C40E2A2
:1039200050E0B701C6010E94741BF1E0AF1AB10864
:10393000B1F783E6898392E89A8393E59B838C832E
:1039400085E38D8381E08E837F829DE3988797E076
:1039500099878A8786E0F401DE011B9601900D921B
:103960008A95E1F78CE0898B8A8B6EEF73E0CE014C
:1039700043960E94F1ADD8011B966C91CE014996F9
:103980000E94D076F8016485CE014B960E94D076D5
:10399000D8011D966C91CE014D960E94D0764EE1D5
:1039A00050E0B701C6010E94741BB3E07B121EC039
:1039B00082E3898384E08A83F80196859B839785D7
:1039C0009C8390899D8391899E8396E39F838887BA
:1039D000828D8987838D8A87848D8B87858D8C875F
:1039E0004CE050E0B701C6010E94741B87E3898355
:1039F00086E08A8391E09B8393E09C838D838FE0B4
:103A00008E838AE38F838BE388878FEF898749E0F2
:103A100050E0B701C6010E94741BC6010E94AE1B94
:103A2000A6960FB6F894DEBF0FBECDBFDF91CF9143
:103A30001F910F91FF90EF90DF90CF90BF90AF90CC
:103A40009F908F907F9008950F931F93CF938C0139
:103A5000FC016481758181E20E949E1AC82F883022
:103A6000F8F480E591E00E94A7758C2F0E9408145D
:103A7000833131F08C2FCF911F910F910C94291825
:103A800062E070E08C2F0E946614F80184819581B9
:103A9000EC2FF0E0EE0FFF1FEF56F34F9183808382
:103AA000CF911F910F9108950F931F93CF93DF93A1
:103AB0001F921F92CDB7DEB7FC0124852830E0F4B9
:103AC0008C0180E591E00E94A77522E030E0AE0114
:103AD0004F5F5F4F60E170E0F80184850E947614CB
:103AE00089819A819827892798270F900F90DF91D5
:103AF000CF911F910F91089590E080E0F6CF0F9342
:103B00001F93CF93DF931F921F92CDB7DEB7FC01B7
:103B100024852830E0F48C0180E591E00E94A775AF
:103B200022E030E0AE014F5F5F4F64E070E0F801EB
:103B300084850E94761489819A81982789279827FD
:103B40000F900F90DF91CF911F910F91089590E00A
:103B500080E0F6CFCF92DF92EF92FF921F93CF9348
:103B6000DF93EC017B016A018C85883048F40E9468
:103B70008F18882319F08C850E94291888E08C877B
:103B8000F70182819381A481B5810097A105B105D8
:103B900051F490E080E0DF91CF911F91FF90EF9082
:103BA000DF90CF9008958F3F9F4FAF4FBF4F89F366
:103BB00070E060E081E20E949E1A182F8C878830A6
:103BC00040F780E591E00E94A775A7014E5F5F4F27
:103BD00024E030E06CE070E0812F0E940C14B6010C
:103BE000812F0E941D1464E070E0812F0E946614F2
:103BF0000E94DB816B017C018C850E948F188731CC
:103C000011F18C3101F1882321F20E94DB81AB019B
:103C1000BC014C195D096E097F098D859E85B0E058
:103C2000A0E084179507A607B70738F061E070E0B9
:103C300080E090E00E940C7FDFCF8C850E943518D9
:103C400088E08C87A6CF81E090E0A5CFCF93DF936B
:103C5000EC018CEF93E0998388831A821B821C828B
:103C60001D8280E591E00E94A775BE016E5F7F4FC7
:103C700044E050E08FE090E00E947612CE01DF91A8
:103C8000CF9108954F925F926F927F928F929F9201
:103C9000AF92BF92CF92DF92EF92FF920F931F935A
:103CA000CF93DF93EC018090A8029090A902E5E405
:103CB000F2E081E090E0512C412C8816990654F0F6
:103CC000219131912130310519F42FEF421A520A16
:103CD0000196F3CF1C161D060CF04AC08C169D06EB
:103CE0000CF446C04E018E01000F111F7E01EE0C38
:103CF000FF1CEE0CFF1C8C169D060CF4D9C0C701EE
:103D0000895C9D4F6C01FC0180819181A281B3810E
:103D10009701215B3D4F5901181619061A061B061B
:103D200054F50E943986F501208131814281538109
:103D3000621B730B840B950BF6012081318142814C
:103D40005381261737074807590758F41082118204
:103D5000128213820E943986F50160837183828307
:103D6000938321960E5F1F4FF4E0EF0EF11CC3CF3B
:103D7000C1E0D0E0B8CF98012E553D4F3901F9018F
:103D80008081918198012D5B3D4F6901F90120816E
:103D9000318182179307F1F0F3E04F16510414F0CC
:103DA0000097C1F4880F991FFC01E951F44F60811D
:103DB000F801E451F44F80810E94997DF3018081E4
:103DC0009181F601918380836CE271E080E090E064
:103DD0000E940C7FF50180819181A281B381181628
:103DE00019061A061B060CF0BCCF0E943986F50195
:103DF0002081318142815381621B730B840B950BAF
:103E0000F701E55AFD4F2081318142815381261708
:103E100037074807590708F0A4CFF501108211822F
:103E2000128213829801275B3D4F5901F90180816D
:103E30009181F601208131818217930709F491CF96
:103E40006091A8027091A902E5E4F2E041E050E03F
:103E500030E020E0641775074CF0A191B191119703
:103E600011F42F5F3F4F4F5F5F4FF4CF2330310589
:103E70001CF0009709F075CF880F991FFC01E951DC
:103E8000F44F6081F801E451F44F80810E94997DE4
:103E9000F50180819181F60191838083F301918303
:103EA00080836CE271E080E090E00E940C7F59CF4B
:103EB000DF91CF911F910F91FF90EF90DF90CF9006
:103EC000BF90AF909F908F907F906F905F904F903A
:103ED0000895CF93DF93FC0124813581232B69F072
:103EE000EC01BC0181E89FE00E94957CBE0184EE5C
:103EF0009EE0DF91CF910C94957CDF91CF91089556
:103F0000CF93DF93FC0124813581232B69F0EC01F1
:103F1000BC0181E89FE00E94877CBE0184EE9EE0A8
:103F2000DF91CF910C94877CDF91CF910895CF934F
:103F3000DF93FB0122813381DC0113963C932E93A6
:103F40001297448155816681778114964D935D93D4
:103F50006D937C931797408551856285738518967C
:103F60004D935D936D937C931B971C96EF012C965C
:103F70009C01275E3F4F49914D93A217B307D9F794
:103F8000218D328DFC01328F218FDF91CF910895E9
:103F9000CF92DF92EF92FF920F931F93CF93DF9315
:103FA000CDB7DEB7A0970FB6F894DEBF0FBECDBF7A
:103FB0007C018B0150E040E06C018AE0C80ED11C0E
:103FC000CA010196F8012491E1E0F0E0EC0FFD1F39
:103FD000E40FF51F2083222389F08032910551F4EC
:103FE00040E250E0BE016F5F7F4FC6010E94FE15A8
:103FF00090E080E00F5F1F4FAC01E2CF029738F0F6
:10400000BE016F5F7F4FC7010A960E94FE15A09602
:104010000FB6F894DEBF0FBECDBFDF91CF911F91D9
:104020000F91FF90EF90DF90CF900895EF92FF9265
:104030000F931F93CF93DF93EC018B017A0167EF0E
:1040400073E00E94C81FB801CE010E947F7C8E01E0
:10405000065F1F4F42E050E061ED79E0C8010E9429
:10406000FE15E114F10421F0B701CE010E947F7C1E
:1040700042E050E061ED79E0C801DF91CF911F91FE
:104080000F91FF90EF900C94FE1569E973E00C948A
:10409000C81FCF92DF92EF92FF920F931F93CF939F
:1040A000DF9300D000D0CDB7DEB77C01FB01848167
:1040B00095818A01081B190B101611069CF0C70187
:1040C0000E94237BC70126960FB6F894DEBF0FBE71
:1040D000CDBFDF91CF911F910F91FF90EF90DF90B7
:1040E000CF900895CE0101960E94357BCC24C394D5
:1040F000D12C61E876E0CE0101960E941F7AFFEF95
:10410000CF1ADF0A0C151D05A4F7BE016F5F7F4FA4
:10411000C7010E94237BCE0101960E94A57AD2CFCF
:10412000DF92EF92FF920F931F93CF93DF93CDB760
:10413000DEB762970FB6F894DEBF0FBECDBF2091F9
:10414000DE02222379F12091DD02222359F17A0146
:104150008C016F3F7F4FA1F560E080E00E949D8958
:10416000D12CB80183E894E10E94877C63E475E078
:1041700083E894E10E94A97CF801848160E08D0DC0
:104180000E949D890E94DB816093AF0E7093B00EF8
:104190008093B10E9093B20EB701FF0C880B990B70
:1041A0000E940C7F62960FB6F894DEBF0FBECDBFA3
:1041B000DF91CF911F910F91FF90EF90DF900895C5
:1041C00060E080E00E949D890E94DB8128EE33E060
:1041D00040E050E00E94D6A9CA01B90120E831E5CB
:1041E00041E050E00E94F8A9AB01BC0120E0CE0103
:1041F00001960E94DD7ABE016F5F7F4FCE01079668
:104200000E94357B60EF78E0CE0107960E94AA7984
:10421000BC01CE010D960E94357BCE0107960E940F
:10422000A57ACE0101960E94A57ABE01635F7F4FF9
:1042300083E894E10E94877CD98860E08D2D0E94FC
:104240009D89CE010D960E94A57A8BCFEF92FF92A9
:104250000F931F93CF93DF9300D000D0CDB7DEB77D
:104260008C017B0167E074E00E943E7B8AE0E816E7
:10427000F1042CF467E377E0C8010E941F7AB701CC
:10428000CE0101960E948378BE016F5F7F4FC80107
:104290000E94297ACE0101960E94A57AC80126962D
:1042A0000FB6F894DEBF0FBECDBFDF91CF911F9147
:1042B0000F91FF90EF9008952F923F924F925F924F
:1042C0006F927F928F929F92AF92BF92CF92DF9226
:1042D000EF92FF920F931F93CF93DF93CDB7DEB78B
:1042E000C258D1090FB6F894DEBF0FBECDBF6C0126
:1042F0005B0188EE482E83E0582E612C712C0EED68
:1043000013E09BE5892E912C8C0E9D1E8CE0880E6F
:10431000911C1B019FEF291A390AD6015996ED907D
:10432000FC90F7018581823008F493C082859385E3
:10433000A485B5858F719927AA27BB27892B8A2B3E
:104340008B2B09F086C040E250E0BE016F5F7F4FCB
:10435000C7010E94B791803209F07BC08981882310
:1043600009F477C0853E79F38E3269F38C8583FD3D
:10437000EACF22961FAE1EAE22978CE593E09FAF48
:104380008EAF24961FAE2497BE016F5F7F4FE0E093
:1043900080E04EE2DB019D91BD019032A1F08830BA
:1043A00049F426E730E02C0F3D1F2E0F311DD901B7
:1043B0004C93EF5F26E730E02C0F3D1F2E0F311D91
:1043C000D9019C93EF5F8F5F8B3021F786E790E0F8
:1043D0008C0F9D1F8E0F911DFC011082D6015996E6
:1043E0006D917C9121E0AE014A585F4FCE01CE968F
:1043F0000E94510E882369F1BE01625C7F4FCE019D
:1044000081960E94C911AE014A585F4FBE016F5D8F
:104410007F4FCE01855A9F4F0E943712CE01855A99
:104420009F4F0E941912882309F4ACC0F12CFA1492
:104430001B042CF569E0CE0101960E940A7BCE0197
:1044400001960E94801FCE0101960E94A57AF394E6
:10445000EECF6F961FAE1EAE6F97A3964CAE5DAEBD
:104460006EAE7FAEA3976D961FAF0EAF6D97E696BB
:104470001FAE1EAEE697A8961FAEA897CFCFB40189
:10448000CE0101960E943E7BCE0101960E94801FC4
:10449000CE0101960E94A57AE696EEADFFADE697B5
:1044A000309709F447C08581823008F443C06EE13B
:1044B00074E0CE0101960E943E7BCE0101960E94DF
:1044C000691FCE0101960E94A57A6F968EAD9FADB1
:1044D0006F979C838B83A3968CAD9DADAEADBFAD26
:1044E000A3978D839E83AF83B887A7968CAD9DAD30
:1044F000AEADBFADA79789879A87AB87BC871A8374
:1045000009838DE0F401DE011D9601900D928A95DC
:10451000E1F7E6968EAD9FADE6979B8F8A8FB1014E
:10452000CE0101960E945C21CE01855A9F4F0E94C8
:104530002512F3CE65E074E0CE0101960E943E7B29
:10454000CE0101960E94801FCE0101960E94A57A9D
:10455000E696EEADFFADE69740E050E0BA01309749
:1045600021F04389548965897689CE0101960E949C
:10457000AF78CE0101960E94691FCE0101960E947C
:10458000A57AD2CFCE57DF4F0FB6F894DEBF0FBE5D
:10459000CDBFDF91CF911F910F91FF90EF90DF90F2
:1045A000CF90BF90AF909F908F907F906F905F90D3
:1045B0004F903F902F9008951F93CF93DF93CDB7E7
:1045C000DEB72C970FB6F894DEBF0FBECDBF2B8998
:1045D0003C893093A9022093A802FE017396ACEEA9
:1045E000BBE090E080E032962817390734F0408134
:1045F00051814D935D930196F6CF8B8D9C8D909359
:10460000E80B8093E70B8D8D9E8D9093EA0B809342
:10461000E90BAC968FADAC97BE0165597F4F8F32D9
:1046200009F0B3C1CE0107960E943E7B68E074E0BA
:10463000CE0101960E943E7BBE01695F7F4FCE0195
:1046400001960E94C079BC018BE294E10E94557AE8
:10465000CE0101960E94A57ACE0107960E94A57A06
:104660006BE274E1CE0101960E94357BCE0101968A
:104670000E94691FCE0101960E94A57A6EE174E046
:10468000CE0101960E943E7BBE016F5F7F4F8BE2A1
:1046900094E10E946F79182FCE0101960E94A57AAD
:1046A00040912F1450913014112309F475C1BA01AF
:1046B000625071098BE294E10E945E79682FCE010D
:1046C00001960E940A7BBE016F5F7F4F8DE094E1EF
:1046D0000E946C7ACE0101960E94A57A65E073E192
:1046E000CE0107960E943E7B60E274E0CE01019607
:1046F0000E943E7BBE01695F7F4FCE0101960E9402
:10470000C079BC0185E294E10E94557ACE01019600
:104710000E94A57ACE0107960E94A57A23968FADB6
:1047200023971F928F9322968FAD22971F928F937C
:1047300021968FAD21971F928F938FAD1F928F93EC
:1047400086E294E09F938F938EEF9BE09F938F93ED
:104750000E942FAECF52DF4F88819981C15DD0403A
:104760009093860280938502BE016D527F4FCE01E9
:1047700001960E943E7BBE016F5F7F4F8FE194E107
:104780000E946C7ACE0101960E94A57ABE01625207
:104790007F4FCE0101960E943E7BBE016F5F7F4F2F
:1047A00089E194E10E946C7ACE0101960E94A57A7B
:1047B00040911D1450911E144250510969E174E159
:1047C000CE0101960E94220ACE0101960E94F6783F
:1047D0006C596093B502CE0101960E94A57ACD5E18
:1047E000DE4F688179818A819B81C351D1400E94CB
:1047F00093A80FB6F894DEBF0FBECDBF9B01AC01EE
:104800000E9453AB882389F08CE390E0A0E0B0E0F5
:10481000CD5EDE4F88839983AA83BB83C351D14089
:10482000CE5EDE4F1882C251D140CE5EDE4F88810F
:10483000C251D140882399F0CD5EDE4F88819981A5
:10484000AA81BB81C351D1408093AA029093AB024D
:10485000A093AC02B093AD0281E08093AC0CC95E32
:10486000DE4F688179818A819B81C751D1409B014C
:10487000AC010E9453AB882361F080E090E0A0E798
:10488000B2E4C95EDE4F88839983AA83BB83C75194
:10489000D140C55EDE4F68817981CB51D140072E72
:1048A000000C880B990B0E9493A89B01AC010E94FD
:1048B00053AB882341F082E090E0C55EDE4F9983E0
:1048C0008883CB51D140C55CDE4F68817981CB5361
:1048D000D140072E000C880B990B0E9493A89B01D6
:1048E000AC010E9453AB882341F080E590E0C55CA9
:1048F000DE4F99838883CB53D140C55CDE4F8881DE
:104900009981CB53D140909336028093350288E24F
:10491000FE01E651FF4FAFEBBBE001900D928A958F
:10492000E1F7CF5CDE4F88819981AA81BB81C153B9
:10493000D1408093200290932102A0932202B09351
:104940002302CB5CDE4F88819981AA81BB81C5534C
:10495000D14080931C0290931D02A0931E02B0933D
:104960001F02C75CDE4F88819981C953D140909363
:104970006802809367022C960FB6F894DEBF0FBED4
:10498000CDBFDF91CF911F910895CE0107960E9470
:104990003E7B6DE074E04CCE415051096BE274E116
:1049A000CE0101960E94220ABE016F5F7F4F8DE00B
:1049B00094E10E946C7ACE0101960E94A57A6BE286
:1049C00074E1CE0101960E94357B6EE174E0CE0168
:1049D00001960E94AA79BC018BE294E10E94557A6B
:1049E00079CE0F931F93CF93DF9300D000D0CDB734
:1049F000DEB72091EB0B2223A9F08C0160E178E077
:104A0000CE0101960E943E7BB801CE0101960E9424
:104A1000C079BC0181E89FE00E94957CCE0101969F
:104A20000E94A57A26960FB6F894DEBF0FBECDBFC2
:104A3000DF91CF911F910F910895DF92EF92FF9236
:104A40000F931F93CF93DF93CDB7DEB762970FB667
:104A5000F894DEBF0FBECDBF8C011092F50A67E05F
:104A600074E0CE010D960E943E7BFF24F39481E812
:104A70009FE00E9406732091F50A181619067CF52E
:104A800021112DC081E89FE00E94E4728A3009F074
:104A90007EC089899A89892B09F481C0F092F50A30
:104AA00062E374E0CE0101960E943E7BBE01635F2B
:104AB0007F4FCE0101960E94C079BC01CE010796BE
:104AC0000E94357BCE0107960E94F124CE01079605
:104AD0000E94A57ACE0101960E94A57A60C0F12CB1
:104AE000E12CDD24D394222309F460C089899A89BA
:104AF000019709F045C061EB74E0CE0107960E9472
:104B00003E7BBE01695F7F4FCE010D960E948F797B
:104B1000F12C811115C062E474E0CE0101960E946F
:104B20003E7BBE016F5F7F4FCE010D960E948F7955
:104B3000FF24F3948111F12CCE0101960E94A57AF5
:104B4000CE0107960E94A57AFF20A1F050E040E038
:104B5000BE01635F7F4FCE0101960E94220ABE0113
:104B60006F5F7F4F8EEB91E10E946C7ACE010196D0
:104B70000E94A57A64E170E080E090E00E940C7FE2
:104B8000BE01635F7F4FC8010E94237B96C08D30BA
:104B900009F47FCF682FCE010D960E94FD796AE05F
:104BA00070E080E090E00E940C7F61CF84EE9EE098
:104BB0000E9406731816190614F584EE9EE00E94F2
:104BC000E4728A30A9F08D3099F09091F50A911134
:104BD0000FC0682FCE010D960E94FD798FEFE81A65
:104BE000F80A65E070E080E090E00E940C7FDECF84
:104BF00089899A89892BA9F3D092F50AF2CF64E1C9
:104C000070E080E090E00E940C7FEF2809F43FC044
:104C100089899A89892BD9F18091EB0B882389F1B5
:104C200060E178E0CE0101960E943E7BBE016F5F9D
:104C30007F4FCE010D960E948F79F82ECE010196FE
:104C40000E94A57AF1101DC06BE374E0CE010196BD
:104C50000E943E7BCE0101960E94801FCE010196EC
:104C60000E94A57ABE01635F7F4FCE0101960E942C
:104C7000357BCE0101960E94691FCE0101960E94EC
:104C8000A57A64E170E080E090E00E940C7F898961
:104C90009A892091F50A21112BCF009709F028CF8E
:104CA00064E670E080E090E00E940C7F0E94DB816F
:104CB00067E074E0C8010E943E7BCE010D960E9421
:104CC000A57AC80162960FB6F894DEBF0FBECDBFBD
:104CD000DF91CF911F910F91FF90EF90DF9008959A
:104CE0000F931F93CF93DF93CDB7DEB72C970FB6FB
:104CF000F894DEBF0FBECDBF8C010E949A87BC0125
:104D0000C8010E9426210E949287BC01CE0107960D
:104D10000E94262165E677E0CE0101960E943E7B47
:104D2000BE01695F7F4FCE0101960E94C079BC0130
:104D3000C8010E94297ACE0101960E94A57ACE016F
:104D400007960E94A57A61E876E0C8010E941F7A62
:104D50000E948A87BC01CE0101960E942621BE01D5
:104D60006F5F7F4FC8010E94297ACE0101960E9491
:104D7000A57A64E474E0C8010E941F7A0E948287C9
:104D8000BC01CE0101960E942621BE016F5F7F4FBC
:104D9000C8010E94297ACE0101960E94A57A64E496
:104DA00074E0C8010E941F7A0E947887BC01CE017E
:104DB00001960E942621BE016F5F7F4FC8010E94AD
:104DC000297ACE0101960E94A57AC8012C960FB6C9
:104DD000F894DEBF0FBECDBFDF91CF911F910F9131
:104DE0000895CF93DF9300D000D0CDB7DEB70E94F7
:104DF0002E0ACE0101960E9470264AE050E06FEF25
:104E00007FEFCE0101960E949020CE0101960E9474
:104E1000A57A61E080E00E949D89CE0101960E9402
:104E2000261E63E874E1CE0101960E940B7C66E4C5
:104E300074E083E894E10E947F7C0E94DB816093B0
:104E4000490C70934A0C80934B0C90934C0C269613
:104E50000FB6F894DEBF0FBECDBFDF91CF9108959E
:104E60000F931F93CF93DF9300D000D0CDB7DEB761
:104E70008C01CE0101960E9470264AE050E06FEF4F
:104E80007FEFCE0101960E949020CE0101960E94F4
:104E9000A57AB801CE0101960E94357B6AE070E0E8
:104EA000CE0101960E94CA89CE0101960E94A57A80
:104EB00026960FB6F894DEBF0FBECDBFDF91CF911F
:104EC0001F910F9108950F931F93CF93DF93CDB749
:104ED000DEB72C970FB6F894DEBF0FBECDBF8C01A6
:104EE0000E949A87BC01C8010E9426210E949287D5
:104EF000BC01CE0107960E94262165E677E0CE012F
:104F000001960E943E7BBE01695F7F4FCE010196F4
:104F10000E94C079BC01C8010E94297ACE01019685
:104F20000E94A57ACE0107960E94A57A0E94398632
:104F30000E947F866091310C70E0CE0107960E943E
:104F4000262165E677E0CE0101960E943E7BBE01F8
:104F5000695F7F4FCE0101960E94C079BC01C801F4
:104F60000E94297ACE0101960E94A57ACE01079669
:104F70000E94A57A61E876E0C8010E941F7A0E942B
:104F80008A87BC01CE0101960E942621BE016F5F77
:104F90007F4FC8010E94297ACE0101960E94A57A0E
:104FA00064E474E0C8010E941F7A0E948287BC01F9
:104FB000CE0101960E942621BE016F5F7F4FC8017E
:104FC0000E94297ACE0101960E94A57A64E474E0D9
:104FD000C8010E941F7A0E947887BC01CE01019609
:104FE0000E942621BE016F5F7F4FC8010E94297A6F
:104FF000CE0101960E94A57AC8012C960FB6F894AE
:10500000DEBF0FBECDBFDF91CF911F910F910895ED
:105010006115710519F00A960C94997B90E080E077
:105020000895EF92FF920F931F93CF93DF9300D0D9
:105030001F92CDB7DEB78C017B01FB0184858830E0
:10504000A8F08CEF93E0F8019183808312821382A1
:1050500014821582C8010F900F900F900F90DF916E
:10506000CF911F910F91FF90EF90089580E591E00F
:105070000E94A77524E030E0AE014F5F5F4F6CE007
:1050800070E0F70184850E947614BE016F5F7F4F48
:10509000C8010E94CD7CDECF3F924F925F926F920B
:1050A0007F928F929F92AF92BF92CF92DF92EF92B8
:1050B000FF920F931F93CF93DF93CDB7DEB7EA979D
:1050C0000FB6F894DEBF0FBECDBF7C012A013B01B5
:1050D00069010E94DB814B015C0187010D5B1F4F61
:1050E000C8010E94AA17181619069CF00E94DB81BD
:1050F000681979098A099B094616570668067906D0
:1051000008F466C162E370E080E090E00E940C7FEA
:10511000E7CF42E250E0BE016F5F7F4FC8010E94BF
:10512000611789818230D1F0312C832DEA960FB638
:10513000F894DEBF0FBECDBFDF91CF911F910F91CD
:10514000FF90EF90DF90CF90BF90AF909F908F90A7
:105150007F906F905F904F903F900895F801848901
:1051600095898334910501F76D817E818F819885C2
:105170000E9480AB4B015C01F60180829182A28289
:10518000B38246E050E0B701685F7F4FCE014D9695
:105190000E94AEAD892B41F6F70180819181A281F9
:1051A000B38188169906AA06BB0608F4BDCF848190
:1051B0009581A681B78188159905AA05BB0508F4D4
:1051C000B3CF89899A89AB89BC8986879787A08B59
:1051D000B18B4EEC50E070E060E0C8010E946117B6
:1051E000312CC701829698AB8FA7F701B696FAAB20
:1051F000E9AB08969CAB8BAB67019AE1C90ED11C59
:10520000BD96FEABEDABC701429698AF8FABFD9755
:10521000FAAFE9AF4701FEE18F0E911CF801818DD5
:10522000928D181619060CF080CFC8010E948017C5
:105230008333910509F4B2C014F58130910509F466
:1052400064C044F4892B51F3C8010E948017AC015B
:10525000552775C08330910509F462C00697A1F700
:10526000C8010E948017B82E44E050E0B401C80184
:105270000E946117EB2DE450FF0BAF0160C08A3331
:10528000910509F45FC084F585339105B1F1C697A6
:10529000D9F6C8010E9480175C01B601CE0189963B
:1052A0000E94CD7C8BA59CA5ADA5BEA5892B8A2B84
:1052B0008B2BB1F0EDA9FEA94080518062807380F4
:1052C000B601CE0183960E94CD7C8DA19EA1AFA197
:1052D000B8A5A501481659066A067B0609F0B8CF9D
:1052E00044E050E0B60118C08B33910509F440C08A
:1052F0008F3F910509F492CFA7CFC8010E94801774
:10530000C8010E948017382E89CFC8010E948017DB
:1053100044E050E06FA978ADC8010E9461177ECFCC
:10532000C8010E948017B82E44E050E069AD7AAD04
:10533000C8010E9461178B2D8450990BAC0170E05D
:1053400060E0EACFC8010E94801744E050E069A9FC
:105350007AA9C8010E946117F70166A177A180A50B
:1053600091A50E9480AB66A377A380A791A756CF93
:10537000C8010E94801744E050E06BA97CA9C801D5
:105380000E946117F70162A573A584A595A50E94E7
:1053900080AB62A773A784A795A740CFC8010E94DE
:1053A000801744E050E06FA578A9C8010E946117FA
:1053B000F70162A173A184A195A10E9480AB62A3B1
:1053C00073A384A395A366A777A780AB91AB26CFE1
:1053D00033243A94AACE2F923F924F925F926F92CB
:1053E0007F928F929F92AF92BF92CF92DF92EF9275
:1053F000FF920F931F93CF93DF9300D000D0CDB7D0
:10540000DEB78C010E9477A22FEC37E040E050E03D
:105410000E94F8A9DC01CB010196A11DB11DF80184
:1054200084839583A683B78380839183A283B38388
:105430005801F3E4AF0EB11CC5010E94821864E468
:1054400070E0C5010E94561B882309F445C10E94E3
:10545000DB812B013C01480182E4880E911C48EE5F
:10546000C42E43E0D42EE12CF12C52E0252E1E82D6
:105470001D82D4018C918330B1F1811166C0F80195
:1054800084819581A681B7810196A11DB11D848378
:105490009583A683B7830E94DB8164197509860909
:1054A0009709A70196010E94D6A9A90161E0C80148
:1054B0000E94161C81E0D4018C938D819E810197FE
:1054C000C1F20E94DB816419750986099709D80128
:1054D000D6962D913D914D915C91D997261737071E
:1054E0004807590720F6C5010E948218F8018481F7
:1054F0009581A681B7810196A11DB11D84839583F5
:10550000A683B7830E94DB81F801FE9660837183D6
:10551000828393838D819E8126960FB6F894DEBF99
:105520000FBECDBFDF91CF911F910F91FF90EF90F4
:10553000DF90CF90BF90AF909F908F907F906F90B3
:105540005F904F903F902F9008958430F1F4F801D0
:1055500084819581A681B7810196A11DB11D8483A7
:105560009583A683B7830E94DB8164197509860938
:105570009709A70196010E94D6A9A90163E0C80175
:105580000E94161CD4012C9298CF813051F5F8015D
:1055900042AD53AD64AD75AD9E012F5F3F4FC80165
:1055A0000E944C28382EF2E08F1390C089819A8196
:1055B000AB81BC81F80184839583A683B7830E9465
:1055C000DB816419750986099709A70196010E9474
:1055D000D6A9A90163E0C8010E94161CD4013C921F
:1055E0006CCF823009F069CFF80142AD53AD64ADA4
:1055F00075AD9E012F5F3F4FC8010E944C28382E89
:10560000F5E08F135DC0E3E0D401EC93F80182A1D3
:1056100093A1A4A1B5A1892B8A2B8B2B41F484E8FB
:1056200093E0A0E0B0E082A393A3A4A3B5A3F80104
:1056300086A197A1A0A5B1A5892B8A2B8B2B61F4FC
:1056400082A193A1A4A1B5A1B695A7959795879599
:1056500086A397A3A0A7B1A7F80182A593A5A4A5A7
:10566000B5A5892B8A2B8B2BA9F482A193A1A4A188
:10567000B5A1AC01BD0123E0769567955795479597
:105680002A95D1F7841B950BA60BB70B82A793A77E
:10569000A4A7B5A7F80186A197A1A0A5B1A586A743
:1056A00097A7A0ABB1AB82A593A5A4A5B5A582ABE6
:1056B00093ABA4ABB5AB81E090E09E838D83FDCE30
:1056C00096E0891303C0D4011C92F7CEBFEF3B12C2
:1056D000F4CEF4011082F1CE1E821D821BCF7F9288
:1056E0008F929F92AF92BF92CF92DF92EF92FF92F2
:1056F0000F931F93CF93DF93CDB7DEB762970FB6AB
:10570000F894DEBF0FBECDBF10E000E036EFC32E31
:105710003AE0D32E40E3E42E53EEB52E66E0A62EFB
:105720007CEE972EE1E3FE2EFEE48F2EA4E37A2E8C
:1057300068EB72E280ED91E10E94561BF6018E2D1E
:1057400011928A95E9F7B092F60AA092F80A90921F
:10575000F90AF092020B8092030BF092040B709204
:10576000050B60E072E0CE0101960E94CD7C4BE714
:1057700050E0BE016F5F7F4F80ED91E10E94DF1B23
:1057800040E350E066EF7AE080ED91E10E94741B07
:1057900080ED91E10E94AE1B68EE73E080E090E046
:1057A0000E940C7F80ED91E10E94AA17892B31F5B0
:1057B0000A30110509F05FC16AE474E0CE01019678
:1057C0000E943E7BCE0101960E94691FCE01019688
:1057D0000E94A57A62960FB6F894DEBF0FBECDBFC9
:1057E000DF91CF911F910F91FF90EF90DF90CF90BD
:1057F000BF90AF909F908F907F90089540E350E0CE
:1058000066EF7AE080ED91E10E94611760911E0BD6
:1058100070911F0B76276727762790E080E0CB01F9
:1058200077276627C090200BD090210BDC24CD2455
:10583000DC24F12CE12C6C297D298E299F297E50B6
:105840008A4A93480E9414860E9439866093260BE8
:105850007093270B8093280B9093290B0A30110526
:1058600009F4AACF0E94398660934D0C70934E0CB8
:1058700080934F0C9093500C0E9439866093510C8A
:105880007093520C8093530C9093540CCE0101965C
:105890000E946327CE0101960E94691FCE010196E6
:1058A0000E94A57A0E948A87BC01CE0107960E94B9
:1058B000262164E474E0CE0107960E941F7A0E94BC
:1058C0008287BC01CE0101960E942621BE016F5F36
:1058D0007F4FCE0107960E94297ACE0101960E9441
:1058E000A57A64E474E0CE0107960E941F7A0E94B4
:1058F0007887BC01CE0101960E942621BE016F5F10
:105900007F4FCE0107960E94297ACE0101960E9410
:10591000A57A64E574E0CE0101960E943E7BBE014B
:10592000695F7F4FCE0101960E94C079BC01CE0114
:105930000D960E94357B4AE050E06FEF7FEFCE017D
:105940000D960E949020CE010D960E94A57ACE0160
:1059500001960E94A57ACE0107960E94A57A68EE6C
:1059600073E080E090E00E940C7F0E949A87BC0167
:10597000CE010D960E9426210E949287BC01CE0185
:1059800001960E94262165E677E0CE0107960E94E7
:105990003E7BBE016F5F7F4FCE0107960E94C079AC
:1059A000BC01CE010D960E94297ACE0107960E9475
:1059B000A57ACE0101960E94A57A0E9439860E949E
:1059C0007F866091310C70E0CE0101960E94262105
:1059D00065E677E0CE0107960E943E7BBE016F5FD1
:1059E0007F4FCE0107960E94C079BC01CE010D9673
:1059F0000E94297ACE0107960E94A57ACE010196CF
:105A00000E94A57A6AE574E0CE0101960E943E7B71
:105A1000BE01635F7F4FCE0101960E94C079BC0139
:105A2000CE0107960E94357B4AE050E06FEF7FEF92
:105A3000CE0107960E949020CE0107960E94A57A7B
:105A4000CE0101960E94A57ACE010D960E94A57AFC
:105A500068EE73E080E090E00E940C7FCE0101963A
:105A60000E9470264AE050E06FEF7FEFCE01019672
:105A70000E949020ABCE0F5F1F4F68EE73E080E076
:105A800090E00E940C7F4091260B5091270B609173
:105A9000280B7091290BCE0101960E94AF78CE01A0
:105AA00001960E94691FCE0101960E94A57A40CE00
:105AB000EF92FF920F931F93CF93DF93CDB7DEB793
:105AC000E8970FB6F894DEBF0FBECDBF67E074E075
:105AD000CE0187960E943E7B67E074E0CE018D96F2
:105AE0000E943E7B82E0E82EF12C2496FFAEEEAEC3
:105AF000249786E0E9EEF2E0DE01D39601900D9264
:105B00008A95E1F786E0FE01F396DE01AC5BBF4FBC
:105B100001900D928A95E1F72C961FAE1EAE2C9740
:105B200001E010E02E961FAF0EAF2E9788E0EFEE4B
:105B3000F2E0DE01599601900D928A95E1F788E036
:105B4000FE017996DE01A25BBF4F01900D928A950E
:105B5000E1F788E1E7EFF2E0DE01119601900D92A6
:105B60008A95E1F788E1FE013196DE01AA5ABF4F1E
:105B700001900D928A95E1F780910F0390911003A7
:105B8000A0911103B0911203E2968CAF9DAFAEAF1E
:105B9000BFAFE29760E674E0CE0187960E94797805
:105BA00060E0CE0187960E94FD794BA55CA5BE0101
:105BB0006E587F4FCE0187960E94AA7662EF76E0FC
:105BC000CE018D960E94307A68EA74E08DE094E10F
:105BD0000E94797860E0CE018D960E94FD7949A9F6
:105BE0005AA9BE0166567F4FCE018D960E94AA76B5
:105BF00067E074E0CE0187960E94797867E074E0F0
:105C0000CE018D960E947978C250DF4F198218829A
:105C1000CE5FD0408091850290918602C050DF4FC8
:105C200099838883C050D14080E090E0A0E7B2E43F
:105C3000CA5BDE4F88839983AA83BB83C654D14055
:105C4000C65BDE4FF982E882CA54D14080E090E022
:105C5000A0E2B2E4C45BDE4F88839983AA83BB834E
:105C6000CC54D14080E090E0A4E3B2E4C05BDE4FCE
:105C700088839983AA83BB83C055D14084EB90E08D
:105C8000CC5ADE4F99838883C455D14088E790E091
:105C9000CA5ADE4F99838883C655D1408CE291E081
:105CA000A0E0B0E0C85ADE4F88839983AA83BB8303
:105CB000C855D140C45ADE4F19830883CC55D14012
:105CC000C25ADE4FF982E882CE55D14060E08FE1C2
:105CD00094E10E94FD7960E089E194E10E94FD7900
:105CE0004091231450912414BE016E5F7E4F8FE1CA
:105CF00094E10E94AA7640911D1450911E14BE0199
:105D0000635F7E4F89E194E10E94AA7688E2EFEB1F
:105D1000FBE0DE01A75EBE4F01900D928A95E1F790
:105D20008CE390E0A0E0B0E0CE5BDE4F8883998307
:105D3000AA83BB83C254D140CF5BDE4F1882C154CB
:105D4000D14084EE98E3AEE8B2E4C05ADE4F8883D7
:105D50009983AA83BB83C056D14084EE98E3AEE812
:105D6000B1E4CC59DE4F88839983AA83BB83C456A0
:105D7000D140C859DE4F19830883C856D14080E509
:105D800090E0C659DE4F99838883CA56D14084EF8C
:105D900091E090939D0280939C02BE016E5B7F4FC9
:105DA0000E944F0964EF71E080E090E00E940C7F58
:105DB0006BED76E0CE0181960E942C7BCE01819620
:105DC0000E94691FCE0181960E94A57ACE018D9610
:105DD0000E94A57ACE0187960E94A57AE8960FB612
:105DE000F894DEBF0FBECDBFDF91CF911F910F9111
:105DF000FF90EF9008959F92AF92BF92CF92DF9263
:105E0000EF92FF920F931F93CF93DF93CDB7DEB73F
:105E1000C859D1090FB6F894DEBF0FBECDBF5C01E3
:105E20007B016A016DE273E1CE0189579F4F0E94A9
:105E30003E7B6EE174E08E010F5F1F4FC8010E9430
:105E40003E7BB801CE0189579F4F0E948F79982ED3
:105E5000C8010E94A57A911014C06EE174E0C801D7
:105E60000E943E7BBE0169577F4FC8010E94C079E6
:105E7000BC01CE0189579F4F0E94557AC8010E94EC
:105E8000A57AB501CE0183579F4F0E943E7B68E6FD
:105E900074E021E0E216F10441F063E774E032E0DF
:105EA000E316F10411F06BE774E0CE0189579F4FC0
:105EB0000E941F7A60E0CE0189579F4F0E94FD79B2
:105EC000B601C8010E94357B6AE0C8010E94117AC0
:105ED000BC01CE018D569F4F0E94357BC8010E94A8
:105EE000A57AC557DF4F48815981CB58D040B801BA
:105EF000CE0189579F4F0E94AA768091AD0C8823CE
:105F000099F163E874E0CE018F579F4F0E943E7B6A
:105F1000CE018F579F4F0E94801FCE018F579F4FFA
:105F20000E94A57ABE0169577F4FCE018F579F4FC0
:105F30000E94357BCE018F579F4F0E94801FCE015C
:105F40008F579F4F0E94A57AB801CE018F579F4F60
:105F50000E943E7BCE018F579F4F0E94801FCE0133
:105F60008F579F4F0E94A57ACC56DF4F8881C45926
:105F7000D0408F93CD56DF4F8881C359D0408F9347
:105F8000C257DF4F8881CE58D0408F93C357DF4F21
:105F90008881CD58D0408F9383E994E09F938F936D
:105FA00088E2E82E8AE0F82EFF92EF920E942FAE50
:105FB00040913502509136026EEF7BE084EB92E126
:105FC0000E94131A0FB6F894DEBF0FBECDBF019723
:105FD00009F07CC01F930F9389E994E09F938F93FE
:105FE0000AE21BE01F930F930E942FAEB80184EBCF
:105FF00092E10E946B7C8EEF9BE09F938F938AEAE5
:1060000094E09F938F931F930F930E942FAEB8013C
:1060100084EB92E10E946B7C6DE474E084EB92E18E
:106020000E94A97C61ED79E084EB92E10E94997B6A
:10603000F70101900020E9F7CF0189529A409F9320
:106040008F9383EB94E09F938F931F930F930E9402
:106050002FAEB80184EB92E10E946B7CB70184EB18
:1060600092E10E947F7C62E370E080E090E00E9419
:106070000C7F84EB92E10E94C5190FB6F894DEBF45
:106080000FBECDBF11E0CE018D569F4F0E94A57A65
:10609000CE0183579F4F0E94A57ACE0189579F4F0B
:1060A0000E94A57A812FC856DF4F0FB6F894DEBF45
:1060B0000FBECDBFDF91CF911F910F91FF90EF9059
:1060C000DF90CF90BF90AF909F90089560E974E00B
:1060D000CE018F579F4F0E942C7BCE018F579F4F31
:1060E0000E94691FCE018F579F4F0E94A57A6CE9CD
:1060F00074E0CE018F579F4F0E942C7BCE018F57AB
:106100009F4F0E94801FCE018F579F4F0E94A57AFC
:1061100068E27AE0CE018F579F4F0E943E7BCE010E
:106120008F579F4F0E94691FCE018F579F4F0E942C
:10613000A57A10E0A8CF8F929F92AF92BF92EF9274
:10614000FF920F931F93CF93DF93CDB7DEB76E9778
:106150000FB6F894DEBF0FBECDBF0091A80C109112
:10616000A90C0115110509F4D8C00E94DB814B016F
:106170005C0178012EE3E20EF11CF7018081918130
:10618000A281B381A5019401281B390B4A0B5B0B3B
:10619000CA01B901683E33E0730781059105A0F19A
:1061A00028EE33E040E050E00E94D6A9861A970A14
:1061B000A80AB90AD7018D929D92AD92BC9213970D
:1061C000F80186A597A5A0A9B1A949015A01880C93
:1061D000991CAA1CBB1C88159905AA05BB0508F0CB
:1061E000C2C016A617A610AA11AAF80182A993A9DF
:1061F000A4A9B5A988159905AA05BB0508F0BCC0D6
:1062000012AA13AA14AA15AAF80186A597A5A0A9EF
:10621000B1A9892B8A2B8B2B09F0B7C0EE5BFF4FFE
:106220008081833009F0B1C084E08083C8010E947E
:10623000EB290196D801D2964D915D916D917C919B
:10624000D597452B462B472BA1F4F801EE5BFF4F6A
:106250002081233011F021110CC01082F8013E96EC
:1062600084E1DF011D928A95E9F7C8010E94EB29BC
:1062700003968230910519F0049709F04EC080E52D
:1062800091E00E94A7756091A80C7091A90C625FC3
:106290007F4FCE0101960E94CD7CCE0103960E94D5
:1062A0007C156091A80C7091A90C6A5E7F4FCE019D
:1062B00001960E94CD7C44E050E0BE016D5F7F4FAF
:1062C00081E090E00E941E136091A80C7091A90CCF
:1062D0006E5E7F4FCE0101960E94CD7C44E050E07F
:1062E000BE016D5F7F4F85E090E00E941E136091BC
:1062F000A80C7091A90C625E7F4FCE0101960E949E
:10630000CD7C8B819C81AD81BE81809375109093F3
:106310007610A0937710B093781060ED77E080E06E
:1063200090E00E940C7F0E94CA7F7C0168EE73E0BF
:1063300080E090E00E940C7F0BE010E0EF2841F538
:106340000150110929F160ED77E080E090E00E94B2
:106350000C7F0E94CA7F7C0168EE73E080E090E0D1
:106360000E940C7FEBCF821B930BA40BB50B86A76F
:1063700097A7A0ABB1AB39CF821B930BA40BB50B86
:1063800082AB93ABA4ABB5AB3FCF90E080E052CFF4
:1063900083E191E10E94241D0E94F12667E074E0F0
:1063A000CE010D960E943E7B64E775E0CE014396D8
:1063B0000E942C7BCE0149960E94261E8E8D1F9234
:1063C0008F938D8D1F928F938C8D1F928F938B8DBA
:1063D0001F928F9386E294E09F938F938AE29BE0D3
:1063E0009F938F930E942FAE6AE27BE0CE010196CD
:1063F0000E943E7BBE016F5F7F4FCE010D960E94D3
:106400006C7ACE0101960E94A57ABE016D5E7F4F27
:10641000CE0101960E94357BBE01635F7F4FCE01A6
:1064200001960E94C079BC01CE0107960E94357B7F
:10643000CE0107960E94691FCE0107960E94A57A99
:10644000CE0101960E94A57ABE01635F7F4FCE0107
:1064500001960E94357BAE014F5F5F4F63E070E0B5
:1064600087E892E00E94FB2E182FCE0101960E9431
:10647000A57A0FB6F894DEBF0FBECDBF111122C0B2
:1064800068EC74E0CE0101960E943E7BBE016D5E19
:106490007F4FCE0101960E94C0796DEF71E10E949D
:1064A000C079BC01CE0107960E94357BCE010796CC
:1064B0000E94691FCE0107960E94A57ACE0101961F
:1064C0000E94A57ACE0143960E94A57ACE010D9630
:1064D0000E94A57A6E960FB6F894DEBF0FBECDBFB0
:1064E000DF91CF911F910F91FF90EF90BF90AF90F0
:1064F0009F908F900895CF92DF92EF92FF920F932B
:106500001F93CF93DF93CDB7DEB768970FB6F8949C
:10651000DEBF0FBECDBF67E074E0CE0143960E94A0
:106520003E7B60EF77E0CE0101960E942C7BCE018E
:1065300001960E94801FCE0101960E94A57A6CA14F
:106540007DA1CE0101960E948378CE0101960E9422
:10655000691FCE0101960E94A57A63EE77E0CE0115
:1065600001960E942C7BCE0101960E94801FCE01D5
:1065700001960E94A57A7E0188E2E80EF11C01E0F6
:1065800010E08CA19DA1801791070CF1F70161919A
:1065900071917F01CE0101960E948378CE01019610
:1065A0000E94801FCE0101960E94A57A61E876E0E4
:1065B000CE0101960E943E7BCE0101960E94801F73
:1065C000CE0101960E94A57A0F5F1F4FDACF61E8D6
:1065D00076E0CE0101960E943E7BCE0101960E949C
:1065E000691FCE0101960E94A57A64ED77E0CE0185
:1065F00001960E942C7BCE0101960E94801FCE0145
:1066000001960E94A57A6091E70B7091E80BCE018C
:1066100001960E948378CE0101960E94801FCE01D0
:1066200001960E94A57A61E876E0CE0101960E946B
:106630003E7BCE0101960E94801FCE0101960E94F2
:10664000A57A6091E90B7091EA0BCE0101960E9448
:106650008378CE0101960E94691FCE0101960E94A7
:10666000A57A6DEB77E0CE0101960E942C7BCE01DE
:1066700001960E94801FCE0101960E94A57ABE015C
:10668000605D7F4FCE0101960E943E7BCE01019658
:106690000E94801FCE0101960E94A57A61E876E0F3
:1066A000CE0101960E943E7BCE0101960E94801F82
:1066B000CE0101960E94A57ABE016C5C7F4FCE018F
:1066C00001960E943E7BCE0101960E94691FCE0179
:1066D00001960E94A57A6DEA77E0CE0101960E94AC
:1066E0002C7BCE0101960E94691FCE0101960E946B
:1066F000A57A8E010C5D1F4FEE24E394F12C680106
:10670000F8E0CF0ED11C8CA19DA18E159F050CF435
:1067100049C0B701CE0107960E94837860E178E016
:10672000CE0101960E943E7BBE01695F7F4FCE0184
:1067300001960E94C079BC01CE010D960E94357B66
:10674000CE010D960E94801FCE010D960E94A57A63
:10675000CE0101960E94A57ACE0107960E94A57AE5
:1067600065E677E0CE0101960E943E7BCE01019660
:106770000E94801FCE0101960E94A57AB801645E36
:106780007F4FCE0101960E943E7BCE0101960E9472
:10679000691FCE0101960E94A57A8FEFE81AF80AC8
:1067A0008601ADCF63E977E0CE0101960E942C7B94
:1067B000CE0101960E94801FCE0101960E94A57A0B
:1067C0006EEF7BE0CE0101960E943E7BCE010196EA
:1067D0000E94801FCE0101960E94A57A61E977E0B0
:1067E000CE0101960E942C7BCE0101960E94801F53
:1067F000CE0101960E94A57A609135027091360211
:10680000CE0101960E948378CE0101960E94691FF5
:10681000CE0101960E94A57A62E877E0CE0101964A
:106820000E942C7BCE0101960E94801FCE01019612
:106830000E94A57ABE016C5A7F4FCE0101960E943C
:106840003E7BCE0101960E94691FCE0101960E94F7
:10685000A57A61ED74E0CE0101960E943E7BCE01E7
:1068600001960E94801FCE0101960E94A57ABE016A
:1068700064587F4FCE0101960E943E7BCE01019667
:106880000E94691FCE0101960E94A57AC052DF4F77
:1068900088819981C05ED040892B71F46AE777E0E6
:1068A000CE0101960E942C7BCE0101960E94691FA9
:1068B000CE0101960E94A57AC052DF4F888199814E
:1068C000C05ED040019771F460E777E0CE01019699
:1068D0000E942C7BCE0101960E94691FCE01019679
:1068E0000E94A57AC052DF4F88819981C05ED04056
:1068F000029771F467E677E0CE0101960E942C7B47
:10690000CE0101960E94691FCE0101960E94A57AD0
:1069100061E677E0CE0101960E942C7BCE010196C4
:106920000E94801FCE0101960E94A57ACE51DF4FB2
:1069300068817981C25ED040CE0101960E94837841
:10694000CE0101960E94691FCE0101960E94A57A90
:106950004091450C5091460C6091470C7091480C49
:1069600021E0CE0107960E94AD7A6CED74E0CE0175
:1069700001960E943E7BBE01695F7F4FCE0101966A
:106980000E94C07966EE74E00E94AA79BC01CE0133
:106990000D960E94357BCE010D960E94691FCE0197
:1069A0000D960E94A57ACE0101960E94A57ACE018D
:1069B00007960E94A57A4091410C5091420C60913B
:1069C000430C7091440C21E0CE0107960E94AD7AF1
:1069D0006BEE74E0CE0101960E943E7BBE01695FC2
:1069E0007F4FCE0101960E94C07966EE74E00E944E
:1069F000AA79BC01CE010D960E94357BCE010D9681
:106A00000E94691FCE010D960E94A57ACE010196C3
:106A10000E94A57ACE0107960E94A57A64E477E0E9
:106A2000CE0101960E942C7BCE0101960E94801F10
:106A3000CE0101960E94A57A409120025091210238
:106A4000609122027091230225E0CE0101960E94FE
:106A5000AD7ACE0101960E94691FCE0101960E9477
:106A6000A57A6AE277E0CE0101960E942C7BCE01E6
:106A700001960E94801FCE0101960E94A57A409146
:106A80001C0250911D0260911E0270911F0225E0B0
:106A9000CE0101960E94AD7ACE0101960E94691F37
:106AA000CE0101960E94A57A6AE177E0CE010196B7
:106AB0000E942C7BCE0101960E94801FCE01019680
:106AC0000E94A57A6091690270916A02CE010196D6
:106AD0000E948378CE0101960E94691FCE01019623
:106AE0000E94A57A68E077E0CE0101960E942C7B97
:106AF000CE0101960E94801FCE0101960E94A57AC8
:106B0000C65BDE4F68817981CA54D140CE010196BF
:106B10000E948378CE0101960E94691FCE010196E2
:106B20000E94A57ACE0143960E94A57A68960FB678
:106B3000F894DEBF0FBECDBFDF91CF911F910F91B3
:106B4000FF90EF90DF90CF9008952F923F924F9259
:106B50005F926F927F928F929F92AF92BF92CF92ED
:106B6000DF92EF92FF920F931F93CF93DF93CDB7F6
:106B7000DEB7EB970FB6F894DEBF0FBECDBF1C019A
:106B80008B0170E060E00E945E798F8F67E074E0B7
:106B9000CE0149960E943E7B8091690290916A02E3
:106BA0008130910509F092C088E090E090931B023B
:106BB00080931A0289E090E0909319028093180262
:106BC0008091BD0B9091BE0B9093BC0B8093BB0B3F
:106BD0008091140290911502A0911602B0911702B3
:106BE0008093100290931102A0931202B0931302AB
:106BF00080912C0290912D02A0912E02B0912F0233
:106C00008093300290933102A0933202B09333020A
:106C10008091BA0B8093B90B8091B50B9091B60B14
:106C2000A091B70BB091B80B8093B10B9093B20BBE
:106C3000A093B30BB093B40B8AE390E090930F0250
:106C400080930E028091450C9091460CA091470CC8
:106C5000B091480C8093FA0B9093FB0BA093FC0B24
:106C6000B093FD0B80910C0290910D0290930B025A
:106C700080930A028091200290912102A091220229
:106C8000B09123028093240290932502A0932602C0
:106C9000B09327022F8D233509F089C01092BC0BC9
:106CA0001092BB0B8091EB0B882371F062EF74E0C4
:106CB000CE0101960E943E7BCE0101960E94691F83
:106CC000CE0101960E94A57AE12C46C1029711F7E8
:106CD0008AE090E090931B0280931A028BE090E090
:106CE00090931902809318028091AF0B9091B00B92
:106CF0009093BC0B8093BB0B80910602909107028E
:106D0000A0910802B09109028093100290931102A1
:106D1000A0931202B093130280912802909129024D
:106D2000A0912A02B0912B028093300290933102FD
:106D3000A0933202B09333028091AE0B8093B90BD3
:106D40008091AA0B9091AB0BA091AC0BB091AD0BC5
:106D50008093B10B9093B20BA093B30BB093B40B91
:106D60008BE390E090930F0280930E028091410C90
:106D70009091420CA091430CB091440C8093FA0B7B
:106D80009093FB0BA093FC0BB093FD0B809104023E
:106D90009091050290930B0280930A0280911C024D
:106DA00090911D02A0911E02B0911F026BCFC801ED
:106DB0000197029708F0D4C181E090E0A0E0B0E034
:106DC0008093100290931102A0931202B0931302C9
:106DD000D10114968D919C91029748F141E050E0C9
:106DE000B101CE0101960E94220ABE016F5F7F4F62
:106DF000CE0149960E946C7ACE0101960E94A57A36
:106E0000CE0149960130110581F50E94EB7820E012
:106E100030E040E251E40E94F2A80E9418AB609377
:106E20001002709311028093120290931302BF8D8F
:106E300081E090E09093BC0B8093BB0BB13401F5E3
:106E40008091EB0B882309F43FCF67EF74E0CE010C
:106E500001960E943E7BCE0101960E94691FCE01E1
:106E600001960E94A57AE12C44C00E94EB78209103
:106E70002402309125024091260250912702CBCF67
:106E8000EF8DE63409F038C161E080911A020E946A
:106E9000997D02301105C1F4CE0149960E94EB782C
:106EA0009B01AC016091FA0B7091FB0B8091FC0B84
:106EB0009091FD0B0E9439AA6093FA0B7093FB0B23
:106EC0008093FC0B9093FD0B8091EB0B882371F06A
:106ED00060E075E0CE0101960E943E7BCE010196F6
:106EE0000E94801FCE0101960E94A57AEE24E394B1
:106EF000F12C8091EB0B882379F140911002509195
:106F0000110260911202709113022AE0CE010196E3
:106F10000E94DD7ABE016F5F7F4FCE0107960E940F
:106F2000357B64E175E0CE0107960E94AA79BC0129
:106F3000CE010D960E94357BCE010D960E94691FF1
:106F4000CE010D960E94A57ACE0107960E94A57AE1
:106F5000CE0101960E94A57A8091100290911102B3
:106F6000A0911202B0911302181619061A061B06F8
:106F70000CF07BC55F8D563409F482C4523509F498
:106F800083C46E2D80911A020E94997DC12CD12C50
:106F900076019AE0892E912CA12CB12C80911002BF
:106FA00090911102A0911202B0911302C816D90655
:106FB000EA06FB060CF06AC46091BB0B80911802D4
:106FC0000E94997D61E070E080E090E00E940C7F7B
:106FD00060E0809118020E94997D6091300270916A
:106FE000310280913202909133020E940C7F809195
:106FF000300290913102A0913202B0913302459754
:10700000A105B1050CF472C06091100270911102DB
:107010008091120290911302A50194010E94F8A997
:10702000C701B6010E94F8A9672B682B692B09F0EC
:107030005DC0023011050CF459C080916902909135
:107040006A02019731F46CED74E082EB91E10E94E9
:1070500079788091690290916A02029731F46BEE1F
:1070600074E082EB91E10E947978C701B6010E9439
:1070700093A820912402309125024091260250913C
:1070800027020E94A6AAAB01BC0121E0CE0107960F
:107090000E94AD7A62EB71E1CE0101960E94357BD0
:1070A000BE01695F7F4FCE0101960E94C07966EEF6
:1070B00074E00E94AA79BC0182EB91E10E94557AAA
:1070C000CE0101960E94A57ACE0107960E94A57A6C
:1070D00062EB71E1CE0101960E94357BCE010196F3
:1070E0000E943027CE0101960E94A57A8FEFC81A20
:1070F000D80AE80AF80A52CFFF8DF23509F0B3CE6C
:1071000060E080911A020E94997D02301105C1F45D
:10711000CE0149960E94EB789B01AC016091FA0B7D
:107120007091FB0B8091FC0B9091FD0B0E943AAA91
:107130006093FA0B7093FB0B8093FC0B9093FD0B09
:107140008091EB0B882309F4BFCD6AE075E0CE0196
:1071500001960E943E7BCE0101960E94801F7FCE49
:107160000115110521F00330110509F0ADCD81E0C5
:1071700090E090936A02809369029093BC0B809395
:10718000BB0B20916702309168023AAB29AB331FE9
:107190003327331F3BAF632F80911A020E94997DE2
:1071A0008FEF9FEF90930B0280930A02C12CD12C9A
:1071B00076011DA61EA61FA618AA19A61AA61BA60A
:1071C0001CA61BA21CA21DA21EA2412C512C3201E6
:1071D0001FAA18AE19AE1AAE1BAA1CAA1DAA1EAA77
:1071E00061E0809118020E94997D61E070E080E08A
:1071F00090E00E940C7F60E0809118020E94997DCF
:1072000061E070E080E090E00E940C7FC701B60171
:1072100023E030E040E050E00E94F8A9672B682BA3
:10722000692B09F0F8C043E050E058A74FA3812C28
:10723000912C540180910E02863308F086532091E0
:107240007B00982F9870277F922B90937B008770FC
:10725000806480937C0080917A00806480937A00BF
:1072600080917A0086FDFCCF809178006091790052
:10727000762F682F072E000C880B990B0E9493A87D
:107280009B01AC01C501B4010E943AAA4B015C010B
:1072900062E070E080E090E00E940C7F8FA198A5F2
:1072A000019798A78FA3892B29F620E030ED4FE3B3
:1072B00055E4C501B4010E94A6AA4B015C0180916E
:1072C000EB0B882399F12DEC3CEC4CE45EE3C5011B
:1072D000B4010E944EAB87FD29C022E0B501A40194
:1072E000CE0107960E94AD7A6BE175E0CE01019662
:1072F0000E943E7BBE01695F7F4FCE0101960E94D6
:10730000C079BC01CE010D960E94357BCE010D9651
:107310000E94691FCE010D960E94A57ACE010196AA
:107320000E94A57ACE0107960E94A57A2AE939E93A
:1073300049E95EE3C501B4010E944EAB87FD13C06D
:10734000411451046104710411F42601370129A587
:107350003AA54BA55CA5232B242B252B21F4C9A6EC
:10736000DAA6EBA6FCA62DEC3CEC4CE45EE3C501F2
:10737000B4010E948CA818160CF448C041145104A2
:107380006104710409F447C08BA19CA1ADA1BEA109
:10739000892B8A2B8B2B69F42DA53EA54FA558A9C7
:1073A000232B242B252B09F47DC0CBA2DCA2EDA23C
:1073B000FEA28BA19CA1ADA1BEA1481659066A06EA
:1073C0007B064CF580910A0290910B0297FF6FC0EB
:1073D00010920B0210920A022BA13CA14DA15EA1BA
:1073E000420E531E641E751ED301C201B595A795AA
:1073F000979587958FAB98AFA9AFBAAF1BA21CA288
:107400001DA21EA2412C512C320105C04114510471
:107410006104710471F6A0910A02B0910B02B8A741
:10742000AFA3A230B1050CF05EC0B7FD03C00330BE
:107430001105B1F0BFEFCB1ADB0AEB0AFB0AE0E45F
:10744000CE16ECE9DE06E104F10409F0C9CE033002
:10745000110531F05BADE52E0115110509F07CCD6C
:10746000C1010E94EB786B017C01C092FA0BD092B3
:10747000FB0BE092FC0BF092FD0B20E030E044EBC4
:1074800053E4C701B6010E944EAB87FDDEC020E089
:1074900030E044EB53E4C701B6010E9439AA6B0106
:1074A0007C01EBCFCDA6DEA6EFA6F8AA7ECF011514
:1074B000110509F0B0CF019690930B0280930A0258
:1074C0002BA13CA14DA15EA1420E531E641E751E50
:1074D000D301C201B595A795979587958BAB9CABCA
:1074E000ADABBEAB8BCF6BA97CA98DA99EA92FA9F3
:1074F00038AD49AD5AAD621B730B840B950B0E94DE
:1075000093A84B015C014FA158A5BA01550F880BF8
:10751000990B0E9493A89B01AC01C501B4010E9484
:10752000A6AA20E030E044EB53E40E94A6AA4B0157
:107530005C018092240290922502A0922602B092D1
:10754000270220E030E040E85FE30E944EAB87FD79
:1075500058C08091690290916A0281309105F1F5DD
:107560008092F3139092F413A092F513B092F61355
:107570008092200290922102A0922202B0922302D5
:107580006DE975E0CE0101960E942C7BCE0101963B
:107590000E94801FCE0101960E94A57A409124028C
:1075A00050912502609126027091270225E0CE01BC
:1075B00001960E94AD7ACE0101960E94691FCE010C
:1075C00001960E94A57A84EF91E090939D028093AA
:1075D0009C0265ED72E10E944F0939CF029781F656
:1075E0008092F7139092F813A092F913B092FA13C5
:1075F00080921C0290921D02A0921E02B0921F0265
:10760000BFCF61E875E0CE0101960E942C7BCE01D0
:1076100001960E94801FCE0101960E94A57A40919A
:10762000240250912502609126027091270225E0E4
:10763000CE0101960E94AD7ACE0101960E94691F8B
:10764000CE0101960E94A57A02CF20E030E0A90188
:10765000C701B6010E948CA887FF0BC020E030E074
:1076600044EB53E4C701B6010E943AAA6B017C01C6
:10767000ECCFC092B10BD092B20BE092B30BF09270
:10768000B40B4DA45EA46FA478A889A59AA5ABA558
:10769000BCA5481A590A6A0A7B0A01151105D9F4D2
:1076A0001092B10B1092B20B1092B30B1092B40B5C
:1076B000A9A9BAA9812C912C54018394C12CD12C55
:1076C0007601B7FF26C0C12CD12C760188248A947C
:1076D000982C54011EC0E9A9FAA9812C912C5401BF
:1076E0008394F7FF04C088248A94982C5401C09096
:1076F000B10BD090B20BE090B30BF090B40B20E044
:1077000030E044E353E4C701B6010E948CA887FF30
:1077100092C0C701B60190582091240230912502F1
:1077200040912602509127020E94F2A86B017C0131
:10773000A3019201C501B4010E94C6A90E9493A8A9
:1077400020E030E040E05FE30E94F2A89B01AC0142
:10775000C701B6010E9439AA0E9418AB60931002BB
:107760007093110280931202909313028091EB0B9D
:10777000882309F441C02AE04DA55EA56FA578A92C
:10778000CE010D960E94DD7A2AE049A55AA56BA587
:107790007CA5CE0107960E94DD7A62E275E0CE01FB
:1077A00001960E943E7BBE01695F7F4FCE0101962C
:1077B0000E94C07961E876E00E94AA79BE01635F09
:1077C0007F4F0E94C079BC01CE0143960E94357B59
:1077D000CE0143960E94691FCE0143960E94A57A6E
:1077E000CE0101960E94A57ACE0107960E94A57A45
:1077F000CE010D960E94A57A8091100290911102FF
:10780000A0911202B0911302B7FF36C0B095A095B7
:10781000909581959F4FAF4FBF4F809310029093EB
:107820001102A0931202B0931302EE24E394F12C00
:1078300036E43F8F91CB2091240230912502409174
:107840002602509127022F8F38A349A35AA3A701DC
:10785000960160E070E084EB93E40E9439AA6093A3
:10786000B10B7093B20B8093B30B9093B40B2F8D2D
:1078700038A149A15AA158CFE12C42E54F8F6CCBDA
:10788000EE24E394F12C7DCBE12C7BCB023011056F
:1078900024F40115110509F0E0C061E080E00E94C8
:1078A0009D890330110521F00115110509F09CC0D7
:1078B000C090FA0BD090FB0BE090FC0BF090FD0B0E
:1078C00020E030E044EB53E4C701B6010E944EAB28
:1078D00087FD0BC020E030E044EB53E4C701B60164
:1078E0000E9439AA6B017C01EBCF20E030E0A901B6
:1078F000C701B6010E948CA887FF0BC020E030E0D2
:1079000044EB53E4C701B6010E943AAA6B017C0123
:10791000ECCFC092FA0BD092FB0BE092FC0BF092F2
:10792000FD0B8091690290916A020197B1F46CEDB0
:1079300074E082EB91E10E9479788091FA0B90914A
:10794000FB0BA091FC0BB091FD0B8093450C909329
:10795000460CA093470CB093480C8091690290911B
:107960006A020297B1F46BEE74E082EB91E10E943F
:1079700079788091FA0B9091FB0BA091FC0BB09160
:10798000FD0B8093410C9093420CA093430CB09359
:10799000440C4091FA0B5091FB0B6091FC0B7091E1
:1079A000FD0B21E0CE0107960E94AD7A62EB71E1FA
:1079B000CE0101960E94357BBE01695F7F4FCE01EB
:1079C00001960E94C07966EE74E00E94AA79BC011B
:1079D00082EB91E10E94557ACE0101960E94A57A30
:1079E000CE0107960E94A57A0130110509F0C8C0A2
:1079F0004091100250911102609112027091130295
:107A000021E0CE0107960E94DD7A6AE275E0CE01A0
:107A100001960E943E7BBE01695F7F4FCE010196B9
:107A20000E94C079BC0182EB91E10E94557ACE019F
:107A300001960E94A57ACE0107960E94A57A62EB74
:107A400071E1CE0101960E94357BCE0101960E9424
:107A50003027CE0101960E94A57A10921002109252
:107A600011021092120210921302809169029091F9
:107A70006A028130910509F0D9C08091BB0B9091C9
:107A8000BC0B9093BE0B8093BD0B80911002909124
:107A90001102A0911202B0911302809314029093EC
:107AA0001502A0931602B0931702809130029091B4
:107AB0003102A0913202B091330280932C02909354
:107AC0002D02A0932E02B0932F028091B90B8093C8
:107AD000BA0B8091B10B9091B20BA091B30BB09106
:107AE000B40B8093B50B9093B60BA093B70BB093E8
:107AF000B80B8091FA0B9091FB0BA091FC0BB0910D
:107B0000FD0B8093450C9093460CA093470CB093CB
:107B1000480C80910A0290910B0290930D02809381
:107B20000C02012B81F48091240290912502A091F6
:107B30002602B09127028093200290932102A09305
:107B40002202B0932302CE0149960E94A57AEB96B9
:107B50000FB6F894DEBF0FBECDBFDF91CF911F915E
:107B60000F91FF90EF90DF90CF90BF90AF909F90DC
:107B70008F907F906F905F904F903F902F900895DF
:107B80000230110509F05BCFC090FA0BD090FB0BCF
:107B9000E090FC0BF090FD0B20E030E044EB53E470
:107BA000C701B6010E944EAB87FD0BC020E030E05C
:107BB00044EB53E4C701B6010E9439AA6B017C0172
:107BC000EBCF20E030E0A901C701B6010E948CA8EC
:107BD00087FF0BC020E030E044EB53E4C701B6015F
:107BE0000E943AAA6B017C01ECCFC092FA0BD092B2
:107BF000FB0BE092FC0BF092FD0B21E0B701A6011C
:107C0000CE0107960E94AD7A61E375E0CE01019640
:107C10000E943E7BBE01695F7F4FCE0101960E94AC
:107C2000C07967EE74E00E94AA79FCCE029709F051
:107C30008ACF8091BB0B9091BC0B9093B00B80933B
:107C4000AF0B8091100290911102A0911202B0919D
:107C500013028093060290930702A0930802B09348
:107C600009028091300290913102A0913202B091CC
:107C700033028093280290932902A0932A02B093A2
:107C80002B028091B90B8093AE0B8091B10B909138
:107C9000B20BA091B30BB091B40B8093AA0B90934D
:107CA000AB0BA093AC0BB093AD0B8091FA0B909102
:107CB000FB0BA091FC0BB091FD0B8093410C9093BA
:107CC000420CA093430CB093440C80910A02909113
:107CD0000B029093050280930402012B09F033CF2D
:107CE0008091240290912502A0912602B091270252
:107CF00080931C0290931D02A0931E02B0931F025A
:107D000022CF2F923F924F925F926F927F928F92EB
:107D10009F92AF92BF92CF92DF92EF92FF920F931A
:107D20001F93CF93DF93CDB7DEB7CB54D1090FB6F6
:107D3000F894DEBF0FBECDBF40E052EC61E070E0D2
:107D400081E89FE00E94AA7540E855E260E070E09B
:107D500084EE9EE00E94AA7561E088E00E94B67EF3
:107D600061E089E00E94B67E60E08AE30E94B67E10
:107D700061E088E00E94997D60E089E00E94997D41
:107D800061E08AE00E94B67E61E08BE00E94B67EF0
:107D900060E08BE30E94B67E61E08AE00E94997DFC
:107DA00060E08BE00E94997D0E949F7E84EF91E0CD
:107DB00090939D0280939C0268EE73E080E090E0D7
:107DC0000E940C7F81E89FE00E94E472F82E6AE036
:107DD000C62ED12CF1100BC081E89FE00E94E47206
:107DE000F82E6EE170E080E090E00E940C7F21E0D0
:107DF000C21AD10879F780919C0290919D0205EDFD
:107E000012E15FEF852E53E1952E3801FC01E55D0F
:107E1000F2415F01C501860D971D0E94B0A9F301D3
:107E200081933F018E169F06A9F76091EF13709121
:107E3000F013072E000C880B990B0E9493A89B014E
:107E4000AC010E9453AB882331F081E090E0909325
:107E5000F0138093EF136091F1137091F213072EDA
:107E6000000C880B990B0E9493A89B01AC010E9407
:107E700053AB882331F082E090E09093F21380932B
:107E8000F113F5E7FF16B1F06091EB137091EC136D
:107E90008091ED139091EE130E9493A89B01AC0189
:107EA0000E9453AB811106C08091D5129091D612D9
:107EB0008197E8F02DB73EB72A5231400FB6F894BB
:107EC0003EBF0FBE2DBFADB7BEB711968AE291E09F
:107ED000E5EDF2E101900D920197E1F70E94582D36
:107EE0000FB6F894DEBF0FBECDBF45E7F42EEDB759
:107EF000FEB7EA52F1400FB6F894FEBF0FBEEDBFD9
:107F0000ADB7BEB711968AE291E0E5EDF2E10190DE
:107F10000D920197E1F70E94DC220FB6F894DEBFC4
:107F20000FBECDBF35E7F31619F083E7F8121BC07B
:107F3000EDB7FEB7EA52F1400FB6F894FEBF0FBEA0
:107F4000EDBFADB7BEB711968AE291E0E5EDF2E183
:107F500001900D920197E1F70E947B320FB6F894E1
:107F6000DEBF0FBECDBF62EC7AE083E092E10E94FB
:107F7000307A6CEA7AE08DEF91E10E94307A0E94CB
:107F80009F7E68E375E081E89FE00E946B7CB12CE6
:107F9000A12C37E2E32E992493949092DF0EE09285
:107FA000E10E1092E00E1092E20E81E00E946F88C6
:107FB0008111C1C164E475E081E89FE00E947F7C8B
:107FC0008E2D0E94F47BE092871460E675E081E8D4
:107FD0009FE00E947F7C8E2D0E94F47B3FEFA31ACE
:107FE000B30AE39480E4E812D8CF65E975E0AB28E2
:107FF00011F06BEA75E081E89FE00E946B7C0E94C3
:108000009F7E1092881480918C14823018F098E032
:108010009093881490918D14992339F0813029F42C
:108020008091881484608093881462E370E080E01B
:1080300090E00E940C7F60918E1483E894E10E948E
:108040005F8968EE73E080E090E00E940C7F60E35F
:1080500083E894E10E9473898BE4A82E86E4B82E0D
:10806000C5010197F1F760E383E894E10E94738909
:10807000C5010197F1F760E383E894E10E947389F9
:1080800083E592E00197F1F760E283E894E10E94D2
:1080900073898091881480620E948C8984E0809327
:1080A00089148CE00E948C8981E00E948C899BE37A
:1080B000A92E9FE1B92EC5010197F1F782E08093C7
:1080C0008A1486E00E948C8982E00E948C89C50116
:1080D0000197F1F780E40E948C8924E9A22E22E026
:1080E000B22EF50161915F0183E894E10E94FB8962
:1080F000FCE9AF16F2E0BF06A1F70E942E0A0E942B
:10810000120A64E670E080E090E00E940C7F64E96F
:108110007AE0CE0101960E942C7BCE0101960E944E
:10812000691FCE0101960E94A57A61E085E30E9455
:10813000B67E61E085E30E94997D61E08AE00E945D
:10814000B67E61E08AE00E94997D61E084E00E9451
:10815000B67E61E084E00E94997D61E089E30E943F
:10816000B67E80910C11803308F052C061E089E343
:108170000E94B67E80910C11282F30E0F901EE0F9D
:10818000FF1FE20FF31FE758FF4E9081907C996329
:10819000908310920D1110920E112CE0622F0E940C
:1081A00058AB829FB00111249B012C0D3D1DF9019C
:1081B000EE0FFF1FE20FF31FE758FF4E908196FD71
:1081C00019C02FEFC21AD20A3CE0C316D10461F7DE
:1081D000813009F0BDC01092800082E08093810060
:1081E0001092850010928400B19A80916F00826095
:1081F00080936F00E0910C118E2F90E0FC01EE0F48
:10820000FF1FE80FF91FE758FF4E808180648083CD
:1082100068EC70E080E090E00E940C7F68EE73E014
:1082200080E090E00E940C7F63E87AE0CE01019646
:108230000E942C7B4AE050E06FEF7FEFCE01019669
:108240000E949020CE0101960E94A57A10923510CE
:10825000109233101092301010922F1084E08093FF
:108260002E100E94DB816B0161E080912E100E9434
:10827000B67E8AE290E10E94560860E082E30E94A6
:10828000B67E61E083E30E94B67E61E084E30E94F3
:10829000B67E61E085E30E94B67E61E085E30E94E0
:1082A000997D83E58CBD8DB58E7F8DBD6AE0E62E10
:1082B0008FEF0E94DC06EA94E110FACF60E0809133
:1082C0002E100E94997D20E030E0A90160E08AE252
:1082D00090E10E946310E82E8093341081E0E8164C
:1082E00009F462C00E94DB816C197D09613D774011
:1082F00050F381E080932F108AE290E10E945608AB
:1083000065E77AE0CE0101960E942C7BCE010196B2
:108310000E94691FCE0101960E94A57A64E67AE068
:10832000CE0101960E942C7B6AE070E0CE0101969E
:108330000E94CA8958C1843009F053CE6AE775E0BB
:1083400081E89FE00E947F7C8E2D0E94F47B49CEC5
:10835000823061F410929000809391001092950009
:108360001092940088BB8093710044CF833069F4ED
:108370001092A00082E08093A1001092A5001092BC
:10838000A40089BB8093720035CF811133CF109246
:10839000200182E080932101109225011092240196
:1083A0008ABB8093730026CF2AEA31E040E050E098
:1083B00068E08AE290E10E94631082FF2AC0E092A6
:1083C000351080913510812C912C5401823029F484
:1083D000812C912CA12C40E4B42E20E030E0A901A6
:1083E00067E38AE290E10E946310A501940169E2CB
:1083F0008AE290E10E946310809334108823D1F0C8
:108400000E94DB816C197D09613D774030F388E083
:1084100071CF54E0E52E0E945E1080933410EA94F0
:10842000E110F9CF8A3A11F082E064CF82E08093C4
:108430003510C7CF809135108230D1F420E030E084
:10844000A9016AE38AE290E10E946310882311F097
:1084500086E050CF0E945E10807C803C19F483E05F
:10846000809335100E945E100E945E100E945E1084
:108470008AE290E10E9456088DB58E7F8DBD8CB545
:108480008C7F8CBD8CB58CBD81E00E940B8C8823C9
:1084900009F464C180915910811132CF80914D103F
:1084A000803109F062C182E08093591010926B1004
:1084B00010926C1010926D1010926E1080914E10F0
:1084C00090914F10B0E0A0E035E0880F991FAA1FEF
:1084D000BB1F3A95D1F78093671090936810A093D3
:1084E0006910B0936A1086E390E1909370108093C6
:1084F0006F1081E08093581010925A1010925B1008
:1085000010925C1010925D1010925E1010925F102D
:10851000109260101092611010926210109263100D
:1085200010926410109265101092661068E57AE05F
:10853000CE0101960E942C7BCE0101960E94691FFC
:10854000CE0101960E94A57A41E06EE174E0CE0171
:1085500001960E94BE92BE016F5F7F4F8CE494E152
:108560000E94971F80914E1490914F149C838B838F
:108570008091501490915114A0915214B0915314C1
:108580008D839E83AF83B887809154149091551446
:10859000A0915614B091571489879A87AB87BC87EE
:1085A0008EED93E09A8389838DE0E8E5F4E1DE01C6
:1085B0001D9601900D928A95E1F780916514909136
:1085C00066149B8F8A8F70E060E0CE0101960E9456
:1085D0005C2162E57AE0CE0101960E942C7BCE01FF
:1085E00001960E94691FCE0101960E94A57A68EE4D
:1085F00073E080E090E00E940C7F43E160ED72E068
:10860000CE0101960E94BE92BE016F5F7F4F87E64A
:1086100094E10E94971F6AE17AE081EF91E10E9464
:10862000307A6FE07AE081EF91E10E94D37987E6BA
:1086300094E10E941912882309F4B6C061E370E145
:1086400080ED92E00E94E276811122C062EB75E03B
:10865000CE0101960E943E7BCE0101960E94801FB2
:10866000CE0101960E94A57A60ED72E0CE010196DE
:108670000E943E7BCE0101960E94691FCE010196A9
:108680000E94A57A61EF71E187E694E10E94957CF2
:1086900087E694E10E94251266E970E080E090E0B0
:1086A0000E940C7F64EC75E0CE0101960E943E7B37
:1086B000CE0101960E94691FCE0101960E94A57A03
:1086C0001092AA0C6CEE79E0CE0101960E942C7BF0
:1086D000CE0101960E94691FCE0101960E94A57AE3
:1086E0000E94CA7F5C0168EE73E080E090E00E9427
:1086F0000C7FD12CC12CAB2809F017C5FAE0CF169E
:10870000D10409F4D0C2B601CE0101960E9483784B
:10871000CE0101960E94691FCE0101960E94A57AA2
:1087200060ED77E080E090E00E940C7F0E94CA7FBD
:108730005C0168EE73E080E090E00E940C7FCE0167
:1087400001960E94261EBE016F5F7F4F81E89FE069
:108750000E94557C2FEFC21AD20ACDCF80E00E9432
:108760000B8C882309F4CCCD95CE803209F0C8CD8E
:1087700083E08093591040915010509151106091B6
:1087800052107091531040936B1050936C10609383
:108790006D1070936E1027E630E186E390E10E9441
:1087A000578E8111A0CEACCD6AEF79E0CE01019653
:1087B0000E942C7BCE0101960E94801FCE01019663
:1087C0000E94A57A60ED72E06FCF80E0ECC2F40108
:1087D0001182108261EE72E1CE0188960E943E7B8A
:1087E000B801645E7F4FCE0182960E943E7BB70146
:1087F000CE014C960E94837866ED75E0CE0101961D
:108800000E943E7BBE01645E7F4FCE0101960E94B6
:10881000C07965E677E00E94AA79BE016E5D7F4F60
:108820000E94C07964E876E00E94AA79BE01685D82
:108830007F4F0E94C079BC012B968FAD2B972C9651
:108840009FAD2C970E94297ACE0101960E94A57AAD
:10885000CE014C960E94A57ACE0182960E94A57AFE
:10886000CE0188960E94A57AF301108211821282AD
:108870001382F2011082118212821382C7010E94B8
:10888000421EFFEFEF1AFF0A2A960EAD1FAD2A9780
:1088900069C3CE014C960E9463276AED75E0CE0154
:1088A00001960E943E7BBE01645E7F4FCE01019621
:1088B0000E94C07961E876E00E94AA79BE01605CFE
:1088C0007F4F0E94C079BC018BE192E10E94557AF2
:1088D000CE0101960E94A57ACE014C960E94A57AFF
:1088E000CE0101960E94632746E150E0BE016F5F12
:1088F0007F4FCE014C960E944920BE01645E7F4F9F
:10890000CE0182960E94357BBE01665C7F4FCE0110
:1089100082960E94C079BC01CE01CA960E94557A07
:10892000CE0182960E94A57ACE014C960E94A57A2D
:10893000CE0101960E94A57A6BE172E1CE0101960B
:108940000E94357BCE0101960E94691FCE010196DF
:108950000E94A57A6BE172E1CE0101960E94357BFF
:10896000AE014F5F5F4F62E070E088E792E00E94E7
:10897000FB2E182FCE0101960E94A57A111121C05D
:108980006BE172E1CE0101960E94357B6AEC75E0E5
:10899000CE0101960E94AA796DEF71E10E94C07923
:1089A000BC01CE014C960E94357BCE014C960E94B4
:1089B000691FCE014C960E94A57ACE0101960E94B5
:1089C000A57ABE01665C7F4FCE0101960E94357B81
:1089D000AE014F5F5F4F63E070E08BE692E00E9474
:1089E000FB2ECE0101960E94A57ACE01C4960E946C
:1089F000A57ACE01CA960E94A57AC6010E94A57AE0
:108A000001E010E010936A0200936902109368027B
:108A10000093670264EE75E08CEA91E10E94797838
:108A200063E879E0CE0101960E942C7BCE0101968D
:108A30000E94691FCE0101960E94A57A6CEA71E13D
:108A4000CE0101960E94357B62E070E0CE01019676
:108A50000E94A535CE0101960E94A57A63E779E0D0
:108A6000CE0101960E942C7BCE0101960E943027F8
:108A7000CE0101960E94A57A67E377E08CEA91E146
:108A80000E94797862E679E0CE0101960E942C7B03
:108A9000CE0101960E94691FCE0101960E94A57A1F
:108AA0006CEA71E1CE0101960E94357B63E070E0D3
:108AB000CE0101960E94A535CE0101960E94A57AAD
:108AC00082E090E090936A02809369028091FB13A8
:108AD0009091FC13909368028093670266E579E0B9
:108AE000CE0101960E942C7BCE0101960E94302778
:108AF000CE0101960E94A57A67E377E08CEA91E1C6
:108B00000E9479786CEA71E1CE0101960E94357B72
:108B100063E070E0CE0101960E94A535CE0101967A
:108B20000E94A57A8091FB139091FC1391958195F9
:108B300091099093FC138093FB13109368020093A8
:108B4000670284EF91E090939D0280939C0265ED13
:108B500072E10E944F0964E670E080E090E00E94BC
:108B60000C7F10936A020093690287E29EE690935D
:108B70008411809383112091A511822F022E000C65
:108B8000990B88309105C8F4FC01EE0FFF1FEE0F22
:108B9000FF1FEB57FE4E48EE55E0518340832F5F99
:108BA0002093A511880F991F880F991FFC01E95781
:108BB000FE4E83EC9AE6918380832091A511822F4B
:108BC000022E000C990B88309105C8F4FC01EE0FC1
:108BD000FF1FEE0FFF1FEB57FE4E4EEE55E0518389
:108BE00040832F5F2093A511880F991F880F991F2D
:108BF000FC01E957FE4E8CEB91E79183808383E182
:108C000091E10E94241D64E479E0CE0101960E9466
:108C10002C7BCE0101960E94691FCE0101960E9415
:108C2000A57A0E94398660933A0C70933B0C80932E
:108C30003C0C90933D0C10923E0C0E94F1260E9439
:108C400039866093550C7093560C8093570C909313
:108C5000580C8091D4138093AC0C882351F00E945F
:108C6000398660934D0C70934E0C80934F0C90930B
:108C7000500CC55BDF4F0FB6F894DEBF0FBECDBF03
:108C8000DF91CF911F910F91FF90EF90DF90CF90E8
:108C9000BF90AF909F908F907F906F905F904F901C
:108CA0003F902F90089560EE79E0CE0101960E94EA
:108CB0002C7BCE0101960E94691FCE0101960E9475
:108CC000A57A68EE73E080E090E00E940C7F61E39B
:108CD00070E187E892E00E94E276882331F061EF4C
:108CE0007FE087E892E00E94E27666E970E080E04B
:108CF00090E00E940C7F43E167E872E0CE010196AC
:108D00000E94BE92BE016F5F7F4F87E694E10E9492
:108D1000971F81E08093AA0CCE0101960E94261E27
:108D2000BE016F5F7F4F87E694E10E94557C87E626
:108D300094E10E94251262E370E080E090E00E94DE
:108D40000C7F1092AA0C0E946F2B68EE73E080E0FB
:108D500090E00E940C7F0E949B3024E6C22ED12C12
:108D6000F1100BC081E89FE00E94E472F82E64E1EC
:108D700070E080E090E00E940C7F31E0C31AD108DF
:108D800079F763EC79E0CE0101960E942C7BCE014D
:108D900001960E943027CE0101960E94A57A82E7B3
:108DA000F81213CD81E00E94800969EB79E08BE134
:108DB00092E10E94307ACE0101960E946327BE01A3
:108DC0006F5F7F4F8BE192E10E94297ACE0101967D
:108DD0000E94A57A66EA79E08BE192E10E94D3795C
:108DE00064E979E0CE0101960E942C7BCE010196C8
:108DF0000E943027CE0101960E94A57A67E370E0B9
:108E000080918502909186020E94520A90930F0CE5
:108E100080930E0C6BE172E1CE0101960E94357BCE
:108E2000AE014F5F5F4F62E070E088E792E00E9422
:108E3000FB2EF82ECE0101960E94A57AF11021C0DA
:108E40006BE172E1CE0101960E94357B6AEC75E020
:108E5000CE0101960E94AA796DEF71E10E94C0795E
:108E6000BC01CE014C960E94357BCE014C960E94EF
:108E7000691FCE014C960E94A57ACE0101960E94F0
:108E8000A57A6BE172E1CE0101960E94357BAE01BD
:108E90004F5F5F4F63E070E08BE692E00E94FB2E35
:108EA000F82ECE0101960E94A57AF11021C06BE147
:108EB00072E1CE0101960E94357B6AEC75E0CE012D
:108EC00001960E94AA796DEF71E10E94C079BC0100
:108ED000CE014C960E94357BCE014C960E94691FB4
:108EE000CE014C960E94A57ACE0101960E94A57AE9
:108EF00068EE73E080E090E00E940C7F6E0190E4E9
:108F0000C90ED11C67E074E0C6010E943E7B67E099
:108F100074E0CE01CA960E943E7B67E074E0CE0109
:108F2000C4960E943E7BE091A802F091A902289687
:108F3000FFAFEEAF2897A2EA8A2EA2E09A2EBBE5F9
:108F4000AB2EB2E0BB2E8FE4282E82E0382E21011A
:108F50003501EE24E394F12C2B96CFAE2B972C9673
:108F6000DFAE2C97F2E08F0E911C9801285F3F4FE7
:108F70002A963FAF2EAF2A9734E0630E711C84E02F
:108F8000480E511C2896EEADFFAD2897EE15FF0553
:108F90000CF01DCC73E4872E72E0972EE9E4EE2EE0
:108FA000E2E0FE2E01E010E0F8EE4F2EF3E05F2E3F
:108FB000612C712C22E0820E911C34E0A30EB11CB6
:108FC00082E0E80EF11C94E0290E311C8091A80289
:108FD0009091A902801791070CF45BCCF401608199
:108FE0007181CE0188960E94837842E050E0BE01F4
:108FF000685D7F4FCE018E960E944920B801CE0158
:109000004C960E94837842E050E0BE01645E7F4F40
:10901000CE0182960E94492060E178E0CE0101965F
:109020000E943E7BBE016E5D7F4FCE0101960E9485
:10903000C079BE01625D7F4F0E94C079BC01CE0144
:10904000C4960E94557ACE0101960E94A57ACE015F
:1090500082960E94A57ACE014C960E94A57ACE01F6
:109060008E960E94A57ACE0188960E94A57AF50177
:109070006081718182819381A30192010E94F8A98C
:10908000BA01A90120E0CE0101960E94DD7A48E0F4
:1090900050E0BE016F5F7F4FCE014C960E94492089
:1090A000BE01645E7F4FCE01C4960E94297ACE0134
:1090B0004C960E94A57ACE0101960E94A57AF701EE
:1090C00060817181CE0101960E94837843E050E077
:1090D000BE016F5F7F4FCE014C960E944920BE01BA
:1090E000645E7F4FCE01C4960E94297ACE014C96D1
:1090F0000E94A57ACE0101960E94A57ABE016C5C01
:109100007F4FCE01CA960E94297AF5011082118202
:1091100012821382F1011082118212821382C8011D
:109120000E94421E0F5F1F4F45CF63ED79E0BDCD1A
:109130004F925F926F927F928F929F92AF92BF9267
:10914000CF92DF92EF92FF920F931F93CF93DF9313
:10915000CDB7DEB7ED970FB6F894DEBF0FBECDBF2B
:109160006AEC71E1CE01C4960E94357B0CA91DA961
:109170000115110571F0F80181918F01882349F0E3
:10918000082E000C990B0E94A6ADF8013197808340
:10919000F2CF62EF75E0CE0101960E943E7BBE01E8
:1091A0006F5F7F4FCE01C4960E948F79182FCE013A
:1091B00001960E94A57A112309F4FFC045E050E012
:1091C0006AEC71E1CE0101960E94220ABE016F5F36
:1091D0007F4F8CEA91E10E946C7ACE0101960E9449
:1091E000A57A8CEA91E10E94017960E08CEA91E134
:1091F0000E94FD794091B0115091B1116DE273E17F
:109200008CEA91E10E94AA766EE174E0CE010196AB
:109210000E943E7BBE016F5F7F4F8CEA91E10E940E
:109220008F79182FCE0101960E94A57A68E074E02C
:10923000111102C06DE074E0CE0101960E943E7BE8
:109240006CEA71E1CE0101960E94C079BC018BE20B
:1092500094E10E94557ACE0101960E94A57A8BE294
:1092600094E10E94017940912F14509130144150A3
:1092700051096BE274E1CE0101960E94220ABE01FF
:109280006F5F7F4F8DE094E10E946C7ACE01019672
:109290000E94A57A8DE094E10E94F6780E9493A83E
:1092A0009B01AC010E9453AB882309F448C0609134
:1092B0002F1470913014625071098BE294E10E9476
:1092C0005E79682FCE0101960E940A7BBE016F5F16
:1092D0007F4F8DE094E10E946C7ACE0101960E944E
:1092E000A57A6EE174E0CE0101960E943E7BBE013C
:1092F0006F5F7F4F8DE094E10E948F79182FCE0130
:1093000001960E94A57A1123D1F060912F147091DB
:109310003014635071098BE294E10E945E79682FEA
:10932000CE0101960E940A7BBE016F5F7F4F8DE0E8
:1093300094E10E946C7ACE0101960E94A57A84EF96
:1093400091E090939D0280939C0265ED72E10E94F2
:109350004F0964E670E080E090E00E940C7F80910D
:109360003402882371F06AEC71E1CE0101960E940B
:10937000357BCE0101960E94F124CE0101960E9418
:10938000A57ACE01C4960E94A57A81E0ED960FB62B
:10939000F894DEBF0FBECDBFDF91CF911F910F912B
:1093A000FF90EF90DF90CF90BF90AF909F908F9005
:1093B0007F906F905F904F90089568EF75E0CE01B9
:1093C00001960E943E7BBE016F5F7F4FCE01C49627
:1093D0000E948F79182FCE0101960E94A57A112341
:1093E00009F447C045E050E06AEC71E1CE01019616
:1093F0000E94220ABE016F5F7F4F8CEA91E10E94BA
:109400006C7ACE0101960E94A57A8CEA91E10E94C5
:10941000017960E08CEA91E10E94FD794091B01100
:109420005091B11165E073E18CEA91E10E94AA7656
:1094300065E073E1CE014C960E943E7B60E274E0F1
:10944000CE0101960E943E7BBE01645E7F4FCE013D
:1094500001960E94C079BC0185E294E10E94557A90
:10946000CE0101960E94A57ACE014C960E94A57A63
:1094700066CF6EEF75E0CE0101960E943E7BBE0185
:109480006F5F7F4FCE01C4960E948F79182FCE0157
:1094900001960E94A57A1123E1F043E050E06AECC6
:1094A00071E1CE0101960E94220ABE016F5F7F4FDB
:1094B0008CEA91E10E946C7ACE0101960E94A57A15
:1094C0006CEA71E1CE0101960E94357BCE010196D6
:1094D000CDCF62E076E0CE0101960E943E7BBE01D8
:1094E0006F5F7F4FCE01C4960E948F79182FCE01F7
:1094F00001960E94A57A112301F144E050E06AEC44
:1095000071E1CE0101960E94220ABE016F5F7F4F7A
:109510008CEA91E10E946C7ACE0101960E94A57AB4
:109520008CEA91E10E94F678709394136093931300
:10953000709386026093850202CF67E076E0CE01E9
:1095400001960E943E7BBE016F5F7F4FCE01C496A5
:109550000E948F79182FCE0101960E94A57A1123BF
:1095600009F449C045E050E06AEC71E1CE01019692
:109570000E94220ABE016F5F7F4F8CEA91E10E9438
:109580006C7ACE0101960E94A57A8CEA91E10E9444
:10959000F6787093F0136093EF1384EF91E090935B
:1095A0009D0280939C0265ED72E10E944F0964E682
:1095B00070E080E090E00E940C7F60E178E0CE01F6
:1095C00001960E943E7B6AEC71E1CE0101960E94F9
:1095D000C079BC01CE014C960E94357BCE014C96E1
:1095E0000E94691FCE014C960E94A57ACE01019679
:1095F0000E94A57AB4CE6DE076E0CE0101960E947D
:109600003E7BBE016F5F7F4FCE01C4960E948F7973
:10961000182FCE0101960E94A57A1123E1F044E0B3
:1096200050E06AEC71E1CE0101960E94220ABE016F
:109630006F5F7F4F8CEA91E10E946C7ACE010196B8
:109640000E94A57A8CEA91E10E94F6787093F21359
:109650006093F113A2CF62E176E0CE0101960E9401
:109660003E7BBE016F5F7F4FCE01C4960E948F7913
:10967000182FCE0101960E94A57A1123A1F044E093
:1096800050E06AEC71E1CE0101960E94220ABE010F
:109690006F5F7F4F8CEA91E10E946C7ACE01019658
:1096A0000E94A57A84CF67E176E0CE0101960E9400
:1096B0003E7BBE016F5F7F4FCE01C4960E948F79C3
:1096C000182FCE0101960E94A57A1123A1F047E040
:1096D00050E06AEC71E1CE0101960E94220ABE01BF
:1096E0006F5F7F4F8CEA91E10E946C7ACE01019608
:1096F0000E94A57A2ECE6FE176E0CE0101960E94FF
:109700003E7BBE016F5F7F4FCE01C4960E948F7972
:10971000182FCE0101960E94A57A1111D8CF67E2C9
:1097200076E0CE0101960E943E7BBE016F5F7F4FC7
:10973000CE01C4960E948F79182FCE0101960E9407
:10974000A57A112321F081E00E94800902CE61E315
:1097500076E0CE0101960E943E7BBE016F5F7F4F97
:10976000CE01C4960E948F79182FCE0101960E94D7
:10977000A57A112319F00E949B30EBCD68E376E0C7
:10978000CE0101960E943E7BBE016F5F7F4FCE01EE
:10979000C4960E948F79182FCE0101960E94A57A57
:1097A000112309F454C04AE050E06AEC71E1CE01A3
:1097B00001960E94220ABE016F5F7F4F8CEA91E101
:1097C0000E946C7ACE0101960E94A57A8CEA91E102
:1097D0000E94F6780E9414860E94398660934D0C90
:1097E00070934E0C80934F0C9093500C0E943986CE
:1097F0006093510C7093520C8093530C9093540CC3
:10980000CE014C960E94632763E476E0CE01019678
:109810000E943E7BBE01645E7F4FCE0101960E9496
:10982000C079BC01CE0182960E94357BCE01829622
:109830000E94691FCE0182960E94A57ACE010196F0
:109840000E94A57ACE014C960E94A57A88CD69EA3D
:1098500077E0CE0101960E943E7BBE016F5F7F4F95
:10986000CE01C4960E948F79182FCE0101960E94D6
:10987000A57A112309F46CC045E050E06AEC71E16F
:10988000CE0101960E94220ABE016F5F7F4F8CEAD3
:1098900091E10E946C7ACE0101960E94A57A0E9405
:1098A000398660934D0C70934E0C80934F0C9093BF
:1098B000500C8CEA91E10E94F6786093AA027093B2
:1098C000AB028093AC029093AD026093D51370937A
:1098D000D6138093D7139093D8132091D413209349
:1098E000AC0C672B682B692B11F41092AC0C84EF35
:1098F00091E090939D0280939C0265ED72E10E943D
:109900004F0964E670E080E090E00E940C7F65E320
:1099100079E0CE0101960E942C7BCE0101960E9437
:10992000801FCE0101960E94A57A4091AA02509113
:10993000AB026091AC027091AD02CE0101960E9423
:10994000AF78CE0101960E94691FCE0101967CCFAF
:1099500064E576E0CE0101960E943E7BBE016F5F1A
:109960007F4FCE01C4960E948F79182FCE010196A9
:109970000E94A57A1123D9F14AE050E06AEC71E126
:10998000CE0101960E94220ABE016F5F7F4F8CEAD2
:1099900091E10E946C7ACE0101960E94A57A8CEA30
:1099A00091E10E94F678613071058105910519F405
:1099B00081E08093D4138CEA91E10E94F678672BC2
:1099C000682B692B11F41092D4138091D4138093D7
:1099D000AC0C882309F4E1CD0E94398660934D0CCC
:1099E00070934E0C80934F0C9093500CD6CD6FE536
:1099F00076E0CE0101960E943E7BBE016F5F7F4FF5
:109A0000CE01C4960E948F79182FCE0101960E9434
:109A1000A57A1123A1F048E050E06AEC71E1CE0193
:109A200001960E94220ABE016F5F7F4F8CEA91E18E
:109A30000E946C7ACE0101960E94A57ABECD68E69E
:109A400076E0CE0101960E943E7BBE016F5F7F4FA4
:109A5000CE01C4960E948F79182FCE0101960E94E4
:109A6000A57A112321F145E050E06AEC71E1CE01C5
:109A700001960E94220ABE016F5F7F4F8CEA91E13E
:109A80000E946C7ACE0101960E94A57A8CEA91E13F
:109A90000E94F6786130710521F481E08093AD0C6D
:109AA0005ECC672B09F05BCC1092AD0C58CC6EE607
:109AB00076E0CE0101960E943E7BBE016F5F7F4F34
:109AC000CE01C4960E948F79182FCE0101960E9474
:109AD000A57A112309F472C066E070E08AEC91E186
:109AE0000E945E79682FCE0101960E940A7BBE011A
:109AF0006F5F7F4F8CEA91E10E946C7ACE010196F4
:109B00000E94A57A8CEA91E10E94017960E08CEADA
:109B100091E10E94FD798CEA91E10E94F6786B0157
:109B2000CB01181619060CF01ACC2091A80230911E
:109B3000A902261737070CF412CC48E050E06AEC73
:109B400071E1CE0101960E94220ABE016F5F7F4F34
:109B50008CEA91E10E946C7ACE0101960E94A57A6E
:109B60008CEA91E10E9401798091B0119091B1113C
:109B70000997A8F028E030E050E040E06CEA71E19D
:109B8000CE0101960E94537BBE016F5F7F4F8CEA2E
:109B900091E10E946C7ACE0101960E94A57AB601ED
:109BA000E3E0660F771FEA95E1F767517D4E48E0E5
:109BB00050E08CEA91E10E94AA76C1CB65E776E09D
:109BC000CE0101960E943E7BBE016F5F7F4FCE01AA
:109BD000C4960E948F79182FCE0101960E94A57A13
:109BE000112309F4D3C161E876E0CE014C960E94BE
:109BF0003E7B6CE776E0CE0101960E943E7BAE0193
:109C0000445E5F4FBE016F5F7F4FCE01C4960E94DE
:109C1000A6A0CE0101960E94A57ACE014C960E9484
:109C2000A57A61E876E0CE014C960E943E7B6EE715
:109C300076E0CE0101960E943E7BAE01445E5F4F0E
:109C4000BE016F5F7F4FCE01C4960E94A6A0CE01D9
:109C500001960E94A57ACE014C960E94A57A61E8F1
:109C600076E0CE014C960E943E7B60E876E0CE0125
:109C700001960E943E7BAE01445E5F4FBE016F5F66
:109C80007F4FCE01C4960E94A6A0CE0101960E94ED
:109C9000A57ACE014C960E94A57A64E876E0CE01C2
:109CA0004C960E943E7B63E876E0CE0101960E94CE
:109CB0003E7BAE01445E5F4FBE016F5F7F4FCE01C2
:109CC000C4960E94A6A0CE0101960E94A57ACE015C
:109CD0004C960E94A57A64E876E0CE014C960E94EC
:109CE0003E7B6AEA78E0CE0101960E943E7BAE019F
:109CF000445E5F4FBE016F5F7F4FCE01C4960E94EE
:109D0000A6A0CE0101960E94A57ACE014C960E9493
:109D1000A57ACE01C4960E9401790E94398660938B
:109D20003A0C70933B0C80933C0C90933D0C36E0C6
:109D3000E32EF12C44E6442E512C612C712C882406
:109D40008394912C5701F3E0AF0EB11C88AD99AD0F
:109D50000197A816B90608F002CBB701CE01C49648
:109D60000E945E79682FCE014C960E940A7B6701A3
:109D700082E0C80ED11C9FEFE91AF90A9601A701EB
:109D8000BE016C5C7F4FCE0101960E94537BCE01D9
:109D900001960E94F6788B01CE0101960E94A57A69
:109DA0000130110521F40091EF131091F0130330ED
:109DB000110521F40091F1131091F21361E876E09E
:109DC000CE0101960E943E7BA601BE016F5F7F4FD0
:109DD000CE01C4960E949FA16C01CE0101960E9403
:109DE000A57A67E074E0CE0101960E943E7B1C14C8
:109DF0001D0424F59601A501BE016C5C7F4FCE01C8
:109E000082960E94537BBE016E5D7F4FCE0101960C
:109E10000E946C7ACE0182960E94A57A10161106D5
:109E20001CF17601EFEFEE1AFE0ACE0101960E94B8
:109E3000A57ACE014C960E94A57A84CFA501BE01D9
:109E40006C5C7F4FCE0182960E94220ABE016E5D3D
:109E50007F4FCE0101960E946C7ACE0182960E94BD
:109E6000A57A101611060CF78091A8029091A9020C
:109E7000801791070CF445C070E060E0CE014C966D
:109E80000E945E79823509F041C0CE0101960E94A0
:109E9000F678672B682B692B39F4F801EE0FFF1F5A
:109EA000EE55FD4F11821082CE0101960E94F67888
:109EB000613071058105910521F5F801EE0FFF1F55
:109EC000EE55FD4F91828082000F111F000F111F70
:109ED000F801E55AFD4F80819181A281B381181666
:109EE00019061A061B0624F0408251826282738290
:109EF0000E943986015B1D4FF80160837183828364
:109F000093831C141D040CF48CCF8FCF8634F1F492
:109F1000CE0101960E94F678672B682B692B39F4E5
:109F2000F801EE0FFF1FE75BFD4F11821082CE019B
:109F300001960E94F678613071058105910521F640
:109F4000F801EE0FFF1FE75BFD4FBCCF843481F4B7
:109F5000CE0101960E94F678000F111F000F111F0D
:109F6000F801E95CFD4F6083718382839383C0CFE6
:109F7000843539F6CE0101960E94F678000F111F44
:109F8000000F111FF801E55AFD4FEDCF60E379E0B6
:109F9000CE0101960E942C7BBE016F5F7F4FCE01E8
:109FA000C4960E948F79182FCE0101960E94A57A3F
:109FB000112309F414C144E050E06AEC71E1CE01D0
:109FC00001960E94220ABE016F5F7F4F8CEA91E1E9
:109FD0000E946C7ACE0101960E94A57A8CEA91E1EA
:109FE0000E94017960E08CEA91E10E94FD79409144
:109FF000B0115091B1116EEF7BE08CEA91E10E94BB
:10A00000AA7662E475E0CE018E960E943E7B6CEAF1
:10A0100071E1CE0188960E94357B8CA59DA510E04C
:10A02000892BA9F067E074E0CE0182960E943E7B06
:10A030008AA99BA9892B09F05CC0CE0188960E9451
:10A04000F6786AAFCE0182960E94A57A11E0CE0121
:10A0500088960E94A57ACE018E960E94A57A112339
:10A0600009F47DC98E01065C1F4F51E0E52E53E1D6
:10A07000F52E6E018EE3C80ED11CF80181918F017F
:10A08000F70181937F011D8E1C8E1F8E1E8E19A2DB
:10A0900018A24AE0BE016F5F7F4F90E00E9498A433
:10A0A000BE016F5F7F4FCE014C960E947978CE0142
:10A0B0004C960E94691FCE014C960E94A57AC0164C
:10A0C000D106D9F684EF91E090939D0280939C0293
:10A0D00065ED72E10E944F0964E670E080E090E077
:10A0E0000E940C7F65E279E0CE0101960E942C7BF4
:10A0F00028CC50E040E0BE01625D7F4FCE018896E3
:10A100000E949FA18C01892B11F40CA51DA567E06D
:10A1100074E0CE014C960E943E7B4E01FAE38F0E16
:10A12000911C5401F12CE12C6501C818D9081016B6
:10A13000110684F59801A701BE01685D7F4FCE012D
:10A1400001960E94537BBE016F5F7F4FCE014C96FC
:10A150000E946C7ACE0101960E94A57ACE014C969F
:10A160000E94F678F50161935F017801FFEFEF1A25
:10A17000FF0AA701BE01625D7F4FCE0188960E9453
:10A180009FA18C018CA59DA5E816F90668F210E048
:10A1900000E0CACF8CA59DA5E816F906D8F4A70162
:10A1A000BE01685D7F4FCE0101960E94220ABE016A
:10A1B0006F5F7F4FCE014C960E946C7ACE01019664
:10A1C0000E94A57ACE014C960E94F678FE01EC0D15
:10A1D000FD1D62AFCE014C960E94A57A33CF6EE191
:10A1E00079E0CE0101960E942C7BBE016F5F7F4F0C
:10A1F000CE01C4960E948F79182FCE0101960E943D
:10A20000A57A1123E9F146E050E06AEC71E1CE0154
:10A2100001960E94220ABE016F5F7F4F8CEA91E196
:10A220000E946C7ACE0101960E94A57A8CEA91E197
:10A230000E9401798091B0119091B111892B09F49C
:10A240008EC88CEA91E10E94F6787093FE136093B9
:10A25000FD13709336026093350284EF91E0909382
:10A260009D0280939C0265ED72E10E944F0964E6B5
:10A2700070E080E090E00E940C7F6AE079E034CFEB
:10A2800066E876E0CE0101960E943E7BBE016F5FDC
:10A290007F4FCE01C4960E948F79182FCE01019670
:10A2A0000E94A57A1123A1F06DEF78E0CE0101960E
:10A2B0000E942C7B64E670E0CE0101960E94CA8960
:10A2C000CE0101960E94A57AF0E0E0E0199547C81A
:10A2D0006DE876E0CE014C960E943E7BBE01645E46
:10A2E0007F4F8AEC91E10E948F7911E0811115C0B6
:10A2F00065E976E0CE0101960E943E7BBE016F5F6C
:10A300007F4F8AEC91E10E948F7911E0811101C0A9
:10A3100010E0CE0101960E94A57ACE014C960E94D3
:10A32000A57A112389F16DE976E0CE0101960E94AC
:10A330003E7B63E174E1CE0101960E94C079BC01CD
:10A3400082EB91E10E94557ACE0101960E94A57A96
:10A3500060E178E0CE0101960E943E7B62EB71E104
:10A36000CE0101960E94C079BC01CE014C960E949C
:10A37000357BCE014C960E94691FCE014C960E94FF
:10A38000A57ACE0101966BC567EA76E0CE014C96C0
:10A390000E943E7BBE01645E7F4F8AEC91E10E9489
:10A3A0008F7911E0811115C06EEA76E0CE01019639
:10A3B0000E943E7BBE016F5F7F4F8AEC91E10E945D
:10A3C0008F7911E0811101C010E0CE0101960E9449
:10A3D000A57ACE014C960E94A57A112369F06FEE02
:10A3E00078E082EB91E10E94307A69E174E182EBDE
:10A3F00091E10E94297AACCF65EB76E0CE0101961F
:10A400000E943E7BBE016F5F7F4FCE01C4960E94CB
:10A410008F79182FCE0101960E94A57A112331F071
:10A420000E946F2B109234020C94AF496EEB76E0D1
:10A43000CE014C960E943E7BBE01645E7F4F8AEC4B
:10A4400091E10E948F7911E0811115C063EC76E0F3
:10A45000CE0101960E943E7BBE016F5F7F4F8AEC6A
:10A4600091E10E948F7911E0811101C010E0CE01CD
:10A4700001960E94A57ACE014C960E94A57A1123DE
:10A4800009F441C064E876E0CE0101960E943E7B6B
:10A490004091CE115091CF118D819E81481B590B57
:10A4A000BE016F5F7F4F8AEC91E10E9458A0AC0122
:10A4B0004F5F5F4F6AEC71E1CE014C960E94220A19
:10A4C000BE01645E7F4F8CEA91E10E946C7ACE01FE
:10A4D0004C960E94A57ACE0101960E94A57A8CEA3C
:10A4E00091E10E94F6786115710531F481E0809365
:10A4F000DE020E946A9596CF6130710509F092CF15
:10A500001092DE02F6CF68EC76E0CE0101960E9452
:10A510003E7BBE016F5F7F4FCE01C4960E948F7954
:10A52000182FCE0101960E94A57A112309F43AC191
:10A5300043E050E06AEC71E1CE0101960E94220AEC
:10A54000BE016F5F7F4F8CEA91E10E946C7ACE0171
:10A5500001960E94A57A6CEA71E1CE0101960E94F3
:10A56000357BCE0101960E94F124CE0101960E9416
:10A57000A57A84EF91E090939D0280939C026CEA0F
:10A5800071E1CE0101960E94357B60E0CE0101961B
:10A590000E94117ABC018FE194E10E94557ACE01AC
:10A5A00001960E94A57A6CEA71E1CE0101960E94A3
:10A5B000357B60E0CE0101960E94117ABC0189E1F1
:10A5C00094E10E94557ACE0101960E94A57A4091AD
:10A5D00023145091241465E973E18FE194E10E9402
:10A5E000AA7640911D1450911E1460EA73E189E12E
:10A5F00094E10E94AA7665ED72E180919C029091AF
:10A600009D020E944F096CEC76E0CE0101960E94FB
:10A610003E7B6CEA71E1CE0101960E94C079BC01DB
:10A62000CE0182960E94357BCE0101960E94A57ACA
:10A630008091911390919213892B39F4BE016E5D34
:10A640007F4F84EE9EE00E94877C68EB7BE080E099
:10A6500090E00E940C7F8091911390919213029749
:10A6600009F087C06CEA71E1CE0188960E94357BC3
:10A6700064ED76E0CE0101960E943E7BCE0101960C
:10A680000E949695CE0101960E94A57A64EF71E032
:10A6900080E090E00E940C7F67ED76E0CE010196AD
:10A6A0000E943E7BCE0101960E949695CE010196B6
:10A6B0000E94A57A6CED75E080E090E00E940C7F2E
:10A6C00060EE76E0CE0101960E943E7BCE010196BF
:10A6D0000E949695CE0101960E94A57A64EF71E0E2
:10A6E00080E090E00E940C7F6EEE76E0CE01019655
:10A6F0000E943E7BCE0101960E949695CE01019666
:10A700000E94A57A64EF71E080E090E00E940C7FE7
:10A710006CEC76E0CE0101960E943E7BBE01685D46
:10A720007F4FCE0101960E94C079BC01CE014C96AC
:10A730000E94357BCE0101960E94A57ACE014C96EF
:10A740000E940179BE01645E7F4FCE0101960E9496
:10A75000357BCE0101960E949695CE0101960E940E
:10A76000A57ACE014C960E94A57ACE0188960E94C9
:10A77000A57A68EB7BE080E090E00E940C7F65E9C1
:10A7800073E1CE0101960E943E7BCE0101960E94AC
:10A79000F124CE0101960E94A57A10923402CE01D6
:10A7A000829652C86CEF76E0CE0101960E943E7B05
:10A7B000BE016F5F7F4FCE01C4960E948F79182F24
:10A7C000CE0101960E94A57A112309F486C044E0C7
:10A7D00050E06AEC71E1CE0101960E94220ABE01AE
:10A7E0006F5F7F4F8CEA91E10E946C7ACE010196F7
:10A7F0000E94A57A61E077E0CE0101960E943E7B3F
:10A800006CEA71E1CE0101960E94C079BC01CE01D3
:10A810004C960E94357BCE0101960E94A57A8091CC
:10A82000911390919213892B39F4BE01645E7F4F8E
:10A8300084EE9EE00E94877C68E873E180E090E00F
:10A840000E940C7F8091911390919213029759F579
:10A8500068E077E0CE0101960E943E7B8091B011C6
:10A860009091B111892B19F561E177E0CE01019644
:10A870000E947978BE01645E7F4FCE0182960E946D
:10A88000357BCE0182960E949695CE0182960E94DB
:10A89000A57A68E873E180E090E00E940C7FCE0129
:10A8A00001960E94A57A109234020C94224CBE01AB
:10A8B0006F5F7F4FCE0182960E94357BCE018296DC
:10A8C0000E949695CE0182960E94A57A60E777E174
:10A8D00080E090E00E940C7FCDCF6AE177E0CE016E
:10A8E00001960E943E7BBE016F5F7F4FCE01C496F2
:10A8F0000E948F79182FCE0101960E94A57A11230C
:10A9000009F462C06AEC71E18CEA91E10E94557A27
:10A9100081E0809334026AEC71E1CE0101960E94DD
:10A92000357BCE0101960E94F124CE0101960E9452
:10A93000A57A8091911390919213029709F16CEA94
:10A9400071E184EE9EE00E94877C68EB7BE080E012
:10A9500090E00E940C7FCE0101960E942F96BE01CE
:10A960006F5F7F4F8AEC91E10E946C7ACE01019675
:10A970000E94A57A60ED77E080E090E00E940C7F75
:10A980008091911390919213029771F46CEA71E1A6
:10A99000CE0101960E94357BCE0101960E949695CC
:10A9A000CE0101960E94A57A8091CE119091CF118F
:10A9B000892B09F437CD60E178E0CE0101960E9441
:10A9C0003E7B6AEC71E1CCCC6EE177E0CE01019682
:10A9D0000E943E7BBE016F5F7F4FCE01C4960E94F6
:10A9E0008F79182FCE0101960E94A57A112309F4C0
:10A9F00092C18091911390919213019709F012CD19
:10AA000064E277E0CE0188960E943E7BBE01685DDD
:10AA10007F4F84EE9EE00E94877C6CE271E080E0D4
:10AA200090E00E940C7FCE0182960E942F9664E6F1
:10AA300070E080E090E00E940C7F10E000E035E0E4
:10AA4000C32ED12C4AE0A42EB12C6FE277E0CE01C8
:10AA500001960E943E7B50E040E0BE016F5F7F4F59
:10AA6000CE0182960E949FA17C01CE0101960E9498
:10AA7000A57AA7014F5F5F4FBE016E5D7F4FCE018C
:10AA800001960E94220ABE016F5F7F4FCE01889619
:10AA90000E946C7ACE0101960E94A57A8CA59DA594
:10AAA000892B09F170E060E0CE0188960E945E7902
:10AAB000082E000C990BC0970A97A8F461E377E081
:10AAC000CE0101960E943E7BBE016F5F7F4FCE019B
:10AAD00088960E948F79E82ECE0101960E94A57A71
:10AAE000FF24F394E110F12C60E078E0CE010196B0
:10AAF0000E942C7B64E170E0CE0101960E94BBA114
:10AB0000CE0101960E94A57A0F5F1F4F62E370E0AD
:10AB100080E090E00E940C7FC801B6010E9464AB07
:10AB20000197C1F4CE0101960E941D258D819E8161
:10AB3000892B09F4BBC0BE016F5F7F4F8AEC91E1A6
:10AB40000E94557A0E949848FF24F394CE01019602
:10AB50000E94A57ACE0101960E942F96BE016F5FDA
:10AB60007F4FCE0182960E946C7ACE0101960E94A0
:10AB7000A57A62E370E080E090E00E940C7F0436EA
:10AB8000110519F0FF2009F460CF8091EB0B8823A9
:10AB9000F1F060E178E0CE014C960E943E7BBE0170
:10ABA000685D7F4FCE014C960E94C079BC01CE01FA
:10ABB00001960E94357BCE0101960E94691FCE014D
:10ABC00001960E94A57ACE014C960E94A57A8CA58A
:10ABD0009DA5892B69F070E060E0CE0188960E9407
:10ABE0005E79082E000C990BC0970A9708F477C07D
:10ABF00069E377E0CE0101960E943E7BCE0182960A
:10AC00000E94A57ACE0188960E94A57A8D819E81A8
:10AC1000009709F446C0E981FA812081222309F4D2
:10AC200040C00797F0F166EE78E0CE014C960E94A6
:10AC30002C7B68EC70E0CE014C960E94BBA1CE014B
:10AC40004C960E94A57ABE016F5F7F4FCE014C9655
:10AC50000E94357B60ED77E0CE014C960E94CA8958
:10AC6000CE014C960E94A57A65E477E0CE014C9621
:10AC70000E943E7B6AEC71E1CE014C960E94C07945
:10AC8000BC01CE0182960E94357BCE0182960E9445
:10AC9000691FCE0182960E94A57ACE014C960E9431
:10ACA000A57ACE0101960E94A57ABCCB043111058C
:10ACB0000CF44CCFC801B5010E9464AB892B09F09C
:10ACC00045CFBE01685D7F4F84EE9EE00E94877C89
:10ACD00068EC70E080E090E00E940C7F37CF61E389
:10ACE00077E0CE0101960E943E7BBE016F5F7F4FF1
:10ACF000CE0188960E948F79182FCE0101960E946E
:10AD0000A57A111175CFBE01685D7F4FCE01019606
:10AD10000E94237B73CF63E577E0CE0101960E940A
:10AD20003E7BBE016F5F7F4FCE01C4960E948F793C
:10AD3000182FCE0101960E94A57A112309F4E8C0CC
:10AD400025E030E044E050E06AEC71E1CE0101968C
:10AD50000E94537BBE016F5F7F4F8CEA91E10E949E
:10AD60006C7ACE0101960E94A57A6AEC71E1CE015F
:10AD700001960E94357BCE0101960E94F124CE01FE
:10AD800001960E94A57A8CEA91E10E94F6786130E2
:10AD9000710509F067C070939213609391136FE28D
:10ADA00078E0CE0101960E942C7BCE0101960E9494
:10ADB000F124CE0101960E94A57A68E577E0CE01E4
:10ADC0004C960E943E7B69E174E1CE014C960E9454
:10ADD000C079BC01CE0101960E94357B48EC50E061
:10ADE0006FEF7FEFCE0101960E949020CE01019679
:10ADF0000E94A57ACE014C960E94A57A0E943BA0A3
:10AE000040E052EC61E070E084EE9EE00E94AA75A2
:10AE100084EF91E090939D0280939C0265ED72E136
:10AE20000E944F0967E677E0CE014C960E943E7B78
:10AE300063E174E1CE014C960E94C079BC01CE0161
:10AE400001960E94357B60ED77E0CE0101960E946D
:10AE5000CA89CE0101960E94A57ACE014C960E9425
:10AE6000A57AE0CA61157105D1F51092921310927E
:10AE7000911361E278E0CE0101960E942C7BCE0115
:10AE800001960E94F124CE0101960E94A57A6EE5FA
:10AE900077E0CE014C960E943E7B69E174E1CE01E1
:10AEA0004C960E94C079BC01CE0101960E94357B70
:10AEB00048EC50E06FEF7FEFCE0101960E949020AA
:10AEC000CE0101960E94A57ACE014C960E94A57AE9
:10AED0000E943BA040E855E260E070E095CF623010
:10AEE000710509F09FCA709392136093911360E10A
:10AEF00078E0CE0101960E942C7BCE0101960E9443
:10AF0000F124CE0101960E94A57A62E677E0C1CFD6
:10AF10006CE677E0CE0101960E943E7BBE016F5F3A
:10AF20007F4FCE01C4960E948F79182FCE010196D3
:10AF30000E94A57A112309F441C047E050E06AEC71
:10AF400071E1CE0101960E94220ABE016F5F7F4F20
:10AF50008CEA91E10E946C7ACE0101960E94A57A5A
:10AF600067E377E0CE0101960E943E7BBE016F5FF2
:10AF70007F4F8CEA91E10E948F79182FCE010196C4
:10AF80000E94A57A11111092AB0C68EA74E0CE0110
:10AF900001960E943E7BBE016F5F7F4F8CEA91E17C
:10AFA0000E948F79182FCE0101960E94A57A112355
:10AFB00009F401CD81E08093AB0CFDCC64E777E030
:10AFC000CE0101960E943E7BBE016F5F7F4FCE0196
:10AFD000C4960E948F79182FCE0101960E94A57AFF
:10AFE000112381F146E050E06AEC71E1CE01019657
:10AFF0000E94220ABE016F5F7F4F8CEA91E10E949E
:10B000006C7ACE0101960E94A57A8CEA91E10E94A9
:10B01000EB786093D9137093DA138093DB139093DA
:10B02000DC1384EF91E090939D0280939C0265ED88
:10B0300072E10E944F0964E670E080E090E00E94B7
:10B040000C7FB9CC6BE777E0CE0101960E943E7B86
:10B05000BE016F5F7F4FCE01C4960E948F79182F7B
:10B06000CE0101960E94A57A112301F148E050E03B
:10B070006AEC71E1CE0101960E94220ABE016F5F67
:10B080007F4F8CEA91E10E946C7ACE0101960E947A
:10B09000A57A8CEA91E10E94EB786093DF137093BC
:10B0A000E0138093E1139093E213BBCF64E877E061
:10B0B000CE0101960E943E7BBE016F5F7F4FCE01A5
:10B0C000C4960E948F79182FCE0101960E94A57A0E
:10B0D000112301F149E050E06AEC71E1CE010196E3
:10B0E0000E94220ABE016F5F7F4F8CEA91E10E94AD
:10B0F0006C7ACE0101960E94A57A8CEA91E10E94B9
:10B10000EB786093E3137093E4138093E5139093CB
:10B11000E61387CF6EE877E0CE0101960E943E7B72
:10B12000BE016F5F7F4FCE01C4960E948F79182FAA
:10B13000CE0101960E94A57A1123F1F049E050E07A
:10B140006AEC71E1CE0101960E94220ABE016F5F96
:10B150007F4F8CEA91E10E946C7ACE0101960E94A9
:10B16000A57A8CEA91E10E94EB780E9418AB70936B
:10B17000EA136093E91355CF68E977E0CE010196B1
:10B180000E943E7BBE016F5F7F4FCE01C4960E943E
:10B190008F79182FCE0101960E94A57A1123F1F024
:10B1A0004AE050E06AEC71E1CE0101960E94220A69
:10B1B000BE016F5F7F4F8CEA91E10E946C7ACE01F5
:10B1C00001960E94A57A8CEA91E10E94EB780E9498
:10B1D00018AB7093E8136093E71323CF63EA77E02B
:10B1E000CE0101960E943E7BBE016F5F7F4FCE0174
:10B1F000C4960E948F79182FCE0101960E94A57ADD
:10B20000112311F14BE050E06AEC71E1CE0101969F
:10B210000E94220ABE016F5F7F4F8CEA91E10E947B
:10B220006C7ACE0101960E94A57A8CEA91E10E9487
:10B23000EB780E9418AB6093EB137093EC13809340
:10B24000ED139093EE13EDCE6FEA77E0CE01019609
:10B250000E943E7BBE016F5F7F4FCE01C4960E946D
:10B260008F79182FCE0101960E94A57A112389F1BA
:10B2700043E050E0BE016C5C7F4FCE0101960E941E
:10B28000220ABE016F5F7F4F8CEA91E10E946C7AC7
:10B29000CE0101960E94A57A8091B0119091B111D2
:10B2A000892B41F08CEA91E10E94F67870936A0252
:10B2B000609369028091690290916A0201970297F6
:10B2C00008F479CB81E090E090936A028093690260
:10B2D00072CB6CE977E0CE014C960E943E7BBE01BA
:10B2E000645E7F4FCE01C4960E948F7911E0811178
:10B2F00015C065EE77E0CE0101960E943E7BBE014F
:10B300006F5F7F4FCE01C4960E948F7911E081114B
:10B3100001C010E0CE0101960E94A57ACE014C96A4
:10B320000E94A57A112309F468C06CE977E0CE0188
:10B3300001960E943E7BBE016F5F7F4FCE01C49697
:10B340000E948F79182FCE0101960E94A57A1123B1
:10B35000A1F046E050E0BE016C5C7F4FCE0101964B
:10B360000E94220ABE016F5F7F4F8CEA91E10E942A
:10B370006C7ACE0101960E94A57A65EE77E0CE0147
:10B3800001960E943E7BBE016F5F7F4FCE01C49647
:10B390000E948F79182FCE0101960E94A57A112361
:10B3A000A1F042E050E0BE016C5C7F4FCE010196FF
:10B3B0000E94220ABE016F5F7F4F8CEA91E10E94DA
:10B3C0006C7ACE0101960E94A57A8091B01190917D
:10B3D000B111892B09F4EFCA6CEA71E1CE01019633
:10B3E0000E94357B61E070E0CE0101960E94A53598
:10B3F000CE0101960E94A57ADECA6CEB77E0CE0101
:10B4000082960E943E7BBE016E5D7F4FCE01C49648
:10B410000E948F7911E0811129C063EB77E0CE01A2
:10B420004C960E943E7BBE01645E7F4FCE01C49667
:10B430000E948F7911E0811115C06BEB77E0CE018E
:10B4400001960E943E7BBE016F5F7F4FCE01C49686
:10B450000E948F7911E0811101C010E0CE010196A8
:10B460000E94A57ACE014C960E94A57ACE018296C2
:10B470000E94A57A112309F4E6C06CEB77E0CE01B7
:10B4800001960E943E7BBE016F5F7F4FCE01C49646
:10B490000E948F79182FCE0101960E94A57A112360
:10B4A00009F466C046E050E0BE016C5C7F4FCE01FF
:10B4B00001960E94220ABE016F5F7F4F8CEA91E1E4
:10B4C0000E946C7ACE0101960E94A57A8CEA91E1E5
:10B4D0000E94EB786B017C0120E030E0A9010E9422
:10B4E0004EAB18160CF08EC0A701960160E070E01C
:10B4F0008AE794E40E94A6AA0E9418AB60933002E7
:10B500007093310280933202909333028091300223
:10B5100090913102A0913202B091330218161906AF
:10B520001A061B0664F081E090E0A0E0B0E0809392
:10B53000300290933102A0933202B0933302809193
:10B54000690290916A028130910509F068C080918A
:10B55000300290913102A0913202B0913302809377
:10B560002C0290932D02A0932E02B0932F0223CA97
:10B5700047E050E0BE016C5C7F4FCE0101960E9417
:10B58000220ABE016F5F7F4F8CEA91E10E946C7AC4
:10B59000CE0101960E94A57A68E474E0CE0101967E
:10B5A0000E943E7BBE016F5F7F4FCE01C4960E941A
:10B5B0008F79182FCE0101960E94A57A112331F0C0
:10B5C00081E090E090936A028093690265ED76E0F5
:10B5D000CE0101960E943E7BBE016F5F7F4FCE0180
:10B5E000C4960E948F79182FCE0101960E94A57AE9
:10B5F000112309F46BCF82E090E090936A0280936C
:10B60000690264CF81E090E0A0E0B0E08093300276
:10B6100090933102A0933202B093330277CF029716
:10B6200009F0C9C98091300290913102A091320293
:10B63000B09133028093280290932902A0932A02AA
:10B64000B0932B02B8C963EC77E0CE0101960E945B
:10B650003E7BBE016F5F7F4FCE01C4960E946F7923
:10B66000082FCE0101960E94A57A002309F40EC18D
:10B6700063EC77E0CE0101960E943E7BBE016F5FD6
:10B680007F4FCE01C4960E948F79182FCE0101966C
:10B690000E94A57A111134C068E474E0CE010196CD
:10B6A0000E943E7BBE016F5F7F4FCE01C4960E9419
:10B6B0008F79182FCE0101960E94A57A112331F0BF
:10B6C00081E090E090936A028093690265ED76E0F4
:10B6D000CE0101960E943E7BBE016F5F7F4FCE017F
:10B6E000C4960E948F79182FCE0101960E94A57AE8
:10B6F000112331F082E090E090936A028093690216
:10B7000081E090E0A0E0B0E08093300290933102BD
:10B71000A0933202B09333028091690290916A0241
:10B720008130910509F046C09093680280936702CA
:10B7300064EE75E08CEA91E10E94797880913002A4
:10B7400090913102A0913202B091330280932C0289
:10B7500090932D02A0932E02B0932F0265ED78E016
:10B76000CE0101960E942C7BCE0101960E94691F9A
:10B77000CE0101960E94A57A6CEA71E1CE01019694
:10B780000E94357B62E070E0CE0101960E94A535F3
:10B79000CE0101960E94A57A65EC78E0CE01019673
:10B7A0000E942C7BCE0101960E943027CE0101968B
:10B7B0000E94A57A0091690210916A020230110577
:10B7C00009F0F9C867E377E08CEA91E10E947978A3
:10B7D00064EB78E0CE0101960E942C7BCE010196AD
:10B7E0000E94691FCE0101960E94A57A6CEA71E160
:10B7F000CE0101960E94357B63E070E0CE01019698
:10B800000E94A535CE0101960E94A57A10936A0286
:10B81000009369028091FB139091FC13909368024E
:10B820008093670268EA78E0CE0101960E942C7B43
:10B83000CE0101960E943027CE0101960E94A57A82
:10B840008091FB139091FC139195819591099093B0
:10B85000FC138093FB1301E010E010936802009347
:10B86000670284EF91E090939D0280939C0265EDC6
:10B8700072E10E944F0964E670E080E090E00E946F
:10B880000C7F10936A020093690295C868EC77E018
:10B89000CE0188960E943E7BBE01685D7F4FCE013F
:10B8A000C4960E948F7901E081113DC065E178E086
:10B8B000CE0182960E943E7BBE016E5D7F4FCE011F
:10B8C000C4960E948F7901E0811129C064E178E07B
:10B8D000CE014C960E943E7BBE01645E7F4FCE013E
:10B8E000C4960E948F7901E0811115C06FEC77E05A
:10B8F000CE0101960E943E7BBE016F5F7F4FCE015D
:10B90000C4960E948F7901E0811101C000E0CE0150
:10B9100001960E94A57ACE014C960E94A57ACE018E
:10B9200082960E94A57ACE0188960E94A57A00236D
:10B9300009F464C168EC77E0CE0101960E943E7B79
:10B94000BE016F5F7F4FCE01C4960E948F79082F92
:10B95000CE0101960E94A57A46E050E0011117C081
:10B9600065E178E0CE0101960E943E7BBE016F5FEB
:10B970007F4FCE01C4960E948F79082FCE01019689
:10B980000E94A57A002309F467C042E050E0BE019E
:10B990006C5C7F4FCE0101960E94220ABE016F5F50
:10B9A0007F4F8CEA91E10E946C7ACE0101960E9451
:10B9B000A57A8091B0119091B111892B11F40C945A
:10B9C000DB5466E179E0CE014C960E943E7BBE01DD
:10B9D000645E7F4F8CEA91E10E948F79811114C0DF
:10B9E00068ED75E0CE0101960E943E7BBE016F5F5F
:10B9F0007F4F8CEA91E10E948F7911E0811110E074
:10BA0000CE0101960E94A57ACE014C960E94A57A9D
:10BA1000112309F4E2C08CEA91E10E94EB782091B5
:10BA2000FA0B3091FB0B4091FC0B5091FD0B0E94E7
:10BA30003AAA6B017C0120E030E044EB53E40E9421
:10BA40004EAB87FD53C020E030E044EB53E4C70128
:10BA5000B6010E9439AAEDCF43E050E0BE016C5C14
:10BA60007F4FCE0101960E94220ABE016F5F7F4F79
:10BA70008CEA91E10E946C7ACE0101960E94A57A2F
:10BA800068E474E0CE0101960E943E7BBE016F5FC8
:10BA90007F4FCE01C4960E948F79082FCE01019668
:10BAA0000E94A57A002331F081E090E090936A0231
:10BAB0008093690265ED76E0CE0101960E943E7B9F
:10BAC000BE016F5F7F4FCE01C4960E948F79082F11
:10BAD000CE0101960E94A57A002309F46ACF82E084
:10BAE00090E090936A028093690263CF20E030E097
:10BAF000A901C701B6010E948CA887FF0BC020E0F6
:10BB000030E044EB53E4C701B6010E943AAA6B014E
:10BB10007C01ECCFC092FA0BD092FB0BE092FC0BB5
:10BB2000F092FD0B8CEA91E10E94EB7820E030E08E
:10BB3000A9010E944EAB87FD15C068ED75E0CE01EE
:10BB400001960E943E7B6CEA71E1CE0101960E9453
:10BB5000C079BC018CEA91E10E94557ACE01019630
:10BB60000E94A57A8CEA91E10E94EB7820E030E017
:10BB7000A9010E948CA887FF30C08CEA91E10E9445
:10BB8000EB7820E030E0A9010E944EAB181674F566
:10BB90008CEA91E10E94EB78AB01BC0122E0CE017E
:10BBA0004C960E94AD7A66E179E0CE0101960E9442
:10BBB0003E7BBE01645E7F4FCE0101960E94C0793C
:10BBC000BC018CEA91E10E94557ACE0101960E9457
:10BBD000A57ACE014C960E94A57A6CEA71E1CE015D
:10BBE00001960E94357B62E070E0FECB8CEA91E129
:10BBF0000E94EB78AB01BC017058D0CF64ED77E0C8
:10BC0000CE0182960E943E7BBE016E5D7F4FCE01CB
:10BC1000C4960E948F7911E0811129C063ED77E00D
:10BC2000CE014C960E943E7BBE01645E7F4FCE01EA
:10BC3000C4960E948F7911E0811115C06AED77E0FA
:10BC4000CE0101960E943E7BBE016F5F7F4FCE0109
:10BC5000C4960E948F7911E0811101C010E0CE01DD
:10BC600001960E94A57ACE014C960E94A57ACE013B
:10BC700082960E94A57A112309F487C0CE01C4964A
:10BC80000E94017964ED77E0CE0101960E943E7B2F
:10BC9000BE016F5F7F4FCE01C4960E948F79182F2F
:10BCA000CE0101960E94A57A112329F145E050E0CA
:10BCB000BE016C5C7F4FCE0101960E94220ABE013C
:10BCC0006F5F7F4F8CEA91E10E946C7ACE01019602
:10BCD0000E94A57A8091B0119091B111892B11F435
:10BCE0000C94DB546CEA71E1CE0101960E94357B25
:10BCF00063E070E079CB46E050E0BE016C5C7F4FC2
:10BD0000CE0101960E94220ABE016F5F7F4F8CEA2E
:10BD100091E10E946C7ACE0101960E94A57A68E4B6
:10BD200074E0CE0101960E943E7BBE016F5F7F4FA3
:10BD3000CE01C4960E948F79182FCE0101960E94E1
:10BD4000A57A112331F081E090E090936A0280930C
:10BD5000690265ED76E0CE0101960E943E7BBE0150
:10BD60006F5F7F4FCE01C4960E948F79182FCE014E
:10BD700001960E94A57A112309F4ACCF82E090E0ED
:10BD800090936A0280936902A5CF62EE77E0CE01BC
:10BD900082960E943E7BBE016E5D7F4FCE01C496AF
:10BDA0000E948F7911E0811129C061EE77E0CE0108
:10BDB0004C960E943E7BBE01645E7F4FCE01C496CE
:10BDC0000E948F7911E0811115C068EE77E0CE01F5
:10BDD00001960E943E7BBE016F5F7F4FCE01C496ED
:10BDE0000E948F7911E0811101C010E0CE0101960F
:10BDF0000E94A57ACE014C960E94A57ACE01829629
:10BE00000E94A57A112309F425C162EE77E0CE01E4
:10BE100001960E943E7BBE016F5F7F4FCE01C496AC
:10BE20000E948F79182FCE0101960E94A57A1123C6
:10BE300009F443C045E050E0BE016C5C7F4FCE0189
:10BE400001960E94220ABE016F5F7F4F8CEA91E14A
:10BE50000E946C7ACE0101960E94A57A8091B01161
:10BE60009091B111892B61F08CEA91E10E94EB78FD
:10BE70006093FA0B7093FB0B8093FC0B9093FD0B7C
:10BE8000C090FA0BD090FB0BE090FC0BF090FD0BF8
:10BE900020E030E044EB53E4C701B6010E944EAB12
:10BEA00087FD55C020E030E044EB53E4C701B60104
:10BEB0000E9439AA6B017C01EBCF46E050E0BE0145
:10BEC0006C5C7F4FCE0101960E94220ABE016F5F1B
:10BED0007F4F8CEA91E10E946C7ACE0101960E941C
:10BEE000A57A68E474E0CE0101960E943E7BBE0113
:10BEF0006F5F7F4FCE01C4960E948F79182FCE01BD
:10BF000001960E94A57A112331F081E090E0909390
:10BF10006A028093690265ED76E0CE0101960E9487
:10BF20003E7BBE016F5F7F4FCE01C4960E948F792A
:10BF3000182FCE0101960E94A57A112309F48ECF05
:10BF400082E090E090936A028093690287CF20E0BC
:10BF500030E0A901C701B6010E948CA887FF0BC081
:10BF600020E030E044EB53E4C701B6010E943AAA56
:10BF70006B017C01ECCFC092FA0BD092FB0BE092EC
:10BF8000FC0BF092FD0B8091690290916A0201977F
:10BF900071F4C092450CD092460CE092470CF0929E
:10BFA000480C6CED74E082EB91E10E94797880910D
:10BFB000FA0B9091FB0BA091FC0BB091FD0B209123
:10BFC000690230916A022230310571F48093410C8C
:10BFD0009093420CA093430CB093440C6BEE74E02E
:10BFE00082EB91E10E9479784091FA0B5091FB0B22
:10BFF0006091FC0B7091FD0B21E0CE014C960E94EC
:10C00000AD7A62EB71E1CE0101960E94357BBE01F3
:10C01000645E7F4FCE0101960E94C07966EE74E0A7
:10C020000E94AA79BC0182EB91E10E94557ACE016F
:10C0300001960E94A57ACE014C960E94A57A62EBE9
:10C0400071E1CE0101960E94357BCE0101960E94DE
:10C050003027CEC960EF77E0CE0182960E943E7B0A
:10C06000BE016E5D7F4FCE01C4960E948F7911E0B4
:10C07000811129C06FEE77E0CE014C960E943E7B85
:10C08000BE01645E7F4FCE01C4960E948F7911E09D
:10C09000811115C065EF77E0CE0101960E943E7BCD
:10C0A000BE016F5F7F4FCE01C4960E948F7911E071
:10C0B000811101C010E0CE0101960E94A57ACE0147
:10C0C0004C960E94A57ACE0182960E94A57A1123F1
:10C0D00009F412C2C0903002D0903102E0903202D6
:10C0E000F09033026BEF77E0CE0101960E943E7B29
:10C0F000BE016F5F7F4FCE01C4960E948F79182FCB
:10C10000CE0101960E94A57A112309F465C044E08E
:10C1100050E0BE016C5C7F4FCE0101960E94220A66
:10C12000BE016F5F7F4F8CEA91E10E946C7ACE0175
:10C1300001960E94A57A8091690290916A028130ED
:10C14000910509F093C0C0902C02D0902D02E09090
:10C150002E02F0902F0281E090E0A0E0B0E080930A
:10C160002C0290932D02A0932E02B0932F02809167
:10C17000B0119091B111892B09F090C060E078E086
:10C180008CEA91E10E9479788091B0119091B1117F
:10C19000892B81F06CEA71E1CE0101960E94357B1A
:10C1A00070E060E0CE0101960E94A535CE010196B7
:10C1B0000E94A57A8091690290916A02813091056E
:10C1C00009F08CC1C0922C02D0922D02E0922E0276
:10C1D000F0922F020C94DB5445E050E0BE016C5C01
:10C1E0007F4FCE0101960E94220ABE016F5F7F4FF2
:10C1F0008CEA91E10E946C7ACE0101960E94A57AA8
:10C2000068E474E0CE0101960E943E7BBE016F5F40
:10C210007F4FCE01C4960E948F79182FCE010196D0
:10C220000E94A57A112331F081E090E090936A0298
:10C230008093690265ED76E0CE0101960E943E7B17
:10C24000BE016F5F7F4FCE01C4960E948F79182F79
:10C25000CE0101960E94A57A112309F46CCF82E0E9
:10C2600090E090936A028093690265CF029709F08B
:10C270007ECFC0902802D0902902E0902A02F09050
:10C280002B0281E090E0A0E0B0E080932802909340
:10C290002902A0932A02B0932B0269CF66E078E0CE
:10C2A000CE0101960E943E7BBE016F5F7F4F8CEAFC
:10C2B00091E10E946F79182FCE0101960E94A57A14
:10C2C000112309F477CF8CEA91E10E94EB7820E00A
:10C2D00030E0A9010E948CA8811128C080916902D8
:10C2E00090916A02019731F469E078E08CEA91E17B
:10C2F0000E9479788091690290916A02029731F4E4
:10C3000060E078E08CEA91E10E9479788091B01148
:10C310009091B111892B09F44DCF6CEA71E1CE01F6
:10C3200001960E94357B61E070E03CCF64E876E0E6
:10C33000CE0101960E943E7BBE016F5F7F4F8CEA6B
:10C3400091E10E946F79182FCE0101960E94A57A83
:10C35000112309F42FCF41E050E06CEA71E1CE01E6
:10C3600001960E94220ACE0101960E94EB784B01B1
:10C370005C01CE0101960E94A57A20E030E0A9017F
:10C38000C501B4010E948CA8181634F0812C912CA0
:10C3900020E8A22E2FE3B22E0091690210916A02CA
:10C3A0000130110509F075C0A501940160E070E449
:10C3B0008CE995E40E94A6AA60932402709325025A
:10C3C00080932602909327026093F3137093F413E3
:10C3D0008093F5139093F6136093200270932102DB
:10C3E0008093220290932302B801CE014C960E94C2
:10C3F00083786EE078E0CE0101960E943E7BBE011C
:10C40000645E7F4FCE0101960E94C079BC01CE01CF
:10C4100082960E94357BCE0182960E94801FCE01BB
:10C4200082960E94A57ACE0101960E94A57ACE013D
:10C430004C960E94A57A66E978E0CE0101960E94AA
:10C440002C7BCE0101960E94801FCE0101960E9496
:10C45000A57A4091240250912502609126027091A4
:10C46000270225E0CE0101960E94AD7ACE01019609
:10C470000E94691FCE0101960E94A57A84EF91E087
:10C4800090939D0280939C0265ED72E10E944F099A
:10C4900091CE0230110509F0A7CFA501940160E00B
:10C4A00070E48CE196E40E94A6AA60932402709343
:10C4B000250280932602909327026093F7137093CE
:10C4C000F8138093F9139093FA1360931C027093FE
:10C4D0001D0280931E0290931F0286CF029711F0D7
:10C4E0000C94DB54C0922802D0922902E0922A02D6
:10C4F000F0922B020C94DB5463E178E0CE0182963B
:10C500000E943E7BBE016E5D7F4FCE01C4960E94AD
:10C510008F7911E0811129C062E178E0CE014C965B
:10C520000E943E7BBE01645E7F4FCE01C4960E9496
:10C530008F7911E0811115C068E178E0CE01019694
:10C540000E943E7BBE016F5F7F4FCE01C4960E946A
:10C550008F7911E0811101C010E0CE0101960E9497
:10C56000A57ACE014C960E94A57ACE0182960E94B1
:10C57000A57A112309F429C188AD99AD059710F466
:10C580000C94DB5444E050E0BE016C5C7F4FCE0164
:10C5900001960E94220ABE016F5F7F4F8CEA91E1F3
:10C5A0000E946C7ACE0101960E94A57A63E178E040
:10C5B000CE0101960E943E7BBE016F5F7F4FCE0190
:10C5C000C4960E948F79182FCE0101960E94A57AF9
:10C5D000112309F49BC044E050E0BE016C5C7F4F26
:10C5E000CE0101960E94220ABE016F5F7F4F8CEA46
:10C5F00091E10E946C7ACE0101960E94A57A8CEAA4
:10C6000091E10E94EB7820E030E0A9010E944EAB5E
:10C61000181614F00C94DB548CEA91E10E94EB782C
:10C620006093240270932502809326029093270240
:10C630002091690230916A022130310509F0B0C0C1
:10C640006093F3137093F4138093F5139093F613A0
:10C650006093200270932102809322029093230220
:10C66000B901CE014C960E9483786EE078E0CE014D
:10C6700001960E943E7BBE01645E7F4FCE01019613
:10C680000E94C079BC01CE0182960E94357BCE010A
:10C6900082960E94801FCE0182960E94A57ACE01CA
:10C6A00001960E94A57ACE014C960E94A57A64E874
:10C6B00078E0CE0101960E942C7BCE0101960E946B
:10C6C000801FCE0101960E94A57A409124025091CC
:10C6D0002502609126027091270225E0CE01019685
:10C6E0000E94AD7ACE0101960E94691FCE0101968B
:10C6F0000E94A57A84EF91E090939D0280939C0222
:10C7000065ED72E10E944F090C94DB5445E050E066
:10C71000BE016C5C7F4FCE0101960E94220ABE01D1
:10C720006F5F7F4F8CEA91E10E946C7ACE01019697
:10C730000E94A57A68E474E0CE0101960E943E7BD7
:10C74000BE016F5F7F4FCE01C4960E948F79182F74
:10C75000CE0101960E94A57A112331F081E090E08C
:10C7600090936A028093690265ED76E0CE010196AE
:10C770000E943E7BBE016F5F7F4FCE01C4960E9438
:10C780008F79182FCE0101960E94A57A112309F402
:10C7900036CF82E090E090936A02809369022FCFB7
:10C7A0002230310509F05CCF6093F7137093F813D2
:10C7B0008093F9139093FA1360931C0270931D02F7
:10C7C00080931E0290931F024BCF6EE178E0CE0162
:10C7D00001960E943E7BBE016F5F7F4FCE01C496E3
:10C7E0000E948F79182FCE0101960E94A57A11110F
:10C7F0000C949D5766E278E0CE0101960E943E7B44
:10C80000BE016F5F7F4FCE01C4960E948F79182FB3
:10C81000CE0101960E94A57A112371F141E066EBE9
:10C8200072E0CE0101960E94BE92BE016F5F7F4F03
:10C8300081E394E10E94971F81E394E10E94191221
:10C84000811104C068E378E00C94745081E394E1B2
:10C850000E94E106892B51F081E394E10E94AE0829
:10C86000682F81E89FE00E944873F0CF81E394E154
:10C870000E9425120C94AF496DE278E0CE0101963A
:10C880000E943E7BBE016F5F7F4FCE01C4960E9427
:10C890008F79182FCE0101960E94A57A1123E9F015
:10C8A0008DB79EB78A5291400FB6F8949EBF0FBEC7
:10C8B0008DBFADB7BEB711968AE291E0E5EDF2E12A
:10C8C00001900D920197E1F70E947B320FB6F89428
:10C8D000DEBF0FBECDBF0C94AF4966E378E0CE015A
:10C8E00001960E943E7BBE016F5F7F4FCE01C496D2
:10C8F0000E948F79182FCE0101960E94A57A1123EC
:10C9000009F459C08DB79EB78A5291400FB6F8947A
:10C910009EBF0FBE8DBFADB7BEB711968AE291E044
:10C92000E5EDF2E101900D920197E1F70E94582D9B
:10C930000FB6F894DEBF0FBECDBF63E778E0CE013F
:10C9400001960E942C7B8DB79EB78A5291400FB6FC
:10C95000F8949EBF0FBE8DBFADB7BEB711968AE2E9
:10C9600091E0E5EDF2E101900D920197E1F70E946F
:10C97000DC220FB6F894DEBF0FBECDBF8DB79EB7D9
:10C980008A5291400FB6F8949EBF0FBE8DBFADB7CF
:10C99000BEB711968AE291E0E5EDF2E101900D92C9
:10C9A0000197E1F70E947B320FB6F894DEBF0FBE0D
:10C9B000CDBF0C94A54C68E378E0CE0101960E94AF
:10C9C0003E7BBE016F5F7F4FCE01C4960E948F7980
:10C9D000182FCE0101960E94A57A1123B1F061E6CD
:10C9E00078E0CE0101960E942C7BBE016F5F7F4FE5
:10C9F000CE014C960E94357BCE014C960E94691F59
:10CA0000CE014C960E94A57AB9CF6CE378E0CE01B6
:10CA100001960E943E7BBE016F5F7F4FCE01C496A0
:10CA20000E948F79182FCE0101960E94A57A1123BA
:10CA300009F4F5C065E478E0CE0182960E942C7B73
:10CA4000BE016E5D7F4FCE0101960E94357BAE0127
:10CA50004F5F5F4F62E070E088E792E00E94FB2E3C
:10CA6000182FCE0101960E94A57A111122C0BE0195
:10CA70006E5D7F4FCE014C960E94357B60E478E07E
:10CA8000CE014C960E94AA796DEF71E10E94C079A7
:10CA9000BC01CE0101960E94357BCE0101960E9419
:10CAA000691FCE0101960E94A57ACE014C960E9484
:10CAB000A57A68EE73E080E090E00E940C7FBE01F2
:10CAC0006E5D7F4FCE0101960E94357BAE014F5FB8
:10CAD0005F4F63E070E08BE692E00E94FB2E182F20
:10CAE000CE0101960E94A57A111122C0BE016E5D91
:10CAF0007F4FCE014C960E94357B6AEC75E0CE01EB
:10CB00004C960E94AA796DEF71E10E94C079BC0138
:10CB1000CE0101960E94357BCE0101960E94691FCD
:10CB2000CE0101960E94A57ACE014C960E94A57A6C
:10CB300068EE73E080E090E00E940C7F61EF71E1AD
:10CB4000CE0101960E94357BAE014F5F5F4F61E0E1
:10CB500070E080ED92E00E94FB2E182FCE0101962E
:10CB60000E94A57A111121C061EF71E1CE014C96AE
:10CB70000E94357B6AEC75E0CE014C960E94AA7942
:10CB80006DEF71E10E94C079BC01CE0101960E9457
:10CB9000357BCE0101960E94691FCE0101960E944D
:10CBA000A57ACE014C960E94A57A68EE73E080E0EB
:10CBB00090E00E940C7F8091AB0C882311F40C94C0
:10CBC000CF5343E160ED72E0CE0101960E94BE9228
:10CBD000BE016F5F7F4F87E694E10E94971F87E653
:10CBE00094E10E941912882311F40C94CF5361EF41
:10CBF00071E187E694E10E94957C66E970E080E04F
:10CC000090E00E940C7F87E694E10E94251262E387
:10CC100070E080E090E00E940C7F0C94CF5360E5C0
:10CC200078E0CE0101960E943E7BBE016F5F7F4F90
:10CC3000CE01C4960E948F79182FCE0101960E94D2
:10CC4000A57A112301F19CEEE92E9BE0F92E01E07B
:10CC500010E0F2E0EF0EF11C8091A8029091A90281
:10CC60008017910714F40C94AF4960E0F7018081BC
:10CC70000E94997D6CE271E080E090E00E940C7F60
:10CC80000F5F1F4FE6CF64E578E0CE0101960E946A
:10CC90003E7BBE016F5F7F4FCE01C4960E948F79AD
:10CCA000182FCE0101960E94A57A112301F18CEE76
:10CCB000E82E8BE0F82E01E010E0F2E0EF0EF11C20
:10CCC0008091A8029091A9028017910714F40C9406
:10CCD000AF4961E0F70180810E94997D6CE271E0CB
:10CCE00080E090E00E940C7F0F5F1F4FE6CF69E568
:10CCF00078E0CE0101960E943E7BBE016F5F7F4FC0
:10CD0000CE01C4960E948F79182FCE0101960E9401
:10CD1000A57A112311F40C94AF4927E030E046E0E6
:10CD200050E06AEC71E1CE0101960E94537BBE0196
:10CD30006F5F7F4F8CEA91E10E946C7ACE01019681
:10CD40000E94A57A8CEA91E10E94F678672B71F433
:10CD50001092EB0B6AEC71E1CE0101960E94357BDB
:10CD6000CE0101960E94F1240C94515681E08093EB
:10CD7000EB0BF0CF4F925F926F927F928F929F92C8
:10CD8000AF92BF92CF92DF92EF92FF920F931F93D9
:10CD9000CF93DF93CDB7DEB72C970FB6F894DEBFF5
:10CDA0000FBECDBF67E370E080918502909186024F
:10CDB0000E94520A84E1482E512C612C712CD12CF6
:10CDC000C12CAFEFCA1ADA0AC301B2010E940C7F6C
:10CDD000E0908502F090860267E370E0C7010E9450
:10CDE000520A8C01B3E0CB16D10434F08EE1C816A0
:10CDF000D10444F4012B51F094E1490E511C611C03
:10CE0000711CDFCF0115110509F0AEC08BE0E816EB
:10CE1000F10409F08EC08090031490900414A09047
:10CE20000514B09006148091FF1390910014A09106
:10CE30000114B091021489879A87AB87BC8764E696
:10CE400070E080E090E00E940C7F60E475E0CE012D
:10CE500001960E942C7BCE0101960E943027CE01C4
:10CE600001960E94A57A61E082E00E949D8921E0FE
:10CE7000B501A401CE0101960E94AD7ABE016F5F9B
:10CE80007F4F83E894E10E94877CCE0101960E9447
:10CE9000A57A6FED83E894E10E94FB896BE375E06E
:10CEA00083E894E10E94A97C20E049855A856B853E
:10CEB0007C85CE0101960E94AD7ABE016F5F7F4FE7
:10CEC00083E894E10E94877CCE0101960E94A57AB6
:10CED00060E678E083E894E10E947F7C89829A8210
:10CEE000AB82BC8289859A85AB85BC858D839E8308
:10CEF000AF83B88729813A814B815C816D817E81C6
:10CF00008F8198852C960FB6F894DEBF0FBECDBFEB
:10CF1000DF91CF911F910F91FF90EF90DF90CF9015
:10CF2000BF90AF909F908F907F906F905F904F9049
:10CF3000089596E1E916F10409F46DCFACE0EA1624
:10CF4000F10409F07CCF8090EC0A9090ED0AA0905B
:10CF5000EE0AB090EF0A8091E80A9091E90AA09158
:10CF6000EA0AB091EB0A67CF0F3F9FEF1907CCF0A9
:10CF70006DE275E0CE0101960E942C7B4AE050E004
:10CF800070E060E0CE0101960E949020CE010196F3
:10CF90000E94A57A6AE075E082EB91E10E94307A06
:10CFA00032C00E3FAFEF1A07B9F16CEF74E0CE015B
:10CFB00001960E942C7B4AE050E070E060E0CE01D8
:10CFC00001960E949020CE0101960E94A57A6DEEF6
:10CFD00074E082EB91E10E94307AB801CE010196B3
:10CFE0000E948378BE016F5F7F4F82EB91E10E94C8
:10CFF000297ACE0101960E94A57A67ED74E082EB52
:10D0000091E10E94D37919821A821B821C821D82AF
:10D010001E821F8218866ECF6CEC74E0CE010196E2
:10D020000E942C7B4AE050E070E060E0CE01019667
:10D030000E949020CE0101960E94A57A6CEA74E0CD
:10D04000ABCF2F923F924F925F926F927F928F92CF
:10D050009F92AF92BF92CF92DF92EF92FF920F9387
:10D060001F93CF93DF93CDB7DEB7AC970FB6F8948D
:10D07000DEBF0FBECDBF8C0167E074E08BEE91E1A7
:10D080000E94797867E370E0809185029091860232
:10D090000E94520A1C0160E376E0C8010E94C81F8A
:10D0A00062E678E0C8010E947F7C6DE074E1CE0109
:10D0B00001960E94357BBE016F5F7F4FC8010E94C1
:10D0C000877CCE0101960E94A57A6BE678E0C801C4
:10D0D0000E947F7C0E94DB8128EE33E040E050E03C
:10D0E0000E94D6A929013A01CE0109960E94632720
:10D0F00061E778E0CE0101960E943E7BBE01675F4A
:10D100007F4FCE0101960E94C079BC01CE010F96DF
:10D110000E94357BBE01615F7F4FC8010E94877C02
:10D12000CE010F960E94A57ACE0101960E94A57AA3
:10D13000CE0109960E94A57AC301B20120E13EE02A
:10D1400040E050E00E94F8A94B015C01B901CE011A
:10D1500087960E9426214CE3C42ED12CE12CF12C81
:10D16000C501B401A70196010E94F8A9B901CE0139
:10D1700009960E94262165E677E0CE0101960E947D
:10D180003E7BBE01675F7F4FCE0101960E94C07952
:10D19000BC01CE0187960E94297ACE0101960E9499
:10D1A000A57ACE0109960E94A57AC301B201A70112
:10D1B00096010E94F8A9CE0109960E94262165E6F3
:10D1C00077E0CE0101960E943E7BBE01675F7F4FF4
:10D1D000CE0101960E94C079BC01CE0187960E94C3
:10D1E000297ACE0101960E94A57ACE0109960E9465
:10D1F000A57A6BE778E0CE0101960E943E7BBE01E6
:10D20000695D7F4FCE0101960E94C0796EE778E09C
:10D210000E94AA79BC01CE0109960E94357BBE010D
:10D22000675F7F4FC8010E94877CCE0109960E94EC
:10D23000A57ACE0101960E94A57A6CE878E0C80133
:10D240000E947F7CCE0101960E94261EB801CE016D
:10D2500001960E940B7C67E878E0C8010E946B7C15
:10D260000E94BA6629833A834B835C836D837E83F5
:10D270008F83988749815A816B817C8121E0CE011F
:10D2800009960E94AD7ABE01675F7F4FCE010F966F
:10D290000E94357B64E978E0CE010F960E94AA795E
:10D2A000BC018BEE91E10E94557ACE010F960E944F
:10D2B000A57ACE0109960E94A57A6BE978E0CE01A5
:10D2C00009960E943E7B6BEE71E1CE0109960E94A9
:10D2D000C079BC01CE010F960E94357BBE01615F13
:10D2E0007F4FC8010E94877CCE010F960E94A57ACD
:10D2F000CE0109960E94A57A4D815E816F81788565
:10D3000021E0CE0109960E94AD7ABE01675F7F4F92
:10D310008BEE91E10E946C7ACE0109960E94A57A6B
:10D320006DEA78E0CE0109960E943E7B6BEE71E1DA
:10D33000CE0109960E94C0796EEB78E00E94AA792E
:10D34000BC01CE010F960E94357BBE01615F7F4F0D
:10D35000C8010E94877CCE010F960E94A57ACE015B
:10D3600009960E94A57A4091450C5091460C609117
:10D37000470C7091480C22E0CE010F960E94AD7AC6
:10D3800065EC78E0CE0109960E943E7BBE01615FAC
:10D390007F4FCE0109960E94C07967ED78E00E9428
:10D3A000AA79BC01CE0145960E94357BBE016B5E19
:10D3B0007F4FC8010E94877CCE0145960E94A57AC6
:10D3C000CE0109960E94A57ACE010F960E94A57AF9
:10D3D0004091410C5091420C6091430C7091440C6F
:10D3E00022E0CE010F960E94AD7A60EE78E0CE0189
:10D3F00009960E943E7BBE01615F7F4FCE01099678
:10D400000E94C07967ED78E00E94AA79BC01CE0144
:10D4100045960E94357BBE016B5E7F4FC8010E941E
:10D42000877CCE0145960E94A57ACE0109960E947E
:10D43000A57ACE010F960E94A57A86EF28168FEF67
:10D4400038062CF46BE076E0C8010E94C81F6BEE32
:10D4500075E0C8010E94C81F22EAC22E22E0D22E27
:10D46000EE24E394F12CE2E0CE0ED11C8091A802D0
:10D470009091A9028E159F050CF468C0B701CE01EA
:10D480004B960E94837860E178E0CE0145960E9439
:10D490003E7BBE01655E7F4FCE0145960E94C079FE
:10D4A00061E876E00E94AA79BC01CE0181960E94D3
:10D4B000357BBE016F5D7F4FC8010E94877CB7013D
:10D4C00083E0660F771F8A95E1F767517D4ECE01A5
:10D4D0000F960E943E7BBE01615F7F4FC8010E9494
:10D4E000877C6EEE78E0C8010E947F7CF601608147
:10D4F0007181660F771F660F771F6F517D4ECE01CA
:10D5000009960E943E7BBE01675F7F4FC8010E9463
:10D51000877C63EF78E0C8010E947F7CCE0109968A
:10D520000E94A57ACE010F960E94A57ACE0181961F
:10D530000E94A57ACE0145960E94A57ACE014B960F
:10D540000E94A57AFFEFEF1AFF0A8DCFCE018796D2
:10D550000E94A57AAC960FB6F894DEBF0FBECDBF81
:10D56000DF91CF911F910F91FF90EF90DF90CF90BF
:10D57000BF90AF909F908F907F906F905F904F90F3
:10D580003F902F9008952F923F924F925F926F920B
:10D590007F928F929F92AF92BF92CF92DF92EF9243
:10D5A000FF920F931F93CF93DF93CDB7DEB7CA528D
:10D5B000D1400FB6F894DEBF0FBECDBFCB5DDE4FBE
:10D5C00059834883C552D14020913F0C3091400C83
:10D5D0002F5F3F4F3093400C20933F0C20913E0C27
:10D5E00021110FC38B016C0181E080933E0C1092DE
:10D5F000400C10923F0C67E074E0CE01875E9E4FB6
:10D600000E943E7B67E074E0CE01815E9E4F0E94E7
:10D610003E7B8091A8029091A9028230910594F0FE
:10D6200020914502309146023093A5022093A40236
:10D63000029741F080914702909148029093A7028F
:10D640008093A60250E040E068EF78E0C6010E94B7
:10D6500016200130110509F0CAC267E074E08BE1C1
:10D6600092E10E9479787E0121E8E20EF11CC70167
:10D67000880F991F880F991FFC01EF51FD4EC75D60
:10D68000DE4FF983E883C952D140312C212C3AE096
:10D69000832E912CA12CB12C44E6442E512C612CCC
:10D6A000712CCB5DDE4FE881F981C552D14080817C
:10D6B000882309F415C2A701BE016F5F7F4FCE0119
:10D6C0008B5D9E4F0E94EE75049759F3BE016F5F0C
:10D6D0007F4FCE018F5F9E4F0E943E7BBE016F5FEA
:10D6E0007E4FCE01875E9E4F0E946C7ACE018F5F87
:10D6F0009E4F0E94A57AB701CE018F5F9E4F0E9478
:10D700003E7BBE016F5F7E4FCE01815E9E4F0E94C9
:10D710006C7ACE018F5F9E4F0E94A57A8091EB0BB1
:10D720008823A1F1BE01675E7E4FCE018F5F9E4FC1
:10D730000E94357B64E876E0CE018F5F9E4F0E94A9
:10D74000AA79BC01CE01895F9E4F0E94357BCE0134
:10D75000895F9E4F0E94801FCE01895F9E4F0E946D
:10D76000A57ACE018F5F9E4F0E94A57AB701CE01A8
:10D770008F5F9E4F0E943E7BCE018F5F9E4F0E9427
:10D78000691FCE018F5F9E4F0E94A57AC35EDE4F58
:10D7900088819981CD51D140049708F0E0C070E0B4
:10D7A00060E0CE01875E9E4F0E945E79823531F047
:10D7B000843521F08D7F843409F0D1C041E050E000
:10D7C000BE01675E7E4FCE018F5F9E4F0E94220A90
:10D7D000CE018F5F9E4F0E94F6788B0161307105FC
:10D7E00021F40091EF131091F0130330110521F48F
:10D7F0000091F1131091F213101611060CF0A9C04C
:10D800008091A8029091A902801791070CF4A1C001
:10D8100070E060E0CE01875E9E4F0E945E798235A7
:10D8200009F0BFC0C7010E94D6A3892B39F4F801C3
:10D83000EE0FFF1FEE55FD4F11821082C7010E94AF
:10D84000D6A381309105A1F5F801EE0FFF1FEE552B
:10D85000FD4F918380839801220F331F220F331FC6
:10D86000C95DDE4F39832883C752D140F901E55A9B
:10D87000FD4F80819181A281B381181619061A0685
:10D880001B0644F0073011050CF086C0408251821F
:10D89000628273820E943986C95DDE4FE881F98118
:10D8A000C752D140E15BFD4F6083718382839383D4
:10D8B000C75DDE4F68817981C952D140CE018D5E4E
:10D8C0009E4F0E943E7BB801E3E0660F771FEA950A
:10D8D000E1F767517D4ECE01835F9E4F0E943E7BF4
:10D8E0006BE172E1CE01895F9E4F0E94357BBE01E4
:10D8F000635F7E4FCE01895F9E4F0E94C07961E1D8
:10D9000079E00E94AA79BE016F5F7E4F0E94C079C4
:10D9100064E876E00E94AA79BE016D5E7E4F0E94A7
:10D92000C07961E876E00E94AA79BC018BE192E1BE
:10D930000E94557ACE01895F9E4F0E94A57ACE0142
:10D94000835F9E4F0E94A57ACE018D5E9E4F0E94FE
:10D95000A57ACE018F5F9E4F0E94A57AA2CEFBE0F2
:10D960002F1631040CF09DCEF6E0F29D8001F39D60
:10D97000100D1124BE016F5F7F4FC8018D599D4E60
:10D980000E94DC78B701C8018F5D9D4E0E94DC7853
:10D990002FEF221A320A85CE80829182A282B38230
:10D9A00079CF863409F074C0C7010E94D6A3892BB1
:10D9B00039F4F801EE0FFF1FE75BFD4F1182108273
:10D9C000C7010E94D6A38130910539F4F801EE0F0A
:10D9D000FF1FE75BFD4F91838083C801880F991F6C
:10D9E000880F991FC95DDE4F99838883C752D14044
:10D9F000FC01E55AFD4F80819181A281B381181607
:10DA000019061A061B063CF007301105E4F54082A2
:10DA10005182628273820E943986C95DDE4FE8813D
:10DA2000F981C752D140E15BFD4F608371838283EE
:10DA30009383C75DDE4F68817981C952D140CE01A1
:10DA40008D5E9E4F0E943E7BB80143E0660F771FBC
:10DA50004A95E1F767517D4ECE01835F9E4F0E944C
:10DA60003E7B6BE172E1CE01895F9E4F0E94357B68
:10DA7000BE01635F7E4FCE01895F9E4F0E94C079D9
:10DA800064E179E03ECF80829182A282B382C3CFEB
:10DA90008434C1F4C7010E94F4A3000F111F000FCA
:10DAA000111FF801E95CFD4F6083718382839383CA
:10DAB0000E943986015B1D4FF80160837183828368
:10DAC000938347CF843509F044CFC7010E94F4A364
:10DAD000000F111F000F111FF801E55AFD4FE4CF91
:10DAE00081E08093AC0C8091AD0C882319F0C601C5
:10DAF0000E9421688091AD0C882329F061EB75E0CC
:10DB0000C6010E94C81F10923E0C80911F12909176
:10DB10002012892B09F46BC0CE01895F9E4F0E94B1
:10DB200063276BED75E0CE018F5F9E4F0E943E7BB9
:10DB3000BE01695F7E4FCE018F5F9E4F0E94C0790C
:10DB400061E876E00E94AA796BE172E10E94C079F7
:10DB5000BC018BE192E10E94557ACE018F5F9E4F0E
:10DB60000E94A57ACE01895F9E4F0E94A57A6BE143
:10DB700072E1CE018F5F9E4F0E94357BAE014F5FF9
:10DB80005E4F62E070E088E792E00E94FB2E182F63
:10DB9000CE018F5F9E4F0E94A57A6BE172E1CE01AC
:10DBA0008F5F9E4F112309F446C00E94357B6AECBB
:10DBB00075E0CE018F5F9E4F0E94AA7963E072E10B
:10DBC0000E94C079BC01CE01895F9E4F0E94357BC7
:10DBD000CE01895F9E4F0E94691FCE01895F9E4FD3
:10DBE0000E94A57ACE018F5F9E4F0E94A57ACE013A
:10DBF000815E9E4F0E94A57ACE01875E9E4F0E9455
:10DC0000A57AC65DDE4F0FB6F894DEBF0FBECDBF5E
:10DC1000DF91CF911F910F91FF90EF90DF90CF9008
:10DC2000BF90AF909F908F907F906F905F904F903C
:10DC30003F902F9008950E94357B6AEC75E0CE01ED
:10DC40008F5F9E4F0E94AA796DEF71E1B9CFFF926D
:10DC50000F931F93CF93DF93EC018B0180913F0CC7
:10DC60009091400C01969093400C80933F0C209132
:10DC70003E0C222339F06AE070E00E9464AB181673
:10DC80001906F4F0FF24F394F0923E0C1092400C2D
:10DC900010923F0C50E040E068EF78E0CE010E9427
:10DCA00016200230110591F0CE010E942168F092F9
:10DCB000AE0C61EB75E0CE010E94C81F10923E0CC5
:10DCC000DF91CF911F910F91FF9008956BE076E067
:10DCD000CE010E94C81FEDCFAF92BF92CF92DF92CC
:10DCE000EF92FF920F931F93CF93DF93CDB7DEB7E1
:10DCF000A0970FB6F894DEBF0FBECDBF67E074E00B
:10DD000085E192E10E94797867E074E089E092E130
:10DD10000E94797855E4C52E52E0D52E62EAE62EAF
:10DD200062E0F62E7BE3A72E72E0B72E01E010E052
:10DD30008091A8029091A902801791070CF480C0ED
:10DD4000F50181919191A191B1915F01892B8A2B6C
:10DD50008B2B19F5F70182819381F60120813181A6
:10DD600082179307D1F0880F991FFC01E951F44FF6
:10DD7000D801AA0FBB1FA451B44F60818C910E949F
:10DD8000997DF70182819381F6019183808364E616
:10DD900070E080E090E00E940C7FF601619171914B
:10DDA0006F01CE0145960E948378B801CE010F968F
:10DDB0000E948378B80123E0660F771F2A95E1F768
:10DDC00067517D4ECE0109960E943E7B61E876E068
:10DDD000CE0101960E943E7BBE01675F7F4FCE0160
:10DDE00001960E94C07961E179E00E94AA79BE01A2
:10DDF000615F7F4F0E94C07964E876E00E94AA7953
:10DE0000BE016B5E7F4F0E94C079BC0185E192E14B
:10DE10000E94297ACE0101960E94A57ACE01099628
:10DE20000E94A57ACE010F960E94A57ACE01459652
:10DE30000E94A57A0F5F1F4FF2E0EF0EF11C78CF22
:10DE4000E091EF13F091F013EE0FFF1FED5BFD4F2C
:10DE500060817181CE0101960E94837846E050E096
:10DE6000BE016F5F7F4FCE0109960E944920BE011F
:10DE7000675F7F4F89E092E10E94297ACE0109967F
:10DE80000E94A57ACE0101960E94A57AE091F11335
:10DE9000F091F213EE0FFF1FED5BFD4F608171817A
:10DEA000CE0101960E94837846E050E0BE016F5F8C
:10DEB0007F4FCE0109960E944920BE01675F7F4FC8
:10DEC00089E092E10E94297ACE0109960E94A57A02
:10DED000CE0101960E94A57A61E876E0CE014596D2
:10DEE0000E943E7B0E94DB8128EE33E040E050E060
:10DEF0000E94D6A969017A0167E074E0CE014B96D1
:10DF00000E943E7B67E074E08BE192E10E947978A9
:10DF1000CE0101960E94632744E150E0BE016F5F8D
:10DF20007F4FCE0109960E944920BE01675F7F4F57
:10DF30008BE192E10E946C7ACE0109960E94A57A4B
:10DF4000CE0101960E94A57A2AE0B701A601CE0172
:10DF500009960E94DD7A48E050E0BE01675F7F4F7E
:10DF6000CE010F960E9449206BE172E1CE0101962D
:10DF70000E94357BBE01615F7F4FCE0101960E94FA
:10DF8000C079BC018FE092E10E94557ACE010196E2
:10DF90000E94A57ACE010F960E94A57ACE0109961D
:10DFA0000E94A57A2AE0B701A601CE0109960E9437
:10DFB000DD7A68E179E0CE0101960E943E7BBE01E8
:10DFC000675F7F4FCE0101960E94C079BE016B5EF4
:10DFD0007F4F0E94C079BC018BE192E10E94297AB7
:10DFE000CE0101960E94A57ACE0109960E94A57ADB
:10DFF0004091450C5091460C6091470C7091480C33
:10E0000021E0CE0101960E94AD7ABE016F5F7F4F85
:10E01000CE014B960E946C7ACE0101960E94A57AA1
:10E020006FE179E0CE0101960E943E7BBE01655E04
:10E030007F4FCE0101960E94C079BE016B5E7F4F7B
:10E040000E94C079BC018BE192E10E94297ACE0145
:10E0500001960E94A57ABE01655E7F4FCE010196B2
:10E060000E94357B46E050E0BE016F5F7F4FCE01DE
:10E0700009960E944920BE01675F7F4F8FE092E1C1
:10E080000E94297ACE0109960E94A57ACE010196B6
:10E090000E94A57A4091410C5091420C6091430C32
:10E0A0007091440C21E0CE0101960E94AD7ABE0130
:10E0B0006F5F7F4FCE014B960E946C7ACE01019626
:10E0C0000E94A57A6DE279E0CE0101960E943E7B26
:10E0D000BE01655E7F4FCE0101960E94C079BE01F0
:10E0E0006B5E7F4F0E94C079BC018BE192E10E9480
:10E0F000297ACE0101960E94A57ABE01655E7F4F06
:10E10000CE0101960E94357B46E050E0BE016F5F74
:10E110007F4FCE0109960E944920BE01675F7F4F65
:10E120008FE092E10E94297ACE0109960E94A57A99
:10E13000CE0101960E94A57A80910E0C90910F0C51
:10E14000892B61F067E370E08091850290918602EF
:10E150000E94520A90930F0C80930E0C80910E0C2B
:10E1600090910F0C892B09F0EEC00E94BA662983AA
:10E170003A834B835C836D837E838F839887498149
:10E180005A816B817C8121E0CE0109960E94AD7A93
:10E19000BE01675F7F4FCE014B960E946C7ACE0125
:10E1A00009960E94A57A67E379E0CE0109960E945C
:10E1B0003E7BBE01655E7F4FCE0109960E94C0790D
:10E1C000BE016B5E7F4F0E94C079BC018BE192E182
:10E1D0000E94297ACE0109960E94A57ABE01655E49
:10E1E0007F4FCE0109960E94357B46E050E0BE018C
:10E1F000675F7F4FCE010F960E944920BE01615F8D
:10E200007F4F8FE092E10E94297ACE010F960E9403
:10E21000A57ACE0109960E94A57A4D815E816F8113
:10E22000788521E0CE0109960E94AD7ABE01675F34
:10E230007F4FCE014B960E946C7ACE0109960E94C8
:10E24000A57A62E479E0CE0109960E943E7BBE0188
:10E25000655E7F4FCE0109960E94C079BE016B5E5C
:10E260007F4F0E94C079BC018BE192E10E94297A24
:10E27000CE0109960E94A57ABE01655E7F4FCE0150
:10E2800009960E94357B46E050E0BE01675F7F4FF4
:10E29000CE010F960E944920BE01615F7F4F8FE043
:10E2A00092E10E94297ACE010F960E94A57ACE01B2
:10E2B00009960E94A57A65E172E18BE192E10E94E4
:10E2C000297A61E876E0CE0101960E943E7B69E002
:10E2D00072E1CE0101960E94C079BC018FE092E10B
:10E2E0000E94297ACE0101960E94A57A6FE072E120
:10E2F000CE0101960E94357BCE0101960E94691FD6
:10E30000CE0101960E94A57A6AE070E080E090E07C
:10E310000E940C7FCE014B960E94A57ACE014596B5
:10E320000E94A57AA0960FB6F894DEBF0FBECDBFAF
:10E33000DF91CF911F910F91FF90EF90DF90CF90E1
:10E34000BF90AF90089568E479E08BE192E10E947C
:10E350001F7A67E579E08FE092E10E941F7A6EE50F
:10E3600079E08BE192E10E941F7A67E579E08FE026
:10E3700092E10E941F7A9FCFDF92EF92FF920F935C
:10E380001F93CF93DF93CDB7DEB7C451D1400FB603
:10E39000F894DEBF0FBECDBFCD5EDE4F59834883FC
:10E3A000C351D14020913F0C3091400C2F5F3F4F23
:10E3B0003093400C20933F0C20913E0C21113FC024
:10E3C0008B017C01DD24D394D0923E0C1092400C42
:10E3D00010923F0C67E074E0CE01895F9E4F0E946F
:10E3E0003E7B67E074E0CE01835F9E4F0E943E7BE0
:10E3F00050E040E068EF78E0C7010E94162001304D
:10E40000110599F467E074E08BE192E10E9479785C
:10E41000CD5EDE4FE881F981C351D1408081811109
:10E420001DC00E946C6ED092AE0CCE01835F9E4FD9
:10E430000E94A57ACE01895F9E4F0E94A57ACC5E8C
:10E44000DE4F0FB6F894DEBF0FBECDBFDF91CF9188
:10E450001F910F91FF90EF90DF900895CD5EDE4FFA
:10E46000E881F981C351D1408081882309F465C0D6
:10E47000AE014F575F4FBE016F5F7F4FCE018D5E84
:10E480009E4F0E94EE75049749F3BE016F5F7F4F68
:10E49000CE018F5F9E4F0E943E7BBE016F5F7E4F1D
:10E4A000CE01895F9E4F0E946C7ACE018F5F9E4F96
:10E4B0000E94A57ABE016F577F4FCE018F5F9E4F9E
:10E4C0000E943E7BBE016F5F7E4FCE01835F9E4FF9
:10E4D0000E946C7ACE018F5F9E4F0E94A57ABE018A
:10E4E000695F7E4F8BE192E10E94297ACF5EDE4F19
:10E4F00088819981C151D140892B09F4AFCF64E85B
:10E5000076E0CE018F5F9E4F0E943E7BBE01635F2F
:10E510007E4FCE018F5F9E4F0E94C07961E876E00A
:10E520000E94AA79BC018BE192E10E94297ACE0176
:10E530008F5F9E4F0E94A57A91CF6BE172E187EFCA
:10E5400091E10E94557A71CF089508950895089534
:10E55000AF92BF92CF92DF92EF92FF920F931F93F1
:10E56000CF93DF936C017B018B01040F151FEB012F
:10E570005E01AE18BF08C017D10759F06991D601E6
:10E58000ED91FC910190F081E02DC6011995892B48
:10E5900079F7C501DF91CF911F910F91FF90EF9017
:10E5A000DF90CF90BF90AF900895FC01538D448DC4
:10E5B000252F30E0842F90E0821B930B541710F02E
:10E5C000CF96089501970895FC01918D828D98173B
:10E5D00061F0A28DAE0FBF2FB11D5D968C91928D13
:10E5E0009F5F9F73928F90E008958FEF9FEF089544
:10E5F000FC01918D828D981731F0828DE80FF11D0D
:10E60000858D90E008958FEF9FEF0895FC01918D27
:10E61000228D892F90E0805C9F4F821B91098F7320
:10E620009927089584EE9EE00E94067321E0892BCD
:10E6300009F420E0822F089581E89FE00E9406738C
:10E6400021E0892B09F420E0822F0895FC01A48D9C
:10E65000A80FB92FB11DA35ABF4F2C91848D90E004
:10E6600001968F739927848FA689B7892C93A089E7
:10E67000B1898C91837080648C93938D848D981371
:10E6800006C00288F389E02D80818F7D8083089504
:10E69000EF92FF920F931F93CF93DF93EC0181E0F2
:10E6A000888F9B8D8C8D98131AC0E889F989808199
:10E6B00085FF15C09FB7F894EE89FF896083E889CC
:10E6C000F98980818370806480839FBF81E090E0BE
:10E6D000DF91CF911F910F91FF90EF900895F62E4B
:10E6E0000B8D10E00F5F1F4F0F731127E02E8C8DE5
:10E6F0008E110CC00FB607FCFACFE889F98980812A
:10E7000085FFF5CFCE010E942673F1CFEB8DEC0F84
:10E71000FD2FF11DE35AFF4FF0829FB7F8940B8F46
:10E72000EA89FB8980818062CFCFCF93DF93EC01B0
:10E73000888D8823B9F0AA89BB89E889F9898C91E9
:10E7400085FD03C0808186FD0DC00FB607FCF7CFA5
:10E750008C9185FFF2CF808185FFEDCFCE010E94A5
:10E760002673E9CFDF91CF91089580E090E0892B67
:10E7700029F00E941C7381110E94000080E090E04B
:10E78000892B49F080E090E0892B29F00E9400005D
:10E7900081110E94000080E090E0892B49F080E028
:10E7A00090E0892B29F00E94000081110E94000056
:10E7B00080E090E0892B29F00E94127381110C9463
:10E7C000000008958150823108F05AC0E82FF0E02F
:10E7D0008827E251FC488F4F0C9478AB0E7412746A
:10E7E000007406740A74407415741B741F742574C5
:10E7F00029742D743374377440743B7441744574B8
:10E80000809180008F7780938000089580918000B0
:10E810008F7DF9CF80918000877FF5CF84B58F778A
:10E8200084BD089584B58F7DFBCF8091B0008F7734
:10E830008093B00008958091B0008F7DF9CF8091D2
:10E8400090008F77809390000895809190008F7D45
:10E85000F9CF80919000877FF5CF8091A0008F77CE
:10E860008093A00008958091A0008F7DF9CF8091C2
:10E87000A000877FF5CF809120018F7780932001C2
:10E880000895809120018F7DF9CF80912001877FAD
:10E89000F5CFCF93DF93282F30E0F901E250F54F09
:10E8A0008491F901EE58F34FD491F901E854F34FF4
:10E8B000C491CC23A1F081110E94E273EC2FF0E00F
:10E8C000EE0FFF1FEC51F54FA591B491EC91ED23A4
:10E8D00081E090E009F480E0DF91CF91089580E03D
:10E8E00090E0FACF2091BA14260F3327331F21323C
:10E8F0003105ECF42091D90EFC0190E080E0243049
:10E9000069F082E00895A091BA142191AC014656B5
:10E910005B4EA40FB52FB11D2C930196861798F36B
:10E920008091BA14680F6093BA1480E0089581E072
:10E930000895E091A20C8091A10CE81730F4F0E06A
:10E94000EF5EF34F808190E008958FEF9FEF089581
:10E950009091A20C8091A10C2FEF3FEF981748F4F3
:10E96000E92FF0E0EF5EF34F208130E09F5F90935E
:10E97000A20CC90108958091A10C9091A20C891B51
:10E98000990B0895CF92DF92EF92FF920F931F930E
:10E99000CF93DF937C01CB018A012091DF0E2223EC
:10E9A00089F0EB016B01C40ED51ECC15DD0569F0B5
:10E9B0006991D701ED91FC910190F081E02DC701A3
:10E9C0001995F3CF642F0E947274C801DF91CF9123
:10E9D0001F910F91FF90EF90DF90CF900895CF930C
:10E9E000DF931F92CDB7DEB769832091DF0E22231C
:10E9F000F9F02091E20E203258F021E030E0FC01E5
:10EA00003383228390E080E00F90DF91CF910895CF
:10EA10008091E00EE82FF0E0E154F94E9981908367
:10EA20008F5F8093E00E8093E20E81E090E0ECCF68
:10EA300061E0CE0101960E947274F7CF0E94A1ADF1
:10EA40000F931F93CF93DF93EC01888199810097F7
:10EA500059F02A813B812617370730F081E0DF919A
:10EA6000CF911F910F9108958B016F5F7F4F0E948F
:10EA7000C0AC009759F0998388831B830A832C814B
:10EA80003D81232B59F7FC011082E8CF80E0E7CFCE
:10EA9000EF92FF920F931F93CF93DF936115710550
:10EAA00041F480E0DF91CF911F910F91FF90EF90A3
:10EAB000089541155105B1F07B01EC010C811D81D8
:10EAC000040F151FB8010E942075882351F3288177
:10EAD00039818C819D81B701820F931F0E94F1AD16
:10EAE0001D830C8381E0DECFCF93DF93EC0188811F
:10EAF0009981009711F00E9437AC198218821D820B
:10EB00001C821B821A82DF91CF910895EF92FF92AF
:10EB10000F931F93CF93DF93EC017B018A01BA011E
:10EB20000E94207581110BC0CE010E947475CE0128
:10EB3000DF91CF911F910F91FF90EF9008951D836A
:10EB40000C83B701888199810E94F1ADF0CF8CBD13
:10EB50009DBD0895CF93DF93EC019A01AB01E88945
:10EB6000F98982E08083211581EE3807410551053E
:10EB700081F160E079E08DE390E00E94D6A9215018
:10EB80003109410951095695479537952795EC85E7
:10EB9000FD851082EE85FF852083188EEC89FD8926
:10EBA00086E08083EA89FB89808180618083EA89AD
:10EBB000FB89808188608083EA89FB898081806805
:10EBC0008083EA89FB8980818F7D8083DF91CF916B
:10EBD0000895E889F989108220E1D9CF8F929F9218
:10EBE000AF92BF92CF92DF92EF92FF920F931F935B
:10EBF000CF93DF9300D0CDB7DEB74C017B016A0124
:10EC0000DC01ED91FC9180E8DB01982F1D929A9533
:10EC1000E9F7DA011D928A95E9F7808190E8A92E3B
:10EC2000B12C811119C084E090E006C08F0181E011
:10EC300090E0D4010D931C930F900F900F90DF91F3
:10EC4000CF911F910F91FF90EF90DF90CF90BF90E9
:10EC5000AF909F908F9008958F010F5F1F4F60813D
:10EC6000663229F394F4662309F36532D1F0B2E0F9
:10EC7000AB16B10444F0F7016083F1E0AF1AB108BC
:10EC8000C70101967C01F801E7CF6B3209F45EC041
:10EC90006D3369F78181882351F280E8A82EB12C69
:10ECA00045C081818983882311F282818A838F0103
:10ECB000811103C00E5F1F4FBACF0D5F1F4F1B8224
:10ECC00040E150E070E060E0CE0101960E94CFA2EA
:10ECD000CECF663281F06B32A1F560E232C0F8012E
:10ECE000818189838823A1F182818A83811107C070
:10ECF0000E5F1F4F7801870183E090E09ACF780183
:10ED0000F3E0EF0EF11C1B8240E150E070E060E0A8
:10ED1000CE0101960E94CFA214C0D6016C93B1E03F
:10ED2000AB1AB108F60131966F01870178019FEFA8
:10ED3000E91AF90AD8016C91653289F254F6662312
:10ED4000C9F2E2E0AE16B10444F7EFCF60E28FCF34
:10ED50008701D0CF0F931F93CF93DF9341155105B8
:10ED600041F0FC01048115810115110539F4FB0105
:10ED70001082DF91CF911F910F9108954150510959
:10ED80004017510708F48A01EB01FC016081718191
:10ED9000A801CE010E9406AEC00FD11F1882E9CF94
:10EDA00020E3FC0120833296862F82958F706F704E
:10EDB0006A3030F4605D6293682F8111F5CF089559
:10EDC000695CF9CF5F926F927F928F929F92AF9220
:10EDD000BF92CF92DF92EF92FF920F931F93CF9348
:10EDE000DF93CDB7DEB7C754D1090FB6F894DEBFB5
:10EDF0000FBECDBF5C013B0119A218A28CE593E0C8
:10EE00009F8F8E8F1BA21C821B829A8389831E82F6
:10EE100010E000E06E018EE1C80ED11C84E5E82E02
:10EE200080E1F82EF501E00FF11F80818F3211F49F
:10EE30000F5F1F4FD501A00FB11FFE01FB9690E0A1
:10EE400080E04F012D912F3249F0222339F00F5FDE
:10EE50001F4F019621938C309105A1F7880D991DC4
:10EE6000FC011082F501E00FF11F80818F3211F457
:10EE70000F5F1F4FF501E00FF11F508041E051106F
:10EE800040E030E020E0B401C701F30119958111A1
:10EE900021C0F4E5EF16F0E1FF06C1F480E0C95BA4
:10EEA000DF4F0FB6F894DEBF0FBECDBFDF91CF911D
:10EEB0001F910F91FF90EF90DF90CF90BF90AF9098
:10EEC0009F908F907F906F905F900895C7010E94F0
:10EED0004B0DE4CF552091F021E0A401B701C6010C
:10EEE0000E94510E982E84E5E81680E1F80681F024
:10EEF000C7010E944B0D911010C0D0CF94E5E916C8
:10EF000090E1F90619F0C7010E944B0D81E0C7CFCF
:10EF1000992021F2FE0131967F019E2D8F2D7601E1
:10EF2000C92ED82E7FCF8F929F92AF92BF92CF9251
:10EF3000DF92EF92FF920F931F93CF93DF93CDB7A2
:10EF4000DEB760970FB6F894DEBF0FBECDBF7C0171
:10EF50009091A60C992351F108E0933309F404E051
:10EF60006B0180E591E00E94A7759E012F5F3F4FE6
:10EF70005901490110E0812F0E940814F401819386
:10EF80004F018823D9F01F5F0113F5CF00E0F50191
:10EF900081915F018D3161F0883151F08A51823069
:10EFA00038F00F5F1013F3CF0E94831518E08AC06A
:10EFB00060E170E0802F0E946614102FA12EB12C0A
:10EFC000F501EE0FFF1FEF56F34F1182108283EE13
:10EFD00093E00197F1F742E870E060E0812F0E9432
:10EFE00049144FEF62E070E0812F0E944914B6018E
:10EFF000C114D10491F48091AE029091AF020196B8
:10F000008115F0EC9F0708F471C09093AF028093D4
:10F01000AE026091AE027091AF02812F0E94331454
:10F0200086E0E3E1F3E0DE01199601900D928A9506
:10F03000E1F7F70183818F778C8784818D878581C4
:10F040008E87A7014E5F5F4F24E030E06CE070E0F8
:10F05000812F0E940C14B601812F0E941D1426E0FE
:10F0600030E0AE01475F5F4F66E070E0812F0E94A5
:10F070000C1461E070E0812F0E94661427E02A9D45
:10F08000C0012B9D900D11249C01275A334F79010B
:10F09000F9011182108222E030E0AE01415F5F4F42
:10F0A00068E270E0812F0E9476148F8598899827F6
:10F0B00089279827F7019383828316821582148209
:10F0C0000E948315812F60960FB6F894DEBF0FBEA5
:10F0D000CDBFDF91CF911F910F91FF90EF90DF9007
:10F0E000CF90BF90AF909F908F90089580E090EC6C
:10F0F0008CCFFB0101900020E9F73197AF01461B4F
:10F10000570B0C9486750F931F93CF93DF93CDB756
:10F11000DEB762970FB6F894DEBF0FBECDBF8C018D
:10F12000CB01F8011182108213821282158214829F
:10F130004AE0BE016F5F7F4F0E9434A4BE016F5F43
:10F140007F4FC8010E94797862960FB6F894DEBFAF
:10F150000FBECDBFDF91CF911F910F9108950F93F7
:10F160001F93CF93DF93CDB7DEB7A1970FB6F89477
:10F17000DEBF0FBECDBF8C01CB01BA01F8011182F9
:10F18000108213821282158214822AE0AE014F5F30
:10F190005F4F0E9476A4BE016F5F7F4FC8010E943F
:10F1A0007978A1960FB6F894DEBF0FBECDBFDF9180
:10F1B000CF911F910F910895CF93DF93EC016115CB
:10F1C000710531F00E947978CE01DF91CF910895D9
:10F1D0000E947475F9CFFC0180819181009711F034
:10F1E0000C94D2A360E070E0CB010895FC01808113
:10F1F0009181009711F00C94F4A360E070E0CB01D2
:10F200000895AF92BF92CF92DF92EF92FF920F9349
:10F210001F93CF93DF93DC01CD90DC901197C11445
:10F22000D10439F01496CD91DC918C0176012097B0
:10F2300061F4DF91CF911F910F91FF90EF90DF90DC
:10F24000CF90BF90AF90089575015701BFEFAB1AF3
:10F25000BB0AF7018081082E000C990B0E941BA4A9
:10F26000892B91F72197CC0DDD1D8881082E000C8C
:10F27000990B0E941BA4892B29F0CE15DF0510F0F5
:10F280002197F3CFAE014F5F5F4F4E195F09D80151
:10F2900015965C934E931497CE14DF0420F4B701B7
:10F2A000C6010E94BBADD801ED91FC911197149657
:10F2B0008D919C91E80FF91F1082BBCFFC01248136
:10F2C00035816217730748F480819181009729F096
:10F2D000860F971FFC018081089580E00895FC014E
:10F2E00024813581FB014481558124173507A0F025
:10F2F000FC0180819181009779F0FB01608171812F
:10F300006115710549F0241B350B820F931F0E9474
:10F31000E8AD21E0892B09F020E0822F0895FB0160
:10F3200044815581FC01248135812417350778F00B
:10F3300080819181009759F0FB0160817181611595
:10F34000710529F00E94F8AD21E0892B09F020E039
:10F35000822F0895CF93DF93EC01FB0101900020F1
:10F36000E9F73197AF01461B570B0E944875811191
:10F3700003C0CE010E947475CE01DF91CF91089534
:10F38000CF93DF93EC01FB01448155816081718152
:10F390000E944875811103C0CE010E947475CE0190
:10F3A000DF91CF910895EF92FF920F931F93CF9328
:10F3B000DF93EC017B01CB010E942BA40097A9F005
:10F3C0000C811D81080F191FB801CE010E94207504
:10F3D000882361F0288139818C819D81B701820F5A
:10F3E000931F0E9424A41D830C8381E0DF91CF91A1
:10F3F0001F910F91FF90EF900895CF93DF931F928D
:10F400001F92CDB7DEB769831A8241E050E0BE019A
:10F410006F5F7F4F0E9448750F900F90DF91CF91E3
:10F420000895CF93DF93EC010E94FD79811103C011
:10F43000CE010E947475CE01DF91CF910895FB013A
:10F4400001900020E9F73197AF01461B570B0C9450
:10F450004875FB0144815581608171810C94487528
:10F46000EF92FF920F931F93CF93DF93EC018B01E9
:10F47000CB010E942BA47C01BC01CE010E9420750F
:10F4800081110BC0CE010E947475CE01DF91CF9126
:10F490001F910F91FF90EF900895FD82EC82B801CB
:10F4A000888199810E9424A4F0CFCF93DF93EC014F
:10F4B000FB018617970749F060817181611571051D
:10F4C00041F0448155810E948675CE01DF91CF9134
:10F4D00008950E947475F9CF0F931F93CF93DF9314
:10F4E0008C01EB01FC01808191810097E1F0688142
:10F4F000798161157105A9F0428153812C813D818B
:10F500004217530770F00E94F1AD8C819D81F80184
:10F51000958384831D821C82DF91CF911F910F916F
:10F5200008950E9437AC88819981F8019183808386
:10F530008A819B81938382838C819D81958384833F
:10F54000198218821B821A82E5CFFC018081918189
:10F55000009711F00C9437AC0895EF92FF920F933F
:10F560001F93CF93DF93CDB7DEB7A1970FB6F89473
:10F57000DEBF0FBECDBF7C01CB01BA01F701118206
:10F580001082138212821582148242E0420F8E0191
:10F590000F5F1F4F0E940DA2BC01C7010E94DC78C3
:10F5A000A1960FB6F894DEBF0FBECDBFDF91CF910D
:10F5B0001F910F91FF90EF9008950F931F93CF939A
:10F5C000DF93CDB7DEB7A2970FB6F894DEBF0FBEBC
:10F5D000CDBF8C01CB01BA01F801118210821382D8
:10F5E00012821582148230E0AE014F5F5F4F0E949D
:10F5F0003FA4BE016F5F7F4FC8010E947978A29639
:10F600000FB6F894DEBF0FBECDBFDF91CF911F9133
:10F610000F910895CF93DF931F921F92CDB7DEB75E
:10F62000FC01118210821382128215821482698376
:10F630001A82BE016F5F7F4F0E9479780F900F9002
:10F64000DF91CF910895FC01118210821382128202
:10F65000158214820C946C7AFC0111821082138240
:10F660001282158214820C94307AFC01118210826D
:10F6700013821282158214820C94557AFC01118235
:10F68000108213821282158214826115710551F065
:10F69000FB0101900020E9F73197AF01461B570BA2
:10F6A0000C9486750895AF92BF92CF92DF92EF923D
:10F6B000FF920F931F93CF93DF935C016B017A014D
:10F6C00089012417350720F48F2D7901042F182F75
:10F6D00067E074E0C5010E943E7BD6011496CD918F
:10F6E000DC91EC16FD06C8F40C171D0708F4E801C0
:10F6F000D601ED91FC911197EC0FFD1F1081108246
:10F700006D917C916E0D7F1DC5010E94DC78F60124
:10F7100080819181C80FD91F1883C501DF91CF91D6
:10F720001F910F91FF90EF90DF90CF90BF90AF901F
:10F730000895FB0101900020E9F73197AF01461BC6
:10F74000570BDC01ED91FC910280F381E02D1994BF
:10F750008F929F92AF92BF92EF92FF920F931F935F
:10F76000CF93DF93CDB7DEB7A1970FB6F894DEBF86
:10F770000FBECDBF7C01FA01CB0119A2223008F4E3
:10F780002AE08E010F5D1F4F822E912CB12CA12CEF
:10F79000BF01A50194010E94D6A9F901CA016A30EE
:10F7A0000CF5605DD8016E938D01232B242B252B46
:10F7B00079F790E080E0109721F0BD01C7010E9429
:10F7C000997BA1960FB6F894DEBF0FBECDBFDF9137
:10F7D000CF911F910F91FF90EF90BF90AF909F90AE
:10F7E0008F900895695CDECFCF93DF93482F50E070
:10F7F00070E060E020E181E89FE00E94A87BEC01DE
:10F8000061ED79E081E89FE00E94997B8C0F9D1F5C
:10F81000DF91CF9108958F929F92AF92BF92CF9236
:10F82000DF92EF92FF920F931F93CF93DF937C01B0
:10F83000EB016C0182E0C80ED11C4701E5E08E0EA1
:10F84000911C10E000E0F60141916F0150E070E082
:10F8500060E02AE0CE010E94A87B5C01E881F9818A
:10F860000190F081E02D6EE2CE0119958A0D9B1D6D
:10F87000080F191FC814D90431F7F701458150E06A
:10F8800070E060E02AE0CE010E94A87B800F911F0B
:10F89000DF91CF911F910F91FF90EF90DF90CF906C
:10F8A000BF90AF909F908F9008950F931F93CF9329
:10F8B000DF93EC01CB01BE010E940B7C8C0161ED5A
:10F8C00079E0CE010E94997B800F911FDF91CF914B
:10F8D0001F910F9108950F931F93CF93DF93EC0126
:10F8E0000E94997B8C0161ED79E0CE010E94997BA9
:10F8F000800F911FDF91CF911F910F910895611596
:10F90000710511F00C94997B90E080E00895DB0183
:10F9100014964D915C9115976D917C91DC01ED9160
:10F92000FC910280F381E02D19940F931F93CF93E4
:10F93000DF93EC010E94877C8C0161ED79E0CE01C0
:10F940000E94997B800F911FDF91CF911F910F91A2
:10F950000895EF92FF920F931F93CF93DF938C0143
:10F960007B01D0E0C0E0F701EC0FFD1F649166233E
:10F9700061F0D801ED91FC910190F081E02DC8017A
:10F980001995892B11F02196EECFCE01DF91CF9101
:10F990001F910F91FF90EF900895DC018CEF93E0A1
:10F9A0008D939D9384E0FB0101900D928A95E1F780
:10F9B00008951F920F920FB60F9211240BB60F925B
:10F9C0002F933F934F935F936F937F938F939F9367
:10F9D000AF93BF93EF93FF9384EE9EE00E94267354
:10F9E000FF91EF91BF91AF919F918F917F916F9117
:10F9F0005F914F913F912F910F900BBE0F900FBED3
:10FA00000F901F9018951F920F920FB60F9211240E
:10FA10000BB60F922F938F939F93EF93FF93E091E9
:10FA2000F40EF091F50E8081E091FA0EF091FB0E4C
:10FA300082FD1DC090818091FD0E8F5F8F7320919C
:10FA4000FE0E821741F0E091FD0EF0E0EC51F14F17
:10FA5000958F8093FD0EFF91EF919F918F912F9144
:10FA60000F900BBE0F900FBE0F901F9018958081C6
:10FA7000F2CF1F920F920FB60F9211240BB60F9276
:10FA80002F933F934F935F936F937F938F939F93A6
:10FA9000AF93BF93EF93FF9381E89FE00E9426739B
:10FAA000FF91EF91BF91AF919F918F917F916F9156
:10FAB0005F914F913F912F910F900BBE0F900FBE12
:10FAC0000F901F9018951F920F920FB60F9211244E
:10FAD0000BB60F922F938F939F93EF93FF93E09129
:10FAE000910FF091920F8081E091970FF091980F14
:10FAF00082FD1DC0908180919A0F8F5F8F7320913E
:10FB00009B0F821741F0E0919A0FF0E0EF57F04F12
:10FB1000958F80939A0FFF91EF919F918F912F91E5
:10FB20000F900BBE0F900FBE0F901F901895808105
:10FB3000F2CF1F93CF93DF93282F30E0F901E250EB
:10FB4000F54F8491F901EE58F34FD491F901E8543F
:10FB5000F34FC491CC23A9F0162F81110E94E273B8
:10FB6000EC2FF0E0EE0FFF1FE25CF34FA591B49194
:10FB70008FB7F894EC91111108C0D095DE23DC9377
:10FB80008FBFDF91CF911F910895DE2BF8CFAF92F9
:10FB9000BF92CF92DF92EF92FF920F931F93CF937A
:10FBA000DF936B017A01EC01C054DA4E28813CE00E
:10FBB000389F8001399F100D1124A0900F17B12C90
:10FBC00027FF1FC0FB011182108288818F5F88830D
:10FBD00088819801280F311D87FD3A95F6012A1575
:10FBE0003B051CF488818C30C4F18081918104969E
:10FBF00080349C4908F473C0F60180819181049699
:10FC000070C088819801280F311D87FD3A952A150B
:10FC10003B05DCF68881A801480F511D87FD5A95E8
:10FC2000FA01EE0FFF1FE40FF51FE758FF4E80812A
:10FC300086FFCBCF8881F801E80FF11D87FDFA958B
:10FC4000CF01EE0FFF1FE80FF91FE758FF4E80812D
:10FC500060E08F730E94997DB8CF80819181288167
:10FC6000A801420F511D27FD5A959A01FA01EE0F86
:10FC7000FF1FE20FF31FE758FF4E21813281820FF1
:10FC8000931FF7019183808388819801280F311D8C
:10FC900087FD3A95F901EE0FFF1FE20FF31FE758BA
:10FCA000FF4E808186FF22C08881080F111D87FDCD
:10FCB0001A95F801EE0FFF1FE00FF11FE758FF4EF6
:10FCC000808161E08F73DF91CF911F910F91FF9041
:10FCD000EF90DF90CF90BF90AF900C94997D80E42F
:10FCE0009CE9F701918380838FEF8883DF91CF9127
:10FCF0001F910F91FF90EF90DF90CF90BF90AF904A
:10FD000008951092D90E81E08093D80E1092B30E10
:10FD100061E084E10E94997D61E085E10E94997D26
:10FD2000E9EBF0E080818E7F808380818D7F80830E
:10FD300088E48093B80085E48093BC000895109215
:10FD4000A20C1092A10C1092E00E1092E20E0E94F2
:10FD5000817E85EA92E7909352168093511686EA47
:10FD600092E79093501680934F160895CF93DF93A8
:10FD700090E0FC01EE58F34F24918854934FFC011E
:10FD800084918823D1F090E0880F991FFC01E85AF4
:10FD9000F34FA591B491FC01E25CF34FC591D4916E
:10FDA00061110EC09FB7F8948C91E22FE0958E23DD
:10FDB0008C932881E223E8839FBFDF91CF91089540
:10FDC0008FB7F894EC91E22BEC938FBFF6CF3FB74F
:10FDD000F8948091C9159091CA15A091CB15B09156
:10FDE000CC1526B5A89B05C02F3F19F00196A11D83
:10FDF000B11D3FBFBA2FA92F982F8827BC01CD0175
:10FE0000620F711D811D911D42E0660F771F881FD3
:10FE1000991F4A95D1F708958F929F92AF92BF9202
:10FE2000CF92DF92EF92FF926B017C010E94E77EFE
:10FE30004B015C01C114D104E104F104B9F00E944A
:10FE4000E77E681979098A099B09683E7340810534
:10FE5000910580F321E0C21AD108E108F10888EE8B
:10FE6000880E83E0981EA11CB11CE4CFFF90EF9098
:10FE7000DF90CF90BF90AF909F908F900895AF92FA
:10FE8000BF92CF92DF92EF92FF920F931F93CF9387
:10FE9000DF93C82FD62F10920714109208141092D7
:10FEA000091410920A1410920B1461E00E94B67E9D
:10FEB00060E08C2F0E94997D6D2F70E090E080E0D3
:10FEC0000E940C7F60E08C2F0E94B67E8BE990E050
:10FED0000197F1F700E911E08C2F0E944974892BFA
:10FEE00081F401501109C1F78EEF9FEFDF91CF919F
:10FEF0001F910F91FF90EF90DF90CF90BF90AF9048
:10FF0000089500E911E08C2F0E944974019721F4B3
:10FF100001501109C1F7E8CF18E2D0E800E090E9FC
:10FF2000E92EFF24F3948C2F0E944974892B29F425
:10FF300081E0E81AF108B9F7D7CF0E94E77E6B019C
:10FF40007C0180E9A82EBB24B3948C2F0E944974B5
:10FF5000019729F481E0A81AB108B9F7C5CF0E942A
:10FF6000E77E6C197D098E099F096932710581054B
:10FF7000910538F0E02FF0E0E150FC4E80858D2BAC
:10FF80008087D69511F40F5FD0E8115041F690E0CC
:10FF900080E0ACCF0F931F93CF93DF9300D000D0BE
:10FFA0001F921F92CDB7DEB78091B51681112AC07E
:10FFB00010929D1610929C1688EE93E0A0E0B0E09F
:10FFC00080939E1690939F16A093A016B093A116AF
:10FFD00086E893E090939B1680939A168CEF93E0BB
:10FFE0009093A9168093A8161092AA161092AB1699
:10FFF0001092AC161092AD1688E08093B21681E094
:020000021000EC
:100000008093B51687E596E19093A90C8093A80C90
:100010008091561681119DC060E372E080E090E00F
:100020000E940C7F1FB7F89480915516811127C04C
:10003000EDEEFCE08491E7EAFCE09491E82FF0E03B
:10004000EE0FFF1FE85AF34FA591B491EC91E9230D
:1000500021F461E085E30E94997D61E085E30E94DF
:10006000B67E8CB580618CBD8CB580648CBD61E042
:1000700084E30E94B67E61E083E30E94B67E8091B5
:1000800055168F5F809355161FBFE2ECFCE0E4919C
:10009000F0E0EE0FFF1FE25CF34F85919491909397
:1000A000A50C8093A40CECE7FCE0E491E093A30C96
:1000B00061E08AE00E94B67E0E946C1280E591E0C9
:1000C0000E94A77584E38093A60C80E80E94F51334
:1000D0000E94DF13882309F4F5C088E00E94F5131D
:1000E0000E94CC13883009F0EDC080E10E94F51326
:1000F0000E94CC13803109F0E5C080E00E94F51326
:100100000E94CC13182F8111DDC041E050E0BE01E8
:100110006F5F7F4F8FE190E00E947612898183307C
:1001200009F0D0C080E48093A70C42E06EE170E05B
:10013000812F0E94491442E06FE170E0812F0E94FC
:1001400049141F5F183089F70E94831581E080935E
:10015000561680E591E00E94A77546E050E060EBFE
:1001600072E089E090E00E941E138CEF93E09A8386
:1001700089831B821C821D821E82CE0103960E94EF
:100180007C150E9483158091A80C9091A90CDC012C
:1001900092961D921D921D921C929597FC0116A29B
:1001A00017A210A611A69A961D921D921D921C923E
:1001B0009D9740E65AEE60E070E046AB57AB60AF0B
:1001C00071AF40EA5FE060E070E0DA964D935D93D6
:1001D0006D937C93DD973E9624E1DF011D922A9575
:1001E000E9F726E0E0EBF2E0DC01189601900D92D1
:1001F0002A95E1F7FC01EE5BFF4F10820E94EB298C
:100200008C01019709F0CBC080E591E00E94A775B1
:100210006091A80C7091A90C625F7F4FCE0101968E
:100220000E94CD7CCE0103960E947C156091A80CA3
:100230007091A90C6A5E7F4FCE0101960E94CD7C21
:1002400044E050E0BE016D5F7F4F81E090E00E948E
:100250001E136091A80C7091A90C6E5E7F4FCE01A9
:1002600001960E94CD7C44E050E0BE016D5F7F4F5F
:1002700085E090E00E941E130E9483156091A80CF7
:100280007091A90C625E7F4FCE0101960E94CD7CD9
:100290008B819C81AD81BE81809375109093761087
:1002A000A0937710B09378100E94E77E7F738091BF
:1002B000AE029091AF02682779277093AF026093E6
:1002C000AE026DC087E38093A60C80E80E94F51310
:1002D0000E94DF13882329F188E00E94F5130E9411
:1002E000CC138830F1F480E10E94F5130E94CC1306
:1002F000182F8031B1F480E00E94F5130E94CC13D6
:1003000081110FC041E050E0BE016F5F7F4F89E374
:1003100090E00E9476128981843019F41093A70C22
:1003200013CF83E38093A60C80E80E94F5130E940C
:10033000DF13882371F180E10E94F5130E94CC1332
:10034000803139F582E10E94F5130E94CC1382318D
:1003500001F580E00E94F5130E94CC13811119C0B1
:1003600084E08093A70C15E5188741E050E0BE01BA
:10037000685F7F4F8BE190E00E941E131F8341E076
:1003800050E0BE01695F7F4F8AE190E00E941E133A
:10039000DBCE1092A60C0E94831510E000E0C8018D
:1003A00028960FB6F894DEBF0FBECDBFDF91CF9178
:1003B0001F910F9108952FB7F8946091C515709112
:1003C000C6158091C7159091C8152FBF0895CF927B
:1003D000DF92EF92FF92CF93DF93809125118830C7
:1003E00050F0CFEFDFEFCE01DF91CF91FF90EF9094
:1003F000DF90CF900895E0914A11E11142C00E9430
:10040000DB816B017C0128EEC20E23E0D21EE11CD1
:10041000F11C89E191E10E94A319882311F38091D5
:100420008011882331F080914B1190914C11892BD0
:10043000C1F289E191E10E940618EC01CF3FDC078F
:1004400071F080918011882371F280914B1190910D
:100450004C11019790934C1180934B11C4CF0E9483
:10046000DB81C616D706E806F90698F610924A11FF
:1004700089E191E10E94FE1989E191E10E94C5198B
:10048000B2CFE150E0934A110E2E000CFF0BE15F5A
:10049000FE4EC38DD0E0A7CF0F931F93CF93DF9372
:1004A000EC018C01F80181918F018823C1F10E9438
:1004B000E781F8012291022E000C330B821793077B
:1004C00089F38F3F980791F0A0914A1191E09A0F1C
:1004D00090934A110A2E000CBB0BA15FBE4E5B9697
:1004E0008C93903219F48FE180934A112FE1EC172D
:1004F000FD07D9F092919F3FD1F3A0914A1181E07D
:100500008A0F80934A110A2E000CBB0BA15FBE4ECE
:100510005B969C93803259F720934A11E8CF81E093
:10052000DF91CF911F910F91089580E0F9CF0F9344
:100530001F93CF93DF93EC010E94DB818B010E941C
:100540005E108F3F69F00E94DB81601B710B6C179E
:100550007D07A8F380E0DF91CF911F910F9108955F
:1005600081E0F9CF4F925F926F927F928F929F922C
:10057000AF92BF92CF92DF92EF92FF920F931F93B1
:10058000CF93DF93CDB7DEB763970FB6F894DEBF96
:100590000FBECDBF7C016B013A01FB0120E090E072
:1005A00080E06AE03191332309F461C040ED430FEC
:1005B0004A3008F04DC0689FA001699F500D11247A
:1005C000CA01C097830F911D37FD9A958F3F910502
:1005D00049F340F3F7014281538164817581809131
:1005E000051790910617A0910717B09108174817A3
:1005F00059076A077B0709F40DC28701085F1F4F7F
:100600000E94DB816F7077277C5FC8010E94561BB8
:10061000813009F004C28CEF93E09A838983F7015B
:1006200082819381A481B5818B839C83AD83BE83BA
:1006300045E350E0BE016F5F7F4FC8010E94DF1BA2
:10064000892BA9F5D12CC12CC8010E94821817C092
:100650003E3209F0BFCF233009F4BCCFD301A20F43
:10066000B11D12968C932F5F90E080E09BCF2330DA
:1006700009F0B0CFF3018583CC24C394D12CC601FB
:1006800063960FB6F894DEBF0FBECDBFDF91CF915A
:100690001F910F91FF90EF90DF90CF90BF90AF90A0
:1006A0009F908F907F906F905F904F9008950E94E1
:1006B000DB81F7017783668342E050E0B7016A5F30
:1006C0007F4FC8010E94741B81E090E09A83898368
:1006D00042E050E0BE016F5F7F4FC8010E94741B73
:1006E00080E091E09A83898342E050E0BE016F5F31
:1006F0007F4FC8010E94741B1A82198242E050E0A9
:10070000BE016F5F7F4FC8010E94741B42E050E042
:10071000BE016F5F7F4FC8010E94741B42E050E032
:10072000BE016F5F7F4FC8010E94741B5601F60126
:100730008081882301F16501F60181912F018823D1
:1007400011F08E32B1F446018A189B08181419046E
:1007500074F48D8641E050E0BE01635F7F4FC801B5
:100760000E94741BA401B501C8010E94741B5201B0
:10077000DECF6201E1CF1D8641E050E0BE01635F44
:100780007F4FC8010E94741BC12CDD24D394DA82F0
:10079000C98242E050E0BE016F5F7F4FC8010E94F6
:1007A000741BDA82C98242E050E0BE016F5F7F4F66
:1007B000C8010E94741BC8010E94AE1B892B09F45A
:1007C00041CFF3E0AF2EB12C230122E0420E511CA9
:1007D000D4C0F7014281538164817581808D918DF0
:1007E000A28DB38D481759076A077B0709F008C126
:1007F000848D958DC59709F003C181A192A15DEF0C
:10080000C52EDD24DA940C970CF4ADC04CE050E01A
:10081000BE016F5F7F4FC8010E9461178B819C8171
:100820009827892798279A8B898BF70146815781CA
:1008300029813A814217530709F0E7C097FFE5C0C5
:100840008F7092703BEFC32EDD24DA94892B09F070
:100850008AC06F8078847624672476242AEFC22E9B
:10086000DD24DA946114710409F47DC0D12CC12C0B
:100870008D819E81982789279827C816D906F8F474
:1008800041E050E0BE01635F7F4FC8010E946117E5
:100890004D85442331F050E070E060E0C8010E94D3
:1008A00061178D858111ECCF44E050E070E060E08D
:1008B000C8010E946117FFEFCF1ADF0AD9CF912C30
:1008C000812C41E050E0BE016D5E7F4FC8010E9467
:1008D00061174B89842F807C09F06CC0442331F070
:1008E00050E070E060E0C8010E9461178B898111BF
:1008F000E8CF42E050E0BE01615F7F4FC8010E9437
:10090000611742E050E0BE01635F7F4FC8010E9463
:10091000611744E050E070E060E0C8010E94611798
:1009200042E050E0BE016F5E7F4FC8010E94611738
:100930008F85988949895A898115914009F043C06A
:10094000CD84DE84DC24CD24DC2481E0C816D104EF
:10095000D1F54115544009F04AC044E050E0B201DD
:10096000C8010E94611721E0A21AB10809F46CCEF7
:10097000FFEFCF16DF0609F067CE0E94DB813B0157
:100980004C01C8010E94AA17181619060CF421CFB1
:100990000E94DB81661977098809990969387341D2
:1009A0008105910548F562E370E080E090E00E94E7
:1009B0000C7FE7CF41E050E070E060E0C8010E94AA
:1009C00061171B8A93CF54274527542770E060E0B6
:1009D000C8010E946117FFEF8F1A9F0A68147904FB
:1009E00009F06FCF96EFC92EDD24DA94BCCFE7EF84
:1009F000CE2EDD24DA94B7CFCC24CA94DC2CB3CF2E
:100A00006EEFC62EDD24DA94AECF4CEFC42EDD247B
:100A1000DA94A9CF8EEFC82EDD24DA9430CED12C13
:100A2000C12C2DCE1F920F920FB60F9211242F932F
:100A30003F938F939F93AF93BF938091C5159091F0
:100A4000C615A091C715B091C8153091C41523E003
:100A5000230F2D3758F50196A11DB11D2093C41504
:100A60008093C5159093C615A093C715B093C8156C
:100A70008091C9159091CA15A091CB15B091CC1554
:100A80000196A11DB11D8093C9159093CA15A0931D
:100A9000CB15B093CC15BF91AF919F918F913F91A2
:100AA0002F910F900FBE0F901F90189526E8230FDF
:100AB0000296A11DB11DD2CF1F920F920FB60F92B9
:100AC00011240BB60F922F933F934F935F936F9325
:100AD0007F938F939F93AF93BF93EF93FF9348E2DE
:100AE00051E064E271E090E080E00E94C77DFF91F8
:100AF000EF91BF91AF919F918F917F916F915F9196
:100B00004F913F912F910F900BBE0F900FBE0F9002
:100B10001F9018951F920F920FB60F9211240BB6CB
:100B20000F922F933F934F935F936F937F938F9386
:100B30009F93AF93BF93EF93FF9348EA50E064EA2B
:100B400070E083E090E00E94C77DFF91EF91BF913C
:100B5000AF919F918F917F916F915F914F913F9155
:100B60002F910F900BBE0F900FBE0F901F901895F6
:100B70001F920F920FB60F9211240BB60F922F9364
:100B80003F934F935F936F937F938F939F93AF9315
:100B9000BF93EF93FF9348E950E064E970E082E08F
:100BA00090E00E94C77DFF91EF91BF91AF919F911F
:100BB0008F917F916F915F914F913F912F910F9006
:100BC0000BBE0F900FBE0F901F9018951F920F92A3
:100BD0000FB60F9211240BB60F922F933F934F93A2
:100BE0005F936F937F938F939F93AF93BF93EF9395
:100BF000FF9348E850E064E870E081E090E00E94F4
:100C0000C77DFF91EF91BF91AF919F918F917F91A0
:100C10006F915F914F913F912F910F900BBE0F906D
:100C20000FBE0F901F9018956093BC157093BD1563
:100C30008093BE159093BF15645D7E4F8F4F9F4F7D
:100C40006093B8157093B9158093BA159093BB153E
:100C500082E090E09093B7158093B6150E94DB81F7
:100C60006093B2157093B3158093B4159093B51536
:100C70000895CF92DF92EF92FF920F931F930E94FD
:100C8000DB818B019C01C090B215D090B315E09030
:100C9000B415F090B5156091BC157091BD1580919B
:100CA000BE159091BF150C191D092E093F09083E6C
:100CB000134021053105E0F0DC01CB010196A11DB7
:100CC000B11D8093BC159093BD15A093BE15B09334
:100CD000BF15B701A60148515C4F6F4F7F4F40933E
:100CE000B2155093B3156093B4157093B515C7CF73
:100CF0001F910F91FF90EF90DF90CF9008954F924A
:100D00005F926F927F928F929F92AF92BF92CF929B
:100D1000DF92EF92FF920F931F93CF93DF934B01DC
:100D20005C018091AE159091AF15A091B015B09176
:100D3000B11588159905AA05BB0509F4C6C08CE351
:100D4000C82ED12CE12CF12CC501A70196010E94DF
:100D5000D6A96093310CCA01B901A70196010E947E
:100D6000D6A96093320CC501B40120E13EE040E019
:100D700050E00E94D6A9CA01B90128E130E040E064
:100D800050E00E94D6A96093330CC501B40120E85D
:100D900031E541E050E00E94D6A969017A01CA011B
:100DA000B9016C5F7F4F8F4F9F4F27E030E040E0ED
:100DB00050E00E94D6A96F5F6093340C412C512CF7
:100DC000320140E004E610E0C0E9D1E0242F30E039
:100DD0002E54384FF901E370FF273097F9F4C90119
:100DE000B8010E9464AB892B31F4C901BE010E9495
:100DF00064AB892B99F48EE691E0A0E0B0E0480E58
:100E0000591E6A1E7B1ED301C201AA27BB27C81622
:100E1000D906EA06FB0638F04F5FD8CF8DE691E0A1
:100E2000A0E0B0E0ECCF4093370CC90164E670E07D
:100E30000E9464ABEC01C90160E971E00E9464ABFF
:100E4000309721F42097D9F40097C9F04DE651E08E
:100E500060E070E0441A550A660A770AC418D5089B
:100E6000E608F708A3E2B3E020E0213069F4309708
:100E7000E9F5209711F40097C9F54DE106C04EE65B
:100E800051E060E070E0E6CF4C9150E070E060E04F
:100E900031E0320FC416D506E606F70640F0C41A54
:100EA000D50AE60AF70A1196232F3C30F1F62F5F98
:100EB0002093360CC394C092350C8092AE1590925C
:100EC000AF15A092B015B092B115DF91CF911F91DF
:100ED0000F91FF90EF90DF90CF90BF90AF909F90D9
:100EE0008F907F906F905F904F9008954CE1CDCFA1
:100EF0000E9439860E947F868091370C90E08E5444
:100F0000984F08950E9439860E947F868091360C02
:100F100090E008950E9439860E947F868091350C6A
:100F200090E008950E9439860E947F868091320C5D
:100F300090E008950E9439860E947F868091330C4C
:100F400090E008951F920F920FB60F9211240BB6E6
:100F50000F922F933F934F935F936F937F938F9352
:100F60009F93AF93BF93EF93FF938091DE140E9402
:100F700049742091E1143091E2142F5F3F4F309378
:100F8000E2142093E1149091E014953618F096E065
:100F90009093DD149091DD14943009F46EC0F8F450
:100FA000923031F1933009F44CC09091DF149923C1
:100FB00019F0811171C02F9AFF91EF91BF91AF91FC
:100FC0009F918F917F916F915F914F913F912F9161
:100FD0000F900BBE0F900FBE0F901F90189595307D
:100FE00009F457C0963009F791E09093AD154FC0C2
:100FF0008111DBCF2091E1143091E21424363105C8
:1010000028F41092E2141092E114CFCF1092AD1593
:101010001092E014E091E01491E09E0F9093E014A0
:10102000F0E02091E1143091E214EE0FFF1FED513A
:10103000FB4E318320831092E2141092E11493E06E
:1010400019C0813009F0B1CFE091E01491E09E0F1A
:101050009093E014F0E02091E1143091E214EE0F4F
:10106000FF1FED51FB4E318320831092E21410924A
:10107000E11494E09093DD1498CF882359F22091E5
:10108000E1143091E2142536310508F48ECF95E055
:10109000F1CF81118ACFB5CF2F988ECFCF93DF9329
:1010A00091E0909399148823B9F0C091B800D09141
:1010B000BA008091BC008A7B8093BC0060E084E130
:1010C0000E94997D60E085E10E94997D0E94817E69
:1010D000D093BA00C093B800DF91CF9108958F925A
:1010E0009F92AF92BF92CF92DF92EF92FF920F93B7
:1010F0001F93CF93DF93D091E20ED13208F0D7C087
:10110000182FC091E10E0E94E77E6B017C01809157
:10111000D90E81116BC082E08093D90E1093D80E46
:101120008FEF8093D70E1092D60ED093D50EAFEBE3
:10113000B6E1E5EBFEE080E0D81391C01092B40E6A
:101140008091B40ECC0FC82BC093B40E8091B30E17
:10115000813009F088C01092B30E0E94E77E6B01C7
:101160007C018091B40E8093BB008091DB0E909146
:10117000DC0EA091DD0EB091DE0E892B8A2B8B2B1D
:10118000A1F00E94E77E0091DB0E1091DC0E209111
:10119000DD0E3091DE0E6C197D098E099F09061750
:1011A00017072807390708F442C08091BC0083FD67
:1011B000D8CF85EC8093BC000E94E77E6B017C0158
:1011C0008091D90E823009F450C08091D70E8F3FA4
:1011D00009F46FC08091D70E803209F46CC0809101
:1011E000D70E803309F469C084E026C08091DB0EFD
:1011F0009091DC0EA091DD0EB091DE0E892B8A2B32
:101200008B2B09F484CF0E94E77E8090DB0E9090B8
:10121000DC0EA090DD0EB090DE0E6C197D098E09FB
:101220009F0986169706A806B90608F070CF809128
:10123000DA0E0E944E8885E01092E00E1092E20EC7
:101240001092DF0EDF91CF911F910F91FF90EF90E1
:10125000DF90CF90BF90AF909F908F9008959D9119
:1012600091938F5F69CF85EEA5CF8091DB0E909132
:10127000DC0EA091DD0EB091DE0E892B8A2B8B2B1C
:1012800009F49ECF0E94E77E0091DB0E1091DC0EE8
:101290002091DD0E3091DE0E6C197D098E099F09BB
:1012A000061717072807390708F08ACFC0CF81E053
:1012B000C3CF80E0C1CF82E0BFCF83E0BDCFFC01D0
:1012C000248131E03093DF0E2093E10E1092E00E86
:1012D0001092E20E8385682B8EE190E10E94EF74FC
:1012E00081E00C946F880F931F93CF938C01C62FCE
:1012F0000E945F896C2F6460C8010E945F896C2F17
:101300006B7FC8010E945F8983EC90E00197F1F741
:10131000CF911F910F910895CF93C82F682F607FB1
:1013200083E894E10E94738980E1C89FB001112491
:1013300083E894E1CF910C947389CF93DF9300D02D
:1013400000D01F921F92CDB7DEB798E0E9E1F3E03D
:10135000DE01119601900D929A95E1F790918C140F
:10136000961708F46FEF70E0660F771F21E030E00A
:101370002C0F3D1F620F731FFB019081890F806846
:1013800028960FB6F894DEBF0FBECDBFDF91CF9188
:101390000C948C890F931F93CF93DF932091DE02DF
:1013A000222321F12091DD02222301F1EB018C01A6
:1013B00061E080E00E949D89B80183E894E10E9489
:1013C000877C6BE27DE083E894E10E94A97C61E088
:1013D000F80184810E949D89BE01DD0F880B990B65
:1013E000DF91CF911F910F910C940C7FDF91CF91E2
:1013F0001F910F9108950F931F93CF938C01C62FC8
:10140000607F61600E94738980E1C89FB0011124F0
:101410006160C8010E94738981E090E0CF911F91C3
:101420000F91089585ED8093BC008091DB0E909123
:10143000DC0EA091DD0EB091DE0E0796A11DB11D50
:1014400023E0B695A795979587952A95D1F7209192
:10145000BC0024FD03C01092D90E08954091DB0E0C
:101460005091DC0E6091DD0E7091DE0E452B462B07
:10147000472B69F30097A105B10541F025E32A95B3
:10148000F1F700000197A109B109E1CF8091DA0ECF
:101490000C944E881F920F920FB60F9211240BB628
:1014A0000F922F933F934F935F936F937F938F93FD
:1014B0009F93AF93BF93EF93FF938091B900887F81
:1014C000803609F44DC008F040C0883209F4A9C044
:1014D00028F5803109F49DC0C8F4882309F4FBC0C5
:1014E000883009F496C0FF91EF91BF91AF919F9121
:1014F0008F917F916F915F914F913F912F910F90BD
:101500000BBE0F900FBE0F901F901895883109F4F5
:1015100088C0803241F78093D70E14C0803409F41C
:101520009DC040F48033B9F38833E9F68093D70E39
:1015300085ECB0C0803509F485C0883509F496C0C3
:10154000883489F60E94128ACECF883909F48CC07B
:1015500038F5883729F050F4883611F0803719F6BD
:1015600083E08093D90E1092DC1457C0883809F4B8
:101570007BC0803919F0803809F0B5CF8091DC1438
:10158000803208F071C0E091DC1481E08E0F80930E
:10159000DC148091BB00F0E0E454FB4E80833DC03E
:1015A000803B39F0E0F4803A09F479C0883A09F0D8
:1015B0009ACF84E08093D90E1092BB141092BA1483
:1015C000E0915116F091521619958091BA1481113B
:1015D0000FC081E08093BA1410929A1409C0803C25
:1015E00009F4A6CF883C09F4A3CF883B09F07BCF50
:1015F000E091BB1481E08E0F8093BB14F0E0E656BF
:10160000FB4E80818093BB009091BB148091BA14F3
:1016100029C08091B40E8093BB0085EC8093BC0000
:1016200062CF9091D60E8091D50E981758F5E09123
:10163000D60E81E08E0F8093D60EF0E0EB54F14F82
:101640008081E9CFE091D60E81E08E0F8093D60E97
:101650008091BB00F0E0EB54F14F80839091D60E67
:101660008091D50E9817C8F285E8D8CFE091D60EB4
:1016700081E08E0F8093D60E8091BB00F0E0EB549A
:10168000F14F80838091D80E81115CCF81E08093EF
:10169000B30E84EA8093BC001092D90E24CF85EC5F
:1016A0008093BC001092D90E8091DC14803230F40B
:1016B000E091DC14F0E0E454FB4E10826091DC1405
:1016C00070E0E0914F16F09150168CEB94E1199573
:1016D0001092DC1408CF1092D70E34CF8091100CEA
:1016E0008823A9F140919E0250919F026091A0022F
:1016F0007091A1022FEA3CE080915316909154160C
:101700000E945C11811102C080E0089540919514FF
:101710005091961460919714709198144115510549
:101720006105710591F02FEA3CE08091531690918C
:1017300054160E945C11882339F31092951410926C
:10174000961410929714109298141092100C81E035
:1017500008958F929F92AF92BF92EF92FF920F9354
:101760001F93CF934B015C01C42F80919E029091F7
:101770009F02A091A002B091A10288159905AA0527
:10178000BB0549F10E946E8B81110BC080E0CF91A7
:101790001F910F91FF90EF90BF90AF909F908F900F
:1017A00008958FEAE82E8CE0F82E00E012E030E099
:1017B00020E0B501A40180915316909154160E9427
:1017C000B510882319F380929E0290929F02A092F6
:1017D000A002B092A1024091100C4C2B4093100C2F
:1017E00081E0D5CFCF93DF93EC016E857F8588892B
:1017F000998941E00E94A98B882351F08A8920E2CF
:10180000829FC00111248155934FDF91CF9108959C
:1018100090E080E0FACF8F929F92AF92BF92CF92EA
:10182000DF92EF92FF92CF932AE230E13093541689
:1018300020935316882309F46DC040E060E070E007
:10184000CB010E94A98B81110BC080E0CF91FF904A
:10185000EF90DF90CF90BF90AF909F908F900895C2
:1018600080916D0E8F7789F78091790E90917A0E25
:10187000A0917B0EB0917C0E84369105A105B10537
:1018800020F3C090750ED090760EE090770EF09019
:10189000780EC114D104E104F104B9F240E0C701AB
:1018A000B6010E94A98B882381F28091BA0C909195
:1018B000BB0C8115924049F6A091BF0CAA2329F2D6
:1018C0006091BD0C7091BE0C6115710509F4BDCF1E
:1018D0002091BC0C222309F4B8CFA0934810209388
:1018E0003A1090E080E030E0E1E0F0E0C82FAF0196
:1018F000082E02C0440F551F0A94E2F7241735073B
:1019000069F041E0480F01968930910579F74093DD
:1019100043109BCFC12CD12C7601C0CF80934310B4
:101920002091C50C3091C60C50E040E021153105E6
:1019300041F42091D30C3091D40C4091D50C5091AE
:10194000D60C20933B1030933C1040933D105093A5
:101950003E1046015701860E971EA11CB11C8092B5
:10196000491090924A10A0924B10B0924C10E09106
:10197000C00CF091C10CF0934F10E0934E10B0E00A
:101980000E9417AADC01CB01880D991DAA1DBB1D61
:101990008093501090935110A0935210B093531015
:1019A00025E0EE0FFF1F2A95E1F7E150FE4FEF2FE4
:1019B000FF27E6958E0F9F1FA11DB11D8093441038
:1019C00090934510A0934610B09347108090C20C9E
:1019D0009090C30CB12CA12C8114910441F48090FF
:1019E000CF0C9090D00CA090D10CB090D20CC81A13
:1019F000D90AEA0AFB0AC80CD91CEA1CFB1C04C061
:101A0000F694E794D794C794CA95D2F7C0923F1042
:101A1000D0924010E0924110F092421085EFC8162B
:101A20008FE0D806E104F10428F48CE080934D1097
:101A300081E00CCF80E125EFC2162FEFD206E10442
:101A4000F104A0F38091DB0C9091DC0CA091DD0CF3
:101A5000B091DE0C8093501090935110A0935210CF
:101A6000B093531080E2E2CF4F925F926F927F92D9
:101A70008F929F92AF92BF92CF92DF92EF92FF929E
:101A80000F931F93CF93DF93EC0142305105610513
:101A9000710590F480E0DF91CF911F910F91FF903D
:101AA000EF90DF90CF90BF90AF909F908F907F90FE
:101AB0006F905F904F90089589859A85AB85BC851E
:101AC0000196A11DB11D84179507A607B70710F34E
:101AD000CB88DC88ED88FE888F89803109F042C090
:101AE000BB27A72F962F852F480159012A013B01BB
:101AF000C80ED91EEA1EFB1E80919E0290919F0285
:101B0000A091A002B091A102C816D906EA06FB0670
:101B100099F58F898031C1F5B301A2015527662758
:101B20007727440F551F4155534FFA019182808208
:101B30008091100C81608093100C8A89823080F033
:101B40008D819E81AF81B8858C0D9D1DAE1DBF1D01
:101B50008093951490939614A0939714B09398142F
:101B600081E099CFDB01CA01E7E0B695A79597958B
:101B70008795EA95D1F7B8CF40E0C701B6010E943A
:101B8000A98B8111C6CF86CFB301A2014F7755270C
:101B900066277727440F551F440F551F4155534F54
:101BA000FA0180829182A282B382C2CF8F929F92E9
:101BB000AF92BF92CF92DF92EF92FF920F931F935B
:101BC000CF93DF93FC0181859285A385B48501962F
:101BD000A11DB11D84179507A607B70770F480E013
:101BE000DF91CF911F910F91FF90EF90DF90CF90F9
:101BF000BF90AF909F908F90089583889488A58818
:101C0000B6888789803189F5BB27A72F962F852F26
